:100000000C94440F0C94650F0C94650F0C94650FC1
:100010000C94650F0C94650F0C94650F0C94650F90
:100020000C94650F0C94650F0C94FB650C9418668A
:100030000C94650F0C94650F0C94D9660C940667AC
:100040000C9433670C9460670C948D670C94BA67BA
:100050000C94E7670C9414680C9441680C946E68D7
:100060000C94650F0D9448240D947F240C94650F17
:100070000C94650F0C94650F0C94650F0C94650F30
:100080000C94650F0C94650F0C94650F0C94650F20
:100090000C94650F0C94650F0C94650F0D947C4FB8
:1000A0000D94AE4F0D94E04F0D9412500D945F00DF
:1000B0000C94650F0C94650F0C94650F0C945D6A9D
:1000C0000C948A6A0C94B76A0C94E46A0C94116BD1
:1000D0000C943E6B0C946B6B0C94986B0C94C56BEE
:1000E0000C94F26B0C94650F0D946C230D94A32368
:1000F0000C94650F0C94650F0C94650F0C94650FB0
:100100000C94650F0C94650F0D9439050C94650FD4
:100110000C94650F0C94650F0C94650F0D94B44E00
:100120000D94E64E0D94184F0D944A4F0C94650FA4
:100130000C94650F0C949B680C94C8680C94F5683B
:100140000C9422690C944F690C947C690C94A969F5
:100150000C94D6690C94036A0C94306A0C94650F65
:100160000D94DA230D9411240C94650F0C94650FF3
:100170000C94650F0C94650F0C94650F0C94650F2F
:100180000C94650F0C94650F0C94650F0C94650F1F
:100190000C94650F0C94650F0C94650F0C94650F0F
:1001A0000D942C000C94650F0C94650F0C94650F46
:1001B0000C941F6C0C944C6C0C94796C0C94A66C85
:1001C0000C94D36C0C94006D0C94650F0C94650F1B
:1001D0000C94650F0C94650F0C94650F0D94B62468
:1001E0000D94ED240C94650F0C94650F0C94650F21
:1001F0000C94650F0C9498780C9453791E10A110F0
:100200003010A1104210A11054106E10541088101C
:1002100088104F12631277129D12C3123E132B13D4
:100220003E1305130513DA18DA1812194F1993192A
:10023000D0187C1A981AD51A331A331A981A7C1ABD
:1002400093194F191219DA18DA188D229722A12260
:10025000AB22B522BF22C922CE22D322DD22DD224B
:10026000CE22C922B522AB22A12297228D22A52718
:10027000A527AC27AC27BF27E227A527E227AC2775
:10028000AC27A527E227AC27AC27A527A5271B2845
:100290001B282328232838285F281B285F28232889
:1002A00023281B285F28232823281B281B286F2886
:1002B0001029982810291029E9281029C128C128B7
:1002C000E9281029982810296F2843294E295D29EB
:1002D00078298E29B029F629FF291A2AD629D62964
:1002E000FF29F6298E2978295D294E2943290F5F98
:1002F000865F865F9F5E865F865F865F865F865FBE
:10030000865F865F865F865F865F865F865F865FC5
:10031000865FB45E865F865F865F865F865F865F88
:10032000865F095F675F865F865F745F865F865F53
:10033000865F865F865F865F225F865F865F805FFF
:10034000865F835F865F865F865F865F7D5F865F91
:10035000865F865F865F865F865F865F865F865F75
:10036000865F865F865F865F865F865F865F865F65
:10037000865F865F865F865F865F865F865F865F55
:10038000865F865F865F865F865F865F865F865F45
:10039000865F865F865F865F865F865F865F865F35
:1003A000865F0C5F6C736F737273757378737B7396
:1003B0007E73EB7AFE7A117B247B377B4A7B5D7BF5
:1003C00065806580E27F278027809A7F9A7F2780DB
:1003D00027802780278027802780278027802780E5
:1003E0002780278027802780278027809A7F278063
:1003F00027802780278027807185B186AC85DB85A3
:10040000B186B186B186B186B186B186B186B18634
:10041000B186B186B186B186B186B186B186B18624
:10042000B186B186B186B186B186B186B186B18614
:10043000B186B186B186B186B186B186B186B18604
:10044000B186B186B186B186B186B186B186B186F4
:10045000B186B186B186B186B1865686B1861586DB
:10046000B186B1867186B186B186B186B186B18614
:10047000B186B186B186B186B186B1862486B18651
:1004800032863A906A8EA38EED8E538F9E8FB38FF5
:10049000E58F07902890ED917A9082909F90DE9062
:1004A000F1903B915D9174918991E891E891E89187
:1004B000E891E891E891E891E891E891E891A091BC
:1004C000A891B391C891CE918EAEBEAE6AAE76AE13
:1004D000BEAEBEAEBEAEBEAEBEAEBEAEBEAEBEAEBC
:1004E000BEAEBEAEBEAEBEAEBEAEBEAE82AEBEAEE8
:1004F000BEAEBEAEBEAEBEAEBEAEBEAEBEAEBEAE9C
:10050000BEAEBEAEBEAEBEAE8EAEBEAE6AAE76AE57
:10051000BEAEBEAEBEAEBEAEBEAEBEAEBEAEBEAE7B
:10052000BEAEBEAEBEAEBEAEBEAEBEAE82AEF5B965
:10053000F8B949BA49BA49BA49BA49BA49BA49BAF5
:1005400049BA49BA49BA49BA49BA49BA49BA49BA93
:1005500049BA49BA49BA49BA2FBA49BA49BA49BA9D
:1005600049BA49BA49BA15BA49BA49BA49BA49BAA7
:1005700049BAFBB949BA49BA49BA49BA49BA49BAB2
:1005800049BA49BA49BA49BA49BA49BA49BA49BA53
:1005900049BA49BA49BA49BA2FBA49BA49BA49BA5D
:1005A00049BA49BA49BA15BA49BA49BA49BA49BA67
:1005B00049BAFBB9F2BCEFBC04BD04BD04BD04BD27
:1005C00004BD04BD04BD04BD04BD04BD04BD04BD23
:1005D00004BD04BD04BD3BBC0EBC2CBC04BD04BDAD
:1005E000B2BCF5BB04BD04BD04BD04BD04BD1DBC4F
:1005F000F5BC04BD04BD45BC04BD04BD04BD04BDC3
:1006000004BD04BD04BD04BD04BD04BD04BD04BDE2
:1006100004BD04BD04BD3BBC0EBC2CBC04BD04BD6C
:10062000B2BCF5BB04BD04BD04BD04BD04BD1DBC0E
:10063000F5BC04BD04BD45BCF7BF3AC049C049C0C4
:1006400049C049C049C049C049C049C049C049C062
:1006500049C049C049C02ABF49C0E1BFDBBF43BF51
:10066000F1BF49C049C053BF2ABF49C049C006C0F5
:1006700037BFEBBF3FC0E7BF49BFFCBFD5BF4EBFD1
:1006800049C001C026BF44C049C049C03DBF49C0A0
:1006900049C049C049C049C049C0E1BFDBBF43BFF1
:1006A000F1BF49C049C053BF2ABF49C049C006C0B5
:1006B00037BFEBBF3FC0E7BF49BFFCBFD5BF4EBF91
:1006C00049C001C026BF44C049C049C03DBF06BFA4
:1006D00069C559C55BC55DC55FC561C563C565C5F0
:1006E00086C576C578C57AC57CC57EC580C582C5F8
:1006F00093C5C1C59BC5C1C59BC5C1C59BC5C1C56A
:100700009BC5C1C59BC5C1C5C1C5C1C5C1C5C1C505
:10071000C1C5C1C5A2C5A9C5B5C5B5C5F1D820D744
:100720002CD777D7A8D88CD7CED7F2D71BD876D8E6
:10073000A8DFA8DF32E06AE14AE272E35CE44AE55E
:100740005CE496E696E64AE55CE44AE26AE132E079
:10075000A8DFA8DFCCE8CCE80DE96BE9AAE9F8E965
:100760002DEA6CEA2DEABAEABAEA6CEA2DEAAAE9BD
:100770006BE90DE9CCE8CCE817ED82EDEDEDA6EEE6
:1007800052EF42F02BF1E2F12BF1E3F2E3F2E2F16E
:100790002BF152EFA6EEEDED82ED17ED0D94C410A6
:1007A0000D9402100D9437110D94B7110D949F11F3
:1007B0000D941D124E414E494E495459494E46CD55
:1007C000CCCC3D0AD7233C17B7D13877CC2B329508
:1007D00095E6241FB14F0A000020410000C84200E6
:1007E000401C4620BCBE4CCA1B0E5AAEC59D74327E
:1007F00035304D4F686D0032354D4F686D003630E5
:10080000487A003530487A004E6F6E2D496E74007C
:1008100048692D4C4F004750530054696D650044A2
:10082000697374616E6365005075736820427574F6
:10083000746F6E00496D70657269616C004D65740E
:1008400072696300494E4300444543004F4E004FD8
:100850004646005B0956094C094509390932092603
:100860000915090709F408E108CC08BB08A8089A8B
:10087000088B08810877084349505326414356475F
:1008800000444356472641435647004349505326A8
:10089000444356472641435647003278444356471F
:1008A0002632784143564700434950532632784414
:1008B00043564726327841435647003278496D7097
:1008C0002E20434950532641435647003278496D04
:1008D000702E4349505326444356472641435647BA
:1008E00000327843495053263278444356472641D4
:1008F000435647003278496D702E204349505326A5
:1009000032784443564700506172616C6C656C20CC
:1009100043495053003278496D702E20434950535B
:100920002644435647003278496D702E2043495083
:100930005300347844435647004349505326327895
:100940004443564700327844435647004349505386
:1009500026444356470044435647004349505300FA
:100960002B126911A710E50F230F610E9F0DDD0CEF
:100970001B0C590BF80ADD0C9F0D230FE50FA71078
:1009800069112B128C12CA1108114610840FC20E65
:10099000000E3E0D7C0CBA0BF80A3E0D000E840FC3
:1009A00046100811CA118C1253616D706C652F735B
:1009B00065633A004552524F5220202020202000EB
:1009C000432D434950532C20522D434950532C2042
:1009D0000000000000000000000000000000000017
:1009E0000000000000000000000000000000000007
:1009F00000000000000000000000000000000000F7
:100A000000000000000000000000000000000000E6
:100A100000000000000000000000000000000000D6
:100A2000004C6F2D434950532C2048692D434950A9
:100A3000532C200000000000000000000000000017
:100A400000000000000000000000000000000000A6
:100A50000000000000000000000000000000000096
:100A60000000000000000000000000000000000086
:100A70000000000000000000000000000000000076
:100A80000000434950532C200000000000000000EB
:100A90000000000000000000000000000000000056
:100AA0000000000000000000000000000000000046
:100AB0000000000000000000000000000000000036
:100AC0000000000000000000000000000000000026
:100AD0000000000000000000000000000000000016
:100AE0000000004143564752506F6C2C2041435642
:100AF0004752526D732C2000414356474C506F6C47
:100B00002C20414356474C526D732C20414356478D
:100B100052506F6C2C204143564752526D732C201B
:100B200000000000000000000000000000000000C5
:100B300000000000000000000000000000000000B5
:100B400000000000000000000000000000000000A5
:100B5000000000000000000000522D4443564720D2
:100B60004F6E2C204C2D44435647204F6E2C204C6A
:100B70006F2D43495053204F6E2C2048692D434917
:100B80005053204F6E2C20522D44435647204F6621
:100B9000662C204C2D44435647204F66662C204C33
:100BA0006F2D43495053204F66662C2048692D43D2
:100BB000495053204F66662C2000522D444356471F
:100BC000204F66662C204C2D44435647204F6666C6
:100BD0002C204C6F2D43495053204F66662C2048E3
:100BE000692D43495053204F66662C20522D4443B3
:100BF0005647204F6E2C204C2D44435647204F6EB5
:100C00002C204C6F2D43495053204F6E2C204869A7
:100C10002D43495053204F6E2C2000432D43495003
:100C200053204F6E2C20522D43495053204F6E2C91
:100C300020432D43495053204F66662C20522D43AC
:100C4000495053204F66662C200000000000000031
:100C50000000000000000000000000000000000094
:100C60000000000000000000000000000000000084
:100C7000000000000000000000000000432D434978
:100C80005053204F66662C20522D43495053204F1D
:100C900066662C20432D43495053204F6E2C205222
:100CA0002D43495053204F6E2C20000000000000BF
:100CB0000000000000000000000000000000000034
:100CC0000000000000000000000000000000000024
:100CD00000000000000000000000000000522D4451
:100CE000435647204F6E2C204C6F2D4349505320C4
:100CF0004F6E2C2048692D43495053204F6E2C20B5
:100D0000522D44435647204F66662C204C6F2D438E
:100D1000495053204F66662C2048692D4349505353
:100D2000204F66662C20000000000000000000003C
:100D30000000000000000000000000000000522D34
:100D400044435647204F66662C204C6F2D43495034
:100D500053204F66662C2048692D43495053204F3D
:100D600066662C20522D44435647204F6E2C204C53
:100D70006F2D43495053204F6E2C2048692D434915
:100D80005053204F6E2C2000000000000000000097
:100D90000000000000000000000000000000004C07
:100DA0006F2D43495053204F6E2C2048692D4349E5
:100DB0005053204F6E2C204C6F2D43495053204FE1
:100DC00066662C2048692D43495053204F66662C97
:100DD00020000000000000000000000000000000F3
:100DE0000000000000000000000000000000000003
:100DF00000000000000000000000000000000000F3
:100E00004C6F2D43495053204F66662C2048692D66
:100E100043495053204F66662C204C6F2D43495058
:100E200053204F6E2C2048692D43495053204F6E5C
:100E30002C20000000000000000000000000000066
:100E400000000000000000000000000000000000A2
:100E50000000000000000000000000000000000092
:100E600000522D44435647204F6E2C204C2D4443B6
:100E70005647204F6E2C20462D44435647204F6E38
:100E80002C20422D44435647204F6E2C20522D4497
:100E9000435647204F66662C204C2D44435647202E
:100EA0004F66662C20462D44435647204F66662CDD
:100EB00020422D44435647204F66662C20000000F8
:100EC0000000522D44435647204F66662C204C2D7F
:100ED00044435647204F66662C20462D44435647D0
:100EE000204F66662C20422D44435647204F6666AD
:100EF0002C20522D44435647204F6E2C204C2D441D
:100F0000435647204F6E2C20462D44435647204FD2
:100F10006E2C20422D44435647204F6E2C2000005B
:100F2000000000522D44435647204F6E2C204C2D7C
:100F300044435647204F6E2C2043495053204F6E58
:100F40002C20522D44435647204F66662C204C2DB2
:100F500044435647204F66662C2043495053204F48
:100F600066662C2000000000000000000000000069
:100F70000000000000000000000000000000000071
:100F800000000000522D44435647204F66662C2037
:100F90004C2D44435647204F66662C2043495053FE
:100FA000204F66662C20522D44435647204F6E2C0E
:100FB000204C2D44435647204F6E2C20434950531C
:100FC000204F6E2C200000000000000000000000F8
:100FD0000000000000000000000000000000000011
:100FE0000000000000522D44435647204F6E2C2035
:100FF0004C2D44435647204F6E2C20522D444356CF
:1010000047204F66662C204C2D44435647204F66A0
:10101000662C20000000000000000000000000001E
:1010200000000000000000000000000000000000C0
:1010300000000000000000000000000000000000B0
:10104000000000000000522D44435647204F6666C2
:101050002C204C2D44435647204F66662C20522DA1
:1010600044435647204F6E2C204C2D444356472076
:101070004F6E2C2000000000000000000000000067
:101080000000000000000000000000000000000060
:101090000000000000000000000000000000000050
:1010A00000000000000000522D44435647204F6EC0
:1010B0002C2043495053204F6E2C20522D44435630
:1010C00047204F66662C2043495053204F66662CBC
:1010D00020000000000000000000000000000000F0
:1010E0000000000000000000000000000000000000
:1010F00000000000000000000000000000000000F0
:101100000000000000000000522D44435647204FCD
:1011100066662C2043495053204F66662C20522D82
:1011200044435647204F6E2C2043495053204F6E66
:101130002C20000000000000000000000000000063
:10114000000000000000000000000000000000009F
:10115000000000000000000000000000000000008F
:10116000000000000000000000522D4443564720BC
:101170004F6E2C20522D44435647204F66662C203C
:10118000000000000000000000000000000000005F
:10119000000000000000000000000000000000004F
:1011A000000000000000000000000000000000003F
:1011B000000000000000000000000000000000002F
:1011C00000000000000000000000522D444356477C
:1011D000204F66662C20522D44435647204F6E2CDC
:1011E00020000000000000000000000000000000DF
:1011F00000000000000000000000000000000000EF
:1012000000000000000000000000000000000000DE
:1012100000000000000000000000000000000000CE
:10122000000000000000000000000043495053206F
:101230004F6E2C2043495053204F66662C200000EF
:10124000000000000000000000000000000000009E
:10125000000000000000000000000000000000008E
:10126000000000000000000000000000000000007E
:10127000000000000000000000000000000000006E
:10128000000000000000000000000000434950532F
:10129000204F66662C2043495053204F6E2C20006F
:1012A000000000000000000000000000000000003E
:1012B000000000000000000000000000000000002E
:1012C000000000000000000000000000000000001E
:1012D000000000000000000000000000000000000E
:1012E0000000000000000000000000000044656CE9
:1012F00061792054696D653B0046696C65204E61DB
:101300006D653A2000436861696E6167652C200055
:10131000004C6F63616C54696D652C204C6F636188
:101320006C444D592C204C61742D4465672C204E23
:10133000532C204C6F6E2D4465672C2045572C2074
:10134000466978537461742C204E756D5361742C0A
:101350002050444F502C20416C745F4D2C2043682A
:101360006B2C20436F6D6D0000000000000000003A
:10137000000000000000000000000000000000006D
:1013800000000000000000000000000000004C6FA2
:1013900063616C54696D652C204C6F63616C444DC6
:1013A000592C204C61742D4465672C204C61742DA0
:1013B0004D696E2C204C61742D5365632C204E5367
:1013C0002C204C6F6E2D4465672C204C6F6E2D4D7C
:1013D000696E2C204C6F6E2D5365632C2045572C65
:1013E00020466978537461742C204E756D53617476
:1013F0002C2050444F502C20416C745F4D2C2043C6
:10140000686B2C20436F6D6D000000484558434FBA
:10141000524445522043414C4942482E54585400AE
:1014200000007777772E636174682D746563682E8A
:10143000636F6D0000000000004C494D4954454465
:10144000203930352D3835372D313035300000001A
:10145000434154484F44494320544543484E4F4C20
:101460004F47590000007B702C30302C662C007BDD
:10147000702C30302C657D007B702C30302C6F7DD3
:1014800000686369746F6F6C207061697220004539
:101490006E7465722050494E203A2000686369637B
:1014A0006F6E666967206E616D65200061742B62E6
:1014B00074642A007175697400736D6172745A00E6
:1014C00061742B72756E00456E74657220414356CF
:1014D00047202827462720666F722046726F6E7459
:1014E0002C2027422720666F72204261636B290AF5
:1014F0000D20616E6420737570706C79203332300A
:101500002B3634302073696E657761766520776994
:101510007468205065616B546F5065616B20766F05
:101520006C74616765206F6620302E385600456EFA
:101530007465722053434F504520766F6C74616719
:101540006520696E206D5620284E4E4E4E4E290065
:10155000456E746572204349505320766F6C7461F8
:10156000676520696E206D562A313020284E4E4E18
:101570004E4E2900456E74657220444356472076CE
:101580006F6C7461676520696E206D562A3130205A
:10159000284E4E4E4E4E2900CE15C715C315BF1509
:1015A000BB15B715A815A815432D53474E44205B0E
:1015B000352D3430565D00432D4200432D46004307
:1015C0002D5200432D4C00522D53474E4400432DC5
:1015D00053474E440020616E6420656E746572202E
:1015E000766F6C7461676520696E206D562A3130A4
:1015F00020284E4E4E4E4E2900506C65617365207A
:10160000636F6E6E65637420004572726F722C207A
:101610006D697373696E6720414443206E756D2058
:1016200028302D3729000A0D5363616C696E6743BA
:10163000616C6962204F66667365743A200045727A
:10164000726F722C20656E74657220766F6C746197
:10165000676520696E206D562A313020284E4E4E27
:101660004E4E29001217F316DD16D116AD169A1636
:10167000721643535B302F312F322F332F345D5B83
:1016800076767676765D202D204443205363616C18
:10169000696E672043616C6962004342202D2042DD
:1016A0006174746572792043616C696200435A5BAE
:1016B000302F312F322F332F345D202D2044432003
:1016C0005A65726F4F66667365742043616C696218
:1016D0000056202D20566E756D626572004C5B6958
:1016E0006E785D5B4F4E2F4F46465D202D204C653A
:1016F000647300416E6E202D205265616420414468
:10170000433120666F72206E6E207365636F6E6466
:10171000730041202D205265616420414443310013
:101720004552524F52004F4B0043415448205445BC
:10173000434820484558434F524445522056303183
:101740002E303700010002000300040005000600EF
:101750000A000C000F0014001E003C007800B400CA
:10176000F0002C01680100000000120002000100DE
:10177000B80B0F27010064006801100E010010274C
:101780001027102710271027102701000100010043
:101790000100F8010100010002000100F401000055
:1017A00000000100000000000A00F1D80000010064
:1017B0000100C8000000640064006400640064006C
:1017C0006400000000000000000050FE0000000067
:1017D0000000000001000000000001000000000007
:1017E0000A00000001000100020058020000FA0097
:1017F000FA00FA00FA00780078000000000000000B
:1018000001000000010001000000000001000100D3
:101810000080001900800019008000190080001964
:101820000080001900800019008000190080001954
:1018300000000100FF03E600E6007018621854186B
:101840004D18244A42494E2C39342C3100244A5335
:1018500041564500244A4153432C47504753412C9D
:101860003100244A4153432C4750524D432C310000
:10187000244A4153432C47504747412C31002450C0
:101880004D544B3636372A33350024504D544B33A4
:1018900031342C302C312C302C312C312C302C305C
:1018A0002C302C302C302C302C302C302C302C3058
:1018B0002C302C302C302C302A323900756E6C6F65
:1018C00067206C62616E64747261636B73746174BF
:1018D00061006C6F67206C62616E64747261636B2F
:1018E0007374617461206F6E74696D6520313000AE
:1018F000756E6C6F6720707372706F7361006C6FC0
:101900006720707372706F7361206F6E74696D659C
:1019100020313000646174756D207573657200202C
:10192000302E3020302E3020302E3020302E30001F
:1019300075736572646174756D2000646174756D92
:1019400020776773383400756E6C6F67206770613D
:101950006C6D006C6F67206770616C6D206F6E74CA
:10196000696D6520313000D019C119B219A3199BD6
:101970001982197519245047524D432C2C2C393695
:101980002C00245047524D432C412C2C3130302C0C
:101990002C2C2C2C2C2C2C2C2C2C00245047524D35
:1019A000434500245047524D4F2C5047524D542C24
:1019B0003000245047524D4F2C5047524D462C3149
:1019C00000245047524D4F2C47504753562C30005F
:1019D000245047524D4F2C2C3400311A221A131A1E
:1019E000041AF519E619445A203D200000000000B1
:1019F00000000000004459203D20000000000000CD
:101A0000000000004458203D2000000000000000BD
:101A1000000000466C6174203D20000000000000C2
:101A200000004D616A6F7241203D200000000000FF
:101A3000005354505220444154554D2E5458540094
:101A40007D1B701B631B561B491B3C1B2F1B221B42
:101A5000151B081BFB1AEE1AE11AD41AC71ABA1A78
:101A6000AD1AA01A931A861A791A6C1A414356476E
:101A70003220524D53203D200041435647312052E1
:101A80004D53203D200042415454202043616C209E
:101A90003D200041432020205343616C203D200025
:101AA00041432020205A43616C203D2000414443A3
:101AB00037205653636C203D200041444337205A61
:101AC00043616C203D200041444336205653636CF3
:101AD000203D200041444336205A43616C203D2084
:101AE0000041444335205653636C203D200041445F
:101AF0004335205A43616C203D200041444334204B
:101B00005653636C203D200041444334205A4361C6
:101B10006C203D200041444333205653636C203DEC
:101B2000200041444333205A43616C203D20004152
:101B3000444332205653636C203D200041444332DD
:101B4000205A43616C203D200041444331205653CC
:101B5000636C203D200041444331205A43616C2096
:101B60003D200041444330205653636C203D20000B
:101B700041444330205A43616C203D200046696C4B
:101B80006520496E646578203D20002B1E151EFFE0
:101B90001DE91DD31DBD1DA71D911D7B1D651D4F7D
:101BA0001D391D231D0D1DF71CE11CCB1CB51C9FF1
:101BB0001C891C731C5D1C471C311C1B1C051CEF65
:101BC0001BD91B454E44000000000000000000002F
:101BD0000000000000000000004443564720446518
:101BE000666563742056616C203D2000000000444F
:101BF0004356472044656665637420456E203D204A
:101C0000000000000053796E632054797065203D18
:101C10002000000000000000000000434950532055
:101C200052616E6765202B2F2D3556203D20000018
:101C30000047505320436F6F726420696E20444DFB
:101C400053203D200000004C6F63616C475053549B
:101C5000696D654F6666736574203D2000414320C1
:101C60004672657175656E6379203D200000000045
:101C700000000042726F6B656E5769726520416C9F
:101C800061726D203D200000004C6F7720506F7412
:101C900020416C61726D203D200000000000004971
:101CA0006E70757420496D706564616E6365203D6A
:101CB0002000000000444356474D44656C4F4E20C1
:101CC0003D20000000000000000000444356474D46
:101CD00044656C4F4646203D200000000000000097
:101CE0000043495053324D44656C4F4E203D200017
:101CF0000000000000000043495053324D44656C21
:101D00004F4646203D20000000000000004349509F
:101D100053314D44656C4F4E203D200000000000C3
:101D200000000043495053314D44656C4F464620F6
:101D30003D20000000000000005374617274576978
:101D40007468203D20000000000000000000004FEB
:101D5000666654696D65205B6D7365635D203D202B
:101D60000000000000546F74616C4379636C65205F
:101D70005B7365635D203D2000000054696D652044
:101D800056616C7565203D200000000000000000D9
:101D900000436861696E61676520446972656374B8
:101DA000696F6E203D200053746172742043686136
:101DB000696E616765203D20000000000044697382
:101DC00074616E63652056616C7565203D2000006E
:101DD0000000004D6561737572656D656E74205508
:101DE0006E697473203D20000053746F72616765E3
:101DF00020416374696F6E203D2000000000005395
:101E000075727665792054797065203D2000000058
:101E100000000000004F70657261746F72204E61A7
:101E20006D65203D2000000000000053757276654E
:101E300079204E616D65203D20000000000000000B
:101E40000054532D5453204F4E203D200054532D09
:101E50005453204F4646203D20004E4557205453B2
:101E6000204F4E203D20004E4557205453204F46D2
:101E700046203D20005453204F4E203D2000545317
:101E8000204F4646203D200011241FBECFEFCDBF7E
:101E9000DFE5DEBF00E00CBF1FE2A0E0B0E2ECE552
:101EA000F2EB02E00BBF02C007900D92A037B10722
:101EB000D9F723E5A0E7BFE201C01D92AA3EB20711
:101EC000E1F70E94C23D0D942C590C940000CF9371
:101ED000DF93CDB7DEB72B97CDBFDEBFBE016F5FFF
:101EE0007F4F80E092E00F949450AE01485F5F4FC7
:101EF00068E080E092E00F94F0508A819B819F78A7
:101F00009B8395E09D83817E8A831C82BE016F5FE7
:101F10007F4F80E092E00F94445081E0888788E111
:101F20008987AE01485F5F4F68E080E092E00F94E0
:101F3000B75080E092E00F94A54E2B96CDBFDEBF48
:101F4000DF91CF9108959FB7F894E0E0F2E08081AF
:101F5000806280839FBF0895009781F020910602E0
:101F600023FF0EC020913C0230913D02FC012083F2
:101F7000318388E08093060281E0089580E008952F
:101F800080E00895CF92DF92EF92FF92CF93DF939C
:101F90000097D1F061157105C9F0EB01FC01A0813A
:101FA000B18128EE33E00F9444546B017C0183E14E
:101FB0000E9434C19B01AC01C701B6010F94EF53DD
:101FC0002883398381E003C080E001C080E0DF9195
:101FD000CF91FF90EF90DF90CF900895E5E9F8E37F
:101FE0001082118214821582128213821682178245
:101FF0008BE00E9458C1672B682B692B19F4109253
:102000009D3803C081E080939D38E5E9F8E31186AF
:1020100012860895CF93DF93EC01892B09F491C0C8
:10202000862F90E0FC013197EB30F10508F089C074
:102030008827E250FF4F8F4F0D942D5480919D388B
:10204000811107C0888199818093993890939A383B
:1020500078C08A819B818093993890939A3871C017
:1020600080919D38811107C08A819B818093993826
:1020700090939A3866C08E819F818093993890930F
:102080009A385FC080919D38811107C08C819D81F5
:102090008093993890939A3854C08A859B85809311
:1020A000993890939A384DC080919D3881110BC01A
:1020B00088819981E5E9F8E3848395838A819B810E
:1020C000868397833EC08C819D81E5E9F8E3848314
:1020D00095838E819F818683978333C080919D38BD
:1020E00081110BC08A819B81E5E9F8E384839583A4
:1020F0008C819D818683978324C0E5E9F8E38885F8
:102100009985848395838A859B858683978319C067
:1021100080919D3881110BC08C819D81E5E9F8E3A8
:10212000848395838E819F81868397830AC0E5E9A6
:10213000F8E38C859D85848395838E859F85868332
:102140009783DF91CF910895E5E9F8E38481958144
:102150008083918386819781828393830895E5E9C3
:10216000F8E381E0818712860895E5E9F8E31186B6
:102170001286089580919F38089583E10E9458C186
:10218000672B682B692B19F080919E38089580E0A9
:102190000895CF92DF92EF92FF926B01072E000C11
:1021A000EE08FF08C216D306E406F5067CF486178F
:1021B0009707E4F0092E000CAA0BBB0BE1E02817EF
:1021C00039074A075B07ACF4E0E013C06C01092E45
:1021D000000CEE08FF08C216D306E406F50644F02C
:1021E000E1E0681779072CF4E0E003C0E0E001C00B
:1021F000E0E08E2FFF90EF90DF90CF900895FF9258
:102200000F931F93CF93DF93C5E9D8E309E918E350
:10221000F12CE991F991309719F1AF010F2E000CD3
:10222000660B770BDB01CA0177231CF40196A11D15
:10223000B11DB595A795979587959A01AB01280F84
:10224000391F4A1F5B1FBF01FF2314F46F5F7F4FCD
:10225000759567958A819B819CDF813009F0F394A5
:10226000C017D107B1F6FF2011F079DF01C07DDF83
:102270006BDFDF91CF911F910F91FF900895E5E9FA
:10228000F8E381E090E0A0E0B0E08787908BA18B3D
:10229000B28B838B948BA58BB68B178A138614868F
:1022A00015861686108E0895E5E9F8E381E0878BA0
:1022B000108E0895E5E9F8E3178A108E089580914D
:1022C000AD38089584E10E9458C1672B682B692BB3
:1022D00019F08091AC38089580E00895E5E9F8E3BD
:1022E00087859089A189B289838B948BA58BB68BC6
:1022F00083859485A585B6858787908BA18BB28BC6
:1023000008956093A0387093A1388093A238909379
:10231000A33808958F929F92AF92BF92CF92DF928F
:10232000EF92FF92E5E9F8E3C388D488E588F68860
:1023300087859089A189B289C816D906EA06FB0665
:1023400091F48090A0389090A138A090A238B090DD
:10235000A338C4DFC814D904EA04FB0411F4A4DFD1
:1023600004C0A8DF02C0BADFFCCFFF90EF90DF907F
:10237000CF90BF90AF909F908F9008958BE10E9477
:1023800058C16093AE387093AF388093B038909353
:10239000B138A2EBB8E3E5E9F8E38DE998E31D92E3
:1023A00011A212A232968E179F07C9F7E5E9F8E34A
:1023B00011A612A6089581E09091BE38911101C036
:1023C00080E008958AE10E9458C1672B682B692B31
:1023D00039F081E09091BE38911103C080E00895FA
:1023E00080E008950F931F938B019C018091AE387C
:1023F0009091AF38A091B038B091B1380097A10555
:10240000B10529F1880F991FAA1FBB1FAC01BD019F
:10241000440F551F661F771F440F551F661F771FF8
:10242000840F951FA61FB71FB901A80133233CF4E1
:1024300044275527BA01401B510B620B730B21E057
:1024400084179507A607B7071CF020E001C020E01D
:10245000822F1F910F9108950F931F93CF93DF93B6
:10246000009709F40BC1A5E9B8E35D961C925D974E
:102470005E961C925E975F961C925F9790961C9258
:10248000462F50E0FA013297EA30F10508F0F6C025
:10249000EC018827E75FFE4F8F4F0D942D548091FC
:1024A0009D38811108C06C817D818E819F819ADF6A
:1024B0008093B238E3C0688179818A819B8192DF01
:1024C0008093B238DBC080919D38811108C0688547
:1024D00079858A859B8586DF8093B238CFC06881F5
:1024E00079818A819B817EDF8093B238C7C08091D9
:1024F0009D38811111C0688579858A859B8572DF39
:1025000005E918E3F801858F6C857D858E859F85AB
:1025100069DFF801868FB2C0688179818A819B81E9
:1025200061DF05E918E3F801858F6C817D818E817B
:102530009F8158DFF801868FA1C080919D3881115D
:1025400011C06C857D858E859F854CDF05E918E37C
:10255000F801858F688979898A899B8943DFF80129
:10256000868F8CC0688179818A819B813BDF05E9F8
:1025700018E3F801858F6C817D818E819F8132DF28
:10258000F801868F7BC080919D3881111FC06889BA
:1025900079898A899B8926DF05E918E3F801858F07
:1025A0006C897D898E899F891DDFF801868F688DF2
:1025B000798D8A8D9B8D16DFF801878F6C8D7D8DCF
:1025C0008E8D9F8D0FDFF80180A358C068817981BF
:1025D0008A819B8107DF05E918E3F801858F6C810B
:1025E0007D818E819F81FEDEF801868F68857985E9
:1025F0008A859B85F7DEF801878F6C857D858E85C2
:102600009F85F0DEF80180A339C080919D3881114B
:1026100011C0688979898A899B89E4DE05E918E314
:10262000F801858F6C897D898E899F89DBDEF801B1
:10263000868F24C0688179818A819B81D3DE05E9F8
:1026400018E3F801858F6C817D818E819F81CADEC0
:10265000F801868F13C080919D38811108C06C8568
:102660007D858E859F85BEDE8093B23807C06881E8
:1026700079818A819B81B6DE8093B238DF91CF91D8
:102680001F910F910895843040F5E5E9F8E341A5E5
:1026900052A5242F30E0082E02C0359527950A94C4
:1026A000E2F720FF0AC0252F30E0082E02C0359542
:1026B00027950A94E2F720FD10C021E030E0B9012F
:1026C00002C0660F771F8A95E2F7CB01E5E9F8E3D0
:1026D000462B41A78095852382A70895843090F4E6
:1026E00021E030E0A90102C0440F551F8A95E2F7AE
:1026F000CA018095E5E9F8E391A5982391A792A5F1
:10270000892382A70895BF92CF92DF92EF92FF9222
:102710000F931F93CF93DF9302EB18E3C5E9D8E340
:102720006E017801B12CF70181917F01F60121A1A1
:1027300090E0820F911D22A1820F911D039719F441
:102740008B2DA1DF02C08B2DC9DFB394F2E0CF0E39
:10275000D11C84E0B812E7CF2DE938E389A18AA320
:10276000F80181918F0189A32296C217D307B1F78F
:10277000DF91CF911F910F91FF90EF90DF90CF905D
:10278000BF900895843060F42091BE3830E0A901F4
:1027900002C0559547958A95E2F7CA018170089560
:1027A00080E00895843060F42091BF3830E0A901C2
:1027B00002C0559547958A95E2F7CA018170089540
:1027C00081E00895843000F5662379F0E5E9F8E3C7
:1027D00021E030E0A90102C0440F551F8A95E2F7BD
:1027E000CA0192A5892B82A70895E5E9F8E321E0C3
:1027F00030E0A90102C0440F551F8A95E2F7CA01D3
:10280000809592A5892382A70895CF93833009F1FB
:1028100028F4813031F0823061F02CC0883008F12A
:1028200029C08091AC38882329F181E08093AD38AC
:1028300021C0C1DD8823F1F061E080E0C3DF61E009
:1028400081E0C0DF61E082E0BDDF61E083E0BADF0C
:1028500011C080919E38882369F081E080939F3871
:1028600009C0CCEFC80F8C2F8DDF882319F061E0F1
:102870008C2FA8DFCF910895009781F0FC01DC0137
:10288000AD5BBD4F80818C936083643021F481E027
:102890000D94F605089580E00D94F60508950097CF
:1028A00019F0FC018081089580E008950F931F9333
:1028B000CF93DF931F92CDB7DEB7009709F4C6C060
:1028C0008C0181E0D8018C9311961C92119712967D
:1028D0001C92129713961C92139714961C9214979D
:1028E00015961C921597169682E1E5E0F4E20190A8
:1028F0000D928A95E1F7C80148960E947FC6F801BB
:10290000808D8783818D8087828D8187838D82876B
:10291000CE0101960E94A0C689818C3438F4D8017A
:102920005C961C925C975D961C9211C08C3431F4BD
:1029300082E0F801848F81E0858F09C08D3439F4FD
:1029400082E0D8015C968C935C975D961C9280E047
:102950000E9434C1673EB3E07B0781059105BCF45A
:102960009F938F937F936F9384EE90E29F938F93C7
:10297000C801C6969F938F930F945A56F80186A963
:10298000808B87A9818B80AD828BCDBFDEBFD801C4
:102990005E961C925E975F961C925F97D2961C92F1
:1029A000D297D3961C92F801EA5CFD4F10823196C3
:1029B000108231961082319681E0808331961082A8
:1029C000118212821382349681E090E0A0E0B0E0A0
:1029D00080839183A283B383349610823196D80189
:1029E0008C918083E751F24086E0DF011D928A9549
:1029F000E9F7E85EFD4F1082118232961082118253
:102A00003296108211823296108211823296108292
:102A10003196108232961082319610823196108251
:102A20003196108231961082319610823196108242
:102A3000118212821382349610823196108231965E
:102A40001082319688E690E1808391830F90DF9128
:102A5000CF911F910F910895009741F0613021F4BB
:102A600021E0FC0122AB0895FC0112AA0895009711
:102A700019F0FC0182A9089580E00895009741F0C3
:102A8000613021F421E0FC0123AB0895FC0113AA7D
:102A90000895009719F0FC0183A9089580E0089536
:102AA0008F929F92AF92BF92DF92EF92FF920F931D
:102AB0001F93CF93DF934115510509F46BC08A0131
:102AC0007B01C82F0E944EC5D82F8C2F0E946BC54A
:102AD000D82EDD2309F460C0882309F45FC08D2F50
:102AE0000E9434C14B015C018D2D0E9434C1672BC3
:102AF000682B692B39F4F80110821182128213823B
:102B000080E04DC09701280D391D032E000C440BA9
:102B1000550BC63050F4A0E1B7E20F944A54F801C7
:102B2000608371838283938309C0A8EEB3E00F941E
:102B30004A54F80160837183828393838D2D0E94B0
:102B400034C19B01AC01F801608171818281938164
:102B50000F94115488279927DC01821B930BA40B37
:102B6000B50BF80180839183A283B3838C2F0E94DD
:102B700011C9F80180809180A280B380DC01CB0173
:102B8000880D991DAA1DBB1D80839183A283B383E9
:102B900081E005C080E003C080E001C080E0DF91FB
:102BA000CF911F910F91FF90EF90DF90BF90AF906A
:102BB0009F908F900895CF93DF93009709F460C0A2
:102BC000EC010F94B618813091F58C830F941E019F
:102BD0008823F9F08091C13E811119C089E0EAEEA5
:102BE000F0E2A5E0B4E401900D928A95E1F7E5E00A
:102BF000F4E401900020E9F73197AF0145505444C7
:102C000021E065E074E482E299E30F940C210F94D3
:102C100057010F942101882399F183EF97E40E94D3
:102C20005FCF0F941B018A830F94680129C01C8217
:102C30000F94E2188823F9F08091C13E811119C0E8
:102C400089E0E3EFF0E2A5E0B4E401900D928A950B
:102C5000E1F7E5E0F4E401900020E9F73197AF01F6
:102C60004550544421E065E074E482E299E30F9416
:102C70000C210F94E5180F94CE1881110F94D118E0
:102C8000DF91CF9108950F931F93CF93DF93009718
:102C900009F463C0EC010F942D1B882381F18B8113
:102CA00081115BC08091C13E811126C00F94F6183E
:102CB000182F0F941B011F921F931F928F9385E073
:102CC00091E29F938F9305E014E41F930F930F9469
:102CD0005A56F80101900020E9F73197AF014550AD
:102CE000544420E0B80182E299E30F940C218DB79F
:102CF0009EB708968DBF9EBF81E08B832EC08B81CF
:102D0000813059F51B828091C13E811126C00F94FC
:102D1000F618C82F0F941B011F92CF931F928F9309
:102D20008CEF90E29F938F93C5E0D4E4DF93CF9331
:102D30000F945A5609900020E9F72197AE014550AB
:102D4000544420E065E074E482E299E30F940C219E
:102D50008DB79EB708968DBF9EBFDF91CF911F9113
:102D60000F910895CF92DF92EF92FF920F931F93EE
:102D7000CF93DF93009709F4AAC06115710509F498
:102D8000A6C08B01EC010E94FDCE882309F49FC0F0
:102D90000F9475196B017C010F941A1B86E10E9438
:102DA00058C1AB01BC018BE99CE30E9493CFD701D2
:102DB000C6010197A109B109883E9340A105B1055B
:102DC00008F03FC00E946DB9823088F18091C13E09
:102DD00081112DC00F941B011F928F9380915F531F
:102DE0001F928F93FF92EF92DF92CF9288E191E250
:102DF0009F938F930F2EF5E0EF2EF4E4FF2EF02D2E
:102E0000FF92EF920F945A56F70101900020E9F7D4
:102E10003197AF014550544421E0B70182E299E374
:102E20000F940C218DB79EB70C968DBF9EBF2AE0E4
:102E300035E444E257E46EE576E4C8010E9406DB1F
:102E400043C0D701C601895E9340A109B109843608
:102E50009105A105B105C0F584E295E40E94F5CE87
:102E6000811132C08091C13E811125C0FF92EF9245
:102E7000DF92CF9284E291E29F938F930F2EF5E041
:102E8000EF2EF4E4FF2EF02DFF92EF920F945A569E
:102E9000F70101900020E9F73197AF014550544404
:102EA00021E0B70182E299E30F940C218DB79EB720
:102EB00008968DBF9EBF2AE035E444E257E46EE5F4
:102EC00076E4C8010E9406DBCE010E9416CFDF9196
:102ED000CF911F910F91FF90EF90DF90CF900895C9
:102EE000FC01892B39F0118689E0DF011D928A955A
:102EF000E9F712860895FC01892B41F0118689E0DB
:102F0000DF011D928A95E9F71286138608950F93C3
:102F10001F93CF93DF93C3ECD8E30BE119E3CE010A
:102F2000DFDF2B96C017D107D1F787E59CE3E3DFFE
:102F300083E69CE3E0DFDF91CF911F910F9108952D
:102F4000FC01892B31F081E09285913019F080E00D
:102F5000089580E008951F93CF93DF93CDB7DEB738
:102F60006097CDBFDEBF9C01FE013196AE014F5E82
:102F70005F4F21933193255F3F4FE417F507C9F762
:102F8000892B31F110E010C0E12FF0E0EE0FFF1FB0
:102F900081E090E08C0F9D1FE80FF91F80819181E7
:102FA000CFDF8823D1F01F5F0F941A1C181760F32E
:102FB00082E00E9458C16B3068F08091623C8823A7
:102FC00059F081E090916E3C911107C080E005C0FE
:102FD00080E003C081E001C080E06096CDBFDEBF2D
:102FE000DF91CF911F910895CF92DF92EF92FF92E0
:102FF0000F931F93CF93DF93CDB7DEB72597CDBF48
:10300000DEBF19821A821B821C824115510559F1BB
:103010006A017B01182FCA0163DFAE014F5F5F4F6A
:10302000B701812F3DDD8823C9F009811A812B81E9
:103030003C814BE0BE016B5F7F4FC6010F9490282F
:10304000F60101900020E9F73197EC19FD09D6014E
:103050001996EC93199781E01A968C9369817A817D
:103060008B819C8103C060E070E0CB012596CDBFD1
:10307000DEBFDF91CF911F910F91FF90EF90DF9016
:10308000CF9008958F929F92AF92BF92EF92FF924E
:103090000F931F93CF93DF930097A1F061157105F4
:1030A00089F0142F7B01EC010F9429064B015C0180
:1030B000113009F426D9950184014BE0B701CE0106
:1030C0000F94E226DF91CF911F910F91FF90EF9027
:1030D000BF90AF909F908F900895AF92BF92CF9284
:1030E000DF92EF92FF920F931F93CF93DF93CDB7B1
:1030F000DEB76097CDBFDEBF8C01CE0101967C01AB
:103100004096F70161937193655F7F4FE817F90768
:10311000C9F70115110509F475C282E00E9458C172
:10312000D62E96E0D91206C0C8010F9464178111FB
:103130006FC243C38FEF8D0D823030F4C8010F94FE
:103140006417811111C039C38FEE8D0D823030F4B8
:10315000C8010F946417811107C02FC3C8010F94D1
:103160006417882309F429C380E2E4EDFFE3DF015B
:103170001D928A95E9F780E1E0E3FBE3DF011D9210
:103180008A95E9F78D2D90E0FC013197E231F10548
:1031900008F03AC28827ED5EFE4F8F4F0D942D54F4
:1031A00058010F2EF4EDCF2EFFE3DF2EF02D01E0BE
:1031B00010E00EC10F946117C82E49815A81F801A1
:1031C0006081718111DF0F2EF4EDEF2EFFE3FF2EF2
:1031D000F02DD7016D937D938D939C9313974B8125
:1031E0005C81F801628173818C2DFEDED70114961B
:1031F0006D937D938D939C931797B2E0DB1206C27B
:103200008091D43F9091D53FA091D63FB091D73FC8
:103210008093303B9093313BA093323BB093333B50
:1032200081E0CBC258010F2EF4EDCF2EFFE3DF2E4D
:10323000F02D01E010E00BC01F5F0F5FE2E0EE0E2B
:10324000F11CF2E0AF0EB11C84E0C80ED11C1123BA
:1032500009F4FBC1123009F4EAC1D7014D915C9128
:10326000F5016081718180E0BFDED6016D937D93B1
:103270008D939C9313970430F8F28091D43F9091F2
:10328000D53FA091D63FB091D73F8093303B9093EC
:10329000313BA093323BB093333B81E08EC2580167
:1032A0000F2EF4EDCF2EFFE3DF2EF02D01E010E026
:1032B0000BC01F5F0F5FB2E0EB0EF11CE2E0AE0E41
:1032C000B11CF4E0CF0ED11C112309F4DBC1123084
:1032D00009F4CAC1D7014D915C91F50160817181FA
:1032E00082E082DED6016D937D938D939C9313973C
:1032F0000430F8F2E0E3FBE3A4EDBFE34D915D9110
:103300006D917C91139740835183628373831496EC
:103310008D919D910D90BC91A02D84839583A68362
:10332000B78381E04AC258010F2EF4EDCF2EFFE3A0
:10333000DF2EF02D01E010E00BC01F5F0F5FB2E049
:10334000EB0EF11CE2E0AE0EB11CF4E0CF0ED11C8E
:10335000112309F4B8C1133009F4A3C1113009F4E1
:10336000A2C1143009F4A1C1D7014D915C91F501BE
:103370006081718180E038DED6016D937D938D93FD
:103380009C9313970630C8F2E0E3FBE3A4EDBFE3A0
:103390004D915D916D917C91139740835183628330
:1033A000738314968D919D910D90BC91A02D848373
:1033B0009583A683B78381E000C21F5F0F5FB2E0F1
:1033C000EB0EF11CE2E0AE0EB11CF4E0CF0ED11C0E
:1033D000112309F487C1143009F492C1812F8B7F26
:1033E000813009F48FC1823009F48EC1D7014D912B
:1033F0005C91F5016081718185E0F6DDD6016D9308
:103400007D938D939C9313970830B8F2E0E3FBE330
:10341000A4EDBFE34D915D916D917C911397408335
:1034200051836283738314964D915D916D917C916C
:103430001797448355836683778318964D915D91E2
:103440006D917C911B9740875187628773871C968B
:103450008D919D910D90BC91A02D84879587A68715
:10346000B78781E0AAC158010F2EF4EDCF2EFFE3FC
:10347000DF2EF02D01E010E00BC01F5F0F5FB2E008
:10348000EB0EF11CE2E0AE0EB11CF4E0CF0ED11C4D
:10349000112309F458C1143009F445C1812F8B7FE1
:1034A000813009F442C1D7014D915C91F5016081F1
:1034B000718180E099DDD6016D937D938D939C930E
:1034C00013970830D0F2E0E3FBE3A4EDBFE34D91A6
:1034D0005D916D917C9113974083518362837383D7
:1034E00014968D919D910D90BC91A02D8483958310
:1034F000A683B78381E061C1680104ED1FE35E012B
:10350000B9E0AB0EB11CF701419151917F01D60199
:103510006D917D916D0180E067DDF801619371939C
:10352000819391938F01EA14FB0469F781E045C10F
:1035300058010F2EF4EDCF2EFFE3DF2EF02D01E02A
:1035400010E00BC01F5F0F5FF2E0EF0EF11C82E096
:10355000A80EB11C94E0C90ED11C112309F410C1AE
:10356000133009F4FFC0D7014D915C91F5016081E2
:10357000718180E039DDD6016D937D938D939C93AD
:1035800013970630F8F28091D43F9091D53FA091E7
:10359000D63FB091D73F8093303B9093313BA0937F
:1035A000323BB093333B81E008C158010F2EF4ED5C
:1035B000CF2EFFE3DF2EF02D01E010E00BC01F5FE8
:1035C0000F5FB2E0EB0EF11CE2E0AE0EB11CF4E0D6
:1035D000CF0ED11C112309F4E2C0D7014D915C91AB
:1035E000F5016081718181E0123009F480E0FCDC3A
:1035F000D6016D937D938D939C9313970430F8F2CD
:1036000081E0DBC080E0D9C080E0D7C081E0D5C0D8
:1036100080E2E4EDFFE3DF011D928A95E9F780E1A6
:10362000E0E3FBE3DF011D928A95E9F7B9CDF701ED
:1036300040815181D5016D917C9183E0D5DCF6010B
:103640006083718382839383F7CDD7014D915C9121
:10365000F5016081718183E0C7DCD6016D937D93B4
:103660008D939C931397E8CDF70140815181D5014B
:103670006D917C9183E0B8DCF60160837183828375
:10368000938317CED7014D915C91F50160817181D3
:1036900083E0AADCD6016D937D938D939C93139761
:1036A00008CE83E003C082E001C082E0F7014081E0
:1036B0005181D5016D917C9197DCF6016083718316
:1036C000828393833ACED7014D915C91F50160815D
:1036D000718183E089DCD6016D937D938D939C93FA
:1036E00013972BCEF70140815181D5016D917C91CB
:1036F00083E07ADCF60160837183828393835DCEFD
:1037000083E003C082E001C084E0D7014D915C9169
:10371000F5016081718168DCD6016D937D938D9395
:103720009C9313974ACE83E001C082E0F701408169
:103730005181D5016D917C9157DCF60160837183D5
:10374000828393839ACED7014D915C91F50160817C
:10375000718183E049DCD6016D937D938D939C93B9
:1037600013978BCEF70140815181D5016D917C91EA
:1037700083E03ADCF6016083718382839383E2CE37
:10378000D7014D915C91F5016081718183E02CDC62
:10379000D6016D937D938D939C931397D3CEF701B0
:1037A00040815181D5016D917C9180E01DDCF60155
:1037B000608371838283938302CF6096CDBFDEBF27
:1037C000DF91CF911F910F91FF90EF90DF90CF90FD
:1037D000BF90AF9008950F94DB14882329F00F94C5
:1037E000EC1484E0809327060895CF93DF9300972D
:1037F00099F1EC0188818130A8F0833018F086308F
:1038000019F010C0E8DF25C08091280682FD03C0B2
:1038100084E0809325060F9475148823D1F00F94CB
:10382000861417C00F947514882399F00F9486148A
:1038300084E0809327060DC08D8181110DC00F9407
:10384000B914882349F00F94CA1484E080932706A2
:1038500003C08881863081F7DF91CF9108950E945F
:1038600037D30F94FA1920E137E240E050E00F948B
:10387000EF53672B682B692BE1F40E9437D381301B
:1038800019F40C944BD208950E9437D3823021F45E
:1038900081E00C943AD308950E9437D3833019F411
:1038A0000C9440D508950E9437D3843011F40C94C1
:1038B00094D508950F931F93CF93DF931F921F9278
:1038C000CDB7DEB719821A820097B9F08C010E9439
:1038D0008E5490E006969E012F5F3F4F43E060E0DC
:1038E000800F911F0F944125882339F049815A8117
:1038F00060E070E080E00E9443C10F900F90DF9184
:10390000CF911F910F9108959F92AF92BF92CF9246
:10391000DF92EF92FF920F931F93CF93DF931F924B
:10392000CDB7DEB7009709F44BC05C0182E00E947E
:1039300058C1962E8501085D1F4FBE016F5F7F4FF6
:10394000C8010E9415DF882391F0F501C0A4D1A41D
:10395000E2A4F3A489E00E9458C1AB01BC010FE9C5
:1039600018E42FE838E489810F94151A17C0BE01B6
:103970006F5F7F4FC8010E9461E8F501C0A4D1A428
:10398000E2A4F3A489E00E9466C1AB01BC010FE987
:1039900018E42FE838E489810F94151AFAE0F91534
:1039A00058F4F50140A551A562A573A587E898E4F0
:1039B0000F94FA1C81E005C00F94641D81E001C0E2
:1039C00080E00F90DF91CF911F910F91FF90EF90CA
:1039D000DF90CF90BF90AF909F900895CF92DF92ED
:1039E000EF92FF920F931F93CF93DF931F92CDB768
:1039F000DEB7009779F18C01BE016F5F7F4F88962B
:103A00000E945CEB882399F0F801C0A4D1A4E2A441
:103A1000F3A489E00E9458C1AB01BC010FE918E48E
:103A20002FE838E489810F94151A81E014C0F80159
:103A3000C0A4D1A4E2A4F3A489E00E9466C1AB01B2
:103A4000BC010FE918E42FE838E489810F94151AB6
:103A500081E001C080E00F90DF91CF911F910F9125
:103A6000FF90EF90DF90CF90089589E10E9458C1B8
:103A7000623059F482E00E9458C1673041F06930E9
:103A800031F0613021F081E0089580E0089580E018
:103A9000089589E10F941907623059F482E00F9478
:103AA0001907673041F0693031F0613021F081E071
:103AB000089580E0089580E008953F924F925F92CC
:103AC0006F927F928F929F92AF92BF92CF92DF922E
:103AD000EF92FF920F931F93CF93DF93CDB7DEB793
:103AE0006497CDBFDEBFB82E8B017A0189E10E94B9
:103AF00058C1A62E0115110509F472C28091C13E6C
:103B0000882339F00F2EF2E2CF2EF9E3DF2EF02DCD
:103B100006C00F2EF9E2CF2EFAE3DF2EF02D82E061
:103B20008A1508F4A12C8BE7F801808383E7818351
:103B30008CE28283F2E3BF1207C082E38A0DF801B0
:103B400083838CE284830BC0F801B3828CE284838C
:103B5000F0E3BF1609F4F1C182E3B81218C283EC96
:103B600098E3FE0132969E012E5E3F4F8193919322
:103B70000B962E173F07D1F788E08983E114F104F3
:103B800069F086E0F701D801159601900D928A95AB
:103B9000E1F70F2EFBE0FF2EF02D04C00F2EF5E015
:103BA000FF2EF02DF801EF0DF11D8CE2808382E0F5
:103BB0000E9458C1762E872D072C000C990B9F93DD
:103BC0007F9281E291E29F938F93F394C8018F0DCE
:103BD000911D9F938F930F945A56F80101900020E6
:103BE000E9F73197E01BF10B7F01FF24F801EE0D9F
:103BF000FF1D118221E0A701B801C6010F940C211D
:103C00000F900F900F900F900F900F908091C13EEA
:103C1000811112C01A8A21E040E050E0BE016E5EC0
:103C20007F4F82E299E30F940C2120E0A701B801B5
:103C300082E299E30F940C2191E09A1508F402C1F5
:103C40001982912C0F2EFCE28F2EF02DF801319667
:103C5000EB8BFC8B0F2EF1EC4F2EFEE35F2EF02D45
:103C60005BC00F941A1C6980861509F45BC0F801CB
:103C70008082E62CF12CF701EE0FFF1F81E090E02F
:103C80008C0F9D1FE80FF91FA180B280F5014185BF
:103C900050E0B5018B899C890F942C56F5018185E4
:103CA0006894332431F8380E8F5FF801E80FF11D66
:103CB0008082F7013196EE0FFF1F81E090E08C0FBC
:103CC0009D1FE80FF91FA180B280F501418550E0EA
:103CD000B501C801830D911D0F942C56F501E184A7
:103CE0003E0C639463946982E32CF12CF801EE0D91
:103CF000FF1D118221E0A701B801C6010F940C211C
:103D0000F2018081811107C020E0A701B80182E2A1
:103D100099E30F940C2193940F941A1C869598168E
:103D200008F49FCFFAE0F7150CF0D8C08CE07816B5
:103D30004CF09DE097150CF050C180EF870D83305B
:103D400008F44BC1198280E00F2EFCE23F2EF02DCB
:103D50004801EFEF8E1A9E0A0F2EF1EC4F2EFEE374
:103D60005F2EF02DF8013082E82EF12CF701EE0FD6
:103D7000FF1FEE0DFF1DEE0FFF1FEE0FFF1FE95A95
:103D8000F34C82858C3419F0823541F00EC080E30B
:103D90009CE2F4018083918312820FC081E39CE254
:103DA000F40180839183128208C085E0E6E3F1E2AA
:103DB000D40101900D928A95E1F7F801019000205D
:103DC000E9F731975F01A01AB10A3701660C771C39
:103DD000B3016E0D7F1D660F771F660F771F695A3F
:103DE000734CFB01418550E0C8018A0D911D0F9471
:103DF0002C56F301EE0DFF1DEE0FFF1FEE0FFF1F00
:103E0000E95AF34C8185A80EB12CF801EA0DFB1D8F
:103E1000118221E0A501B801C6010F940C21F20125
:103E20008081811107C020E0A501B80182E299E3F9
:103E30000F940C21E98081E08E0D8983823008F493
:103E400091CF4CC01982612C0F2EFCE25F2EF02D19
:103E50004801FFEF8F1A9F0A0F2EF1ECAF2EFEE301
:103E6000BF2EF02D36C00F941A1C79808715B1F142
:103E7000F8015082E72DF0E0EE0FFF1F81E090E0A7
:103E80008C0F9D1FE80FF91FE180F280F70141853B
:103E900050E0B701C4010F942C56F701E184E3947C
:103EA00073947982F12CF801EE0DFF1D118221E04F
:103EB000A701B801C6010F940C21F5018081811181
:103EC00007C020E0A701B80182E299E30F940C211A
:103ED00063940F941A1C8695681628F20F2EFCE244
:103EE000FF2EF02DF801F08284E00E9458C1605D41
:103EF000F8016183F28240E0BE016F5F7F4FC8012D
:103F00000396C0D8898193E0980FF801E90FF11D5D
:103F10009DE790838C5FE82EF12CF801EE0DFF1DDC
:103F2000118221E0A701B801C6010F940C218091F4
:103F3000C13E882309F445C053C00F2EFDE5EF2E86
:103F4000F6E4FF2EF02DF701408150E066E276E4C2
:103F5000C80105960F942C56F701808195E0980FC3
:103F6000F801E90FF11D9DE790838A5FE82EF12C9F
:103F7000F801EE0DFF1D118221E0A701B801C60175
:103F80000F940C218091C13E81112AC011C021E003
:103F900045E050E0B801C6010F940C218091C13E6C
:103FA00081111EC0F0E3BF120FC045E050E002C017
:103FB0004E2D5F2D20E0B80182E299E30F940C2191
:103FC0000FC04E2D5F2D02C045E050E021E0B8014A
:103FD00082E299E30F940C2103C081E08983B4CE7F
:103FE0006496CDBFDEBFDF91CF911F910F91FF90FF
:103FF000EF90DF90CF90BF90AF909F908F907F9089
:104000006F905F904F903F900895CF93892B81F0F0
:104010000E949C53CAE00E945F540E9499538823D7
:1040200021F00E94AF53811105C0C150A1F703C018
:10403000C0E001C0C1E08C2FCF91089589E10E94BA
:1040400058C1611104C00F943201882371F081E0DE
:1040500040916453509165536091665370916753DA
:10406000452B462B472B09F080E008958F929F92B5
:10407000AF92BF92CF92DF92EF92FF920F931F9376
:10408000CF93DF930097A9F1EC0186E00E9458C11D
:104090004B015C0184E00E9458C1162F87E00E940A
:1040A00058C1062F812F0F940D060F9429066B011E
:1040B0007C0186169706A806B906D9F0AB01BC01AB
:1040C00086E00E94ACC68823A1F00F94B605B70124
:1040D000A60186E00E944EC1B701A60186E00F94BA
:1040E0002C07602F812F0F940D0668E0CE010E94EF
:1040F0003C14DF91CF911F910F91FF90EF90DF90D3
:10410000CF90BF90AF909F908F90089582E10E94D2
:1041100058C128E0E6E9F3E5DF01322F1D923A9518
:10412000E9F7EEE9F3E5DF011D922A95E9F721E0D1
:1041300030E0672B682B692B11F420E030E0F901A7
:10414000E153FF4D80818560ECE5F3E582AF83AFFD
:1041500081E00895009761F0613031F4FC01EA5C80
:10416000FD4F21E020830895FC01EA5CFD4F1082A1
:1041700008950097B1F0FC0180818430A1F40F9480
:104180004D19823039F089E10E9458C1672B682BA4
:10419000692B59F00F942A1991E0811107C090E022
:1041A00005C090E003C090E001C090E0892F089521
:1041B0000F931F93CF93DF938C01EB01209709F4AA
:1041C00042C01882892B19F189E10E9458C1F80177
:1041D00080818130C0F0833018F08530D0F013C07A
:1041E000611106C02097B9F087E4888380E02EC073
:1041F0006150623090F0209791F087E4888380E0EE
:1042000025C0209771F082E4888380E01FC080E0A1
:104210001DC081E01BC080E019C081E017C080E0B4
:1042200015C080E013C081E011C080E00FC089E1BB
:104230000E9458C1F8018081813018F3833080F2E8
:10424000853088F3DECF892B91F7EFCFDF91CF91C7
:104250001F910F910895009739F0FC0180818150E2
:10426000843020F481E0089580E0089580E008958E
:10427000009751F0FC018081813040F0843010F0D3
:10428000853021F481E0089580E0089580E008956C
:10429000CF92DF92EF92FF92CF93DF93009709F4D2
:1042A0005FC0EC0183E00E9458C16B017C01AB014F
:1042B000BC0155276627772783E00E94ACC6882378
:1042C00009F44BC08C2DFE01E95CFD4FC0828130AA
:1042D00021F1823009F044C088E00E9458C1FE01FB
:1042E000E75CFD4F6083AB01BC015527662777274C
:1042F00088E00E94ACC6811105C081E0FE01E75C48
:10430000FD4F8083FE01E85CFD4F1082C65CDD4FEF
:10431000188219821A821B8223C087E00E9458C12A
:10432000F62E84E00E9458C1862F6F2D0F940D0643
:1043300085E00E9458C10F94BE06FE01E25CFD4F6D
:1043400060837183828393830F94D605C65CDD4FAF
:10435000188219821A821B8203C0C95CDD4F188241
:10436000DF91CF91FF90EF90DF90CF90089500976D
:1043700061F1FC01E85CFD4F2081319630813217FC
:1043800010F021111BC0FC01E85CFD4F315030835F
:1043900032964081518162817381403821E5520714
:1043A00021E06207710598F44F5F5F4F6F4F7F4FB9
:1043B000408351836283738381E00895FC01E85C4C
:1043C000FD4F2150208380E0089580E0089580E033
:1043D00008950F931F93CF93DF93009741F1EC0162
:1043E0000F94ED05FE01E25CFD4F008111812281F9
:1043F00033816017710782079307D8F00F94D605B1
:10440000FE01E65CFD4F80819181A281B3818038FD
:1044100021E5920721E0A207B10568F40196A11DEC
:10442000B11D80839183A283B38381E005C080E0C6
:1044300003C080E001C080E0DF91CF911F910F9118
:104440000895CF93DF93009709F43DC0FC01EA5C27
:10445000FD4F20812223B9F1EC018BDE813021F464
:10446000CA5CDD4F18822FC089E10E9458C16111DA
:104470001AC00F944D19813031F1823089F4DEDD9C
:10448000882309F10F940719CA5CDD4F188284E272
:1044900095E40E94EFCE83EF97E40E9416CF13C0FD
:1044A0000F943B1910C0CADD882369F00F940719D7
:1044B000CA5CDD4F188284E295E40E94EFCE83EF60
:1044C00097E40E9416CFDF91CF910895FF920F934A
:1044D0001F93CF93DF936115710509F47CC04115DB
:1044E000510509F478C08A01EB01F82E82E10F949E
:1044F000190721E0672B682B692B09F420E08F2D29
:1045000090E0FC013197E231F10508F05BC08827AB
:10451000EB5DFE4F8F4F0D942D541882E22FF0E08B
:10452000E153FF4D80818560F801808354C083E0B2
:104530008883E22FF0E0E153FF4D8081F801808312
:104540004AC01882E22FF0E0E153FF4D8081816084
:10455000F801808340C083E08883E22FF0E0E153DC
:10456000FF4D8081F801808336C01882E22FF0E091
:10457000E153FF4D80818160F80180832CC083E08E
:104580008883E22FF0E0E153FF4D8081F8018083C2
:1045900022C0188285E0F80180831DC0188281E066
:1045A000F801808318C01882E22FF0E0E153FF4D3C
:1045B00080818160F80180830EC0188281E0F8015B
:1045C000808309C01882E22FF0E0E153FF4D808123
:1045D0008560F8018083DF91CF911F910F91FF904B
:1045E00008958F929F92AF92BF92CF92DF92EF92F7
:1045F000FF920F931F93CF93DF93892B09F486C00B
:1046000089E00E9458C19B01AC01A8EEB3E00F9471
:104610004A546B017C010F945E19C616D706E80652
:10462000F90609F475C0C701B60128EE33E040E091
:1046300050E00F94EF53F22ED22F2E3108F06AC0C3
:10464000213009F469C00F945E1928EE33E040E090
:1046500050E00F94EF53822FF21638F46F2D0F9421
:10466000BC53C92F992309F45CC00F94F618E82EA7
:104670006D2F0F94BC53D92F892F90E08E0D911D73
:10468000CA970CF04BC08D2E912CA12CB12C0F94FD
:104690007519162F072FD82EC92EA8EEB3E0A50145
:1046A00094010F944A544F2D0F94A319C091C13E09
:1046B000C11136C00F9475199F938F937F936F9399
:1046C000CF92DF920F931F931F92DF931F92EF926F
:1046D0008BE391E29F938F9305E014E41F930F9374
:1046E0000F945A56F80101900020E9F73197AF0175
:1046F0004550544421E0B80182E299E30F940C2123
:104700008DB79EB740968DBF9EBF0BC0C0E009C05D
:10471000C0E007C0C1E005C0C0E003C0C1E001C007
:10472000C0E08C2FDF91CF911F910F91FF90EF9000
:10473000DF90CF90BF90AF909F908F900895EF92B1
:10474000FF920F931F93CF93DF932091C13E2223BB
:1047500039F00F2EF2E2EF2EF9E3FF2EF02D06C016
:104760000F2EF9E2EF2EFAE3FF2EF02D0097D1F194
:10477000EC018BE7888388E689838CE28A8392E662
:104780009B838C837F936F9386E791E29F938F93B4
:10479000CE0105969F938F930F945A56FE01019078
:1047A0000020E9F73197EC1BFD0B8F01112721E069
:1047B000A801BE01C7010F940C210E946DB90F9092
:1047C0000F900F900F900F900F90873059F48091B9
:1047D000C13E811107C021E0A801BE0182E299E338
:1047E0000F940C21DF91CF911F910F91FF90EF90CB
:1047F00008958F929F92AF92BF92CF92DF92EF92E5
:10480000FF920F931F93CF93DF93009709F470C02B
:104810002091C13E222339F00F2EF2E2EF2EF9E370
:10482000FF2EF02D06C00F2EF9E2EF2EFAE3FF2E39
:10483000F02DEC018BE7888388E689838CE28A83FC
:1048400093E79B838C830FE61CE3F801848C0E9422
:10485000B4A0982EA090C03EB090BD3EF801C2809A
:10486000D0800F9432011F928F921F929F921F92BD
:10487000AF921F92BF921F92CF921F92DF921F9210
:104880008F93F80185811F928F9384811F928F935C
:1048900083811F928F938BE591E29F938F93CE013B
:1048A00005969F938F930F945A56FE010190002016
:1048B000E9F73197EC1BFD0B8F01112721E0A801CF
:1048C000BE01C7010F940C218DB79EB748968DBFCE
:1048D0009EBF8091C13E81110BC0A8014250510979
:1048E000BE016F5F7F4F21E082E299E30F940C21BC
:1048F000DF91CF911F910F91FF90EF90DF90CF90BC
:10490000BF90AF909F908F900895DF92EF92FF92AB
:104910000F931F93CF93DF9300D01F92CDB7DEB7D5
:104920008C010F94FD14882349F00F940E150E94FA
:10493000A30F8AEA92E45DDF80E066C0CE010196B3
:104940000E94AC0F882309F45FC0F090A806E090A5
:104950006806D0902806BE016D5F7F4FCE0101969C
:104960000E94C20F882309F44CC00E9479B98823A1
:10497000C9F18091C13E811135C0D0FADD24D0F853
:104980001F92DF92E4FAEE24E0F81F92EF92F6FA1B
:10499000FF24F0F81F92FF928A818F9389818F9371
:1049A0008C818F938B818F938AE791E29F938F9372
:1049B0000F2EF5E0EF2EF4E4FF2EF02DFF92EF9294
:1049C0000F945A56F70101900020E9F73197AF0193
:1049D0004550544421E0B70182E299E30F940C2141
:1049E000CDBFDEBF6B817C818AEA92E4A8DE01152F
:1049F000110549F08B819C81F8018083918381E0CE
:104A000003C081E001C081E02496CDBFDEBFDF910D
:104A1000CF911F910F91FF90EF90DF900895882321
:104A200021F081E08093C03E08951092C03E089529
:104A30000F931F93CF93DF936115710571F000976A
:104A400061F0EB018C010F941F15882331F00F9456
:104A50003015BE01C8010E94208EDF91CF911F91B9
:104A60000F910895CF93DF93009751F0EC010F94CD
:104A70006B15882329F0CE010E9462900F947C155B
:104A8000DF91CF910895009791F0FC01EC5BFD4F11
:104A90002FEF3FE720833183329620E030E82083F8
:104AA00031833296108211823296108211820895DB
:104AB0000F93CF93DF930097A1F0662371F0EA0183
:104AC000FC01E45BFD4F81E08083C9010F946C1B06
:104AD000602FCE010E9459A204C0FC01E45BFD4F8F
:104AE0001082DF91CF910F910895EF92FF920F9373
:104AF0001F93CF93DF931F921F92CDB7DEB700971E
:104B000009F498C06115710509F494C0FC0122A94B
:104B1000211104C023A9222309F48CC08B017C013C
:104B2000FC0112AA13AA0E94FF100E948A110E947F
:104B30008313F70144A955A9B7016A5C7F4F9E0111
:104B40002F5F3F4FC8010F94514AC8010F94FF4B8C
:104B5000F701E75AFD4FD701AD5ABD4F8C918083C5
:104B6000319611968C9180830F9475199F938F9332
:104B70007F936F9389E991E29F938F9305E014E40B
:104B80001F930F930F945A56F80101900020E9F7F4
:104B90003197AF014550544421E0B80182E299E3D6
:104BA0000F940C21CDBFDEBFF70124A935A989815F
:104BB0009A812817390719F1C70106969F938F9399
:104BC00085EA91E29F938F931F930F930F945A5608
:104BD000F80101900020E9F73197AF0145505444A6
:104BE00021E0B80182E299E30F940C210E9406A310
:104BF0000F900F900F900F900F900F9002C00E9497
:104C000096A2E6EEF2E4808190E0DC01AA51BD4B71
:104C100025853685880F991FFC01EA51FD4B41819E
:104C200052811F960C9161E0C70142DF0E94C6923B
:104C30000F94D21B0F900F90DF91CF911F910F9186
:104C4000FF90EF9008950F931F93CF93DF930097FA
:104C500009F448C06115710509F444C08B01EC01E9
:104C6000FC01E45BFD4F80818823C1F1DB018C9165
:104C7000882341F10F94881B8823A1F1F8016081FA
:104C800061506083611108C00E94CBA20E94B8A24B
:104C9000C45BDD4F188226C070E0F801E60FF71FF5
:104CA000D8011D962D913C911E97660F771FA60F78
:104CB000B71F11964D915C911297078561E0CE0167
:104CC000F7DE10C00F94881B882361F00E94CBA2EE
:104CD0000E94B8A2C45BDD4F188204C00E94CBA220
:104CE0000E94B8A2DF91CF911F910F9108958F92EA
:104CF0009F92BF92CF92DF92FF920F931F93CF9319
:104D0000DF93009709F4DAC06115710509F4D6C084
:104D10002091C13E222309F4C0C0C2E2D9E3BFC042
:104D20008B014C010E946211B82E0E94E211D82E14
:104D30000E94BD10C82E8D2D90E08B0D911D8C0D05
:104D4000911D892B71F4F401E35BFD4F808181306B
:104D500009F4B4C081E0808380E090E00F949F1B51
:104D6000ADC0F401E35BFD4F8081823009F43EC0A9
:104D7000BB2051F00E945F11811108C061E0CE019B
:104D80000E949E9201E003C000E001C000E0CC2040
:104D900009F48AC00E94BA10811186C063E0CE0176
:104DA0000E949E9201E080C0DD2081F0812F0E9450
:104DB000C213882359F0812F0E94D213811106C09B
:104DC00064E0610FCE010E949E9201E01F5F1430EB
:104DD00059F7002309F472C0E401C35BDD4F82E0A0
:104DE000888384EF91E00F949F1B68C00F94BB1BD6
:104DF000882309F463C0BB2009F45DC00E945F11E1
:104E0000811159C00E941DA3CC2009F44FC0FF247A
:104E1000F39401C0F12C0E94BA10811149C00E9484
:104E20001DA316C0D0E0C0E0DD2069F08D2F0E94E8
:104E3000C213882341F08D2F0E94D213811103C029
:104E40000E941BA3C1E0DF5FD43071F7CC23E1F0F7
:104E500084EF91E00F949F1BD8018C9190E0F801B2
:104E6000E80FF91F1D962D913C911E97880F991FF1
:104E7000A80FB91F11964D915C911297078561E0BB
:104E80008FE69CE315DE1AC0F401E35BFD4F8081E1
:104E90008230A1F481E0808311C0C9E2DAE3FC0131
:104EA0002081243059F43CCF10E07ECFFF24F394CE
:104EB000F110CECFB7CFC110ADCFB4CFDF91CF912E
:104EC0001F910F91FF90DF90CF90BF909F908F9098
:104ED0000895009721F0FC01E35BFD4F6083089586
:104EE000CF93DF930097C1F0EC01198218820E94E2
:104EF000491D813031F482E0888389E1898391E022
:104F000006C0CE010E948FEC91E0811190E081E01B
:104F1000992319F080E001C080E0DF91CF910895DE
:104F2000CF93892B09F44CC082E00E9458C1862F90
:104F300090E0FC013297E031F10508F043C088278A
:104F4000E95CFE4F8F4F0D942D5440E050E0BA01C4
:104F500080E00E94E3C837C040E050E0BA0180E042
:104F60000E94E3C8C82F40E050E0BA0181E00E94EF
:104F7000E3C8C80F81E0C23031F180E024C040E0D6
:104F800050E0BA0180E00E94E3C8C82F40E050E042
:104F9000BA0181E00E94E3C8C80F40E050E0BA01C6
:104FA00082E00E94E3C8C80F40E050E0BA0183E00D
:104FB0000E94E3C8C80F81E0C43029F080E003C03C
:104FC00080E001C080E0CF910895CF92DF92EF9210
:104FD000FF92843098F4E82FF0E0EE0FFF1FEE0F01
:104FE000FF1FE05DF44CC080D180E280F3800E941E
:104FF000B3C86C197D098E099F0903C060E070E099
:10500000CB01FF90EF90DF90CF900895CF93892B45
:1050100009F453C082E00E9458C1862F90E0FC0141
:105020003297E031F10508F04AC08827E95BFE4F6E
:105030008F4F0D942D5480E0C8DFAB01BC0180E0A0
:105040000E94E3C83DC080E0C0DFAB01BC0180E04E
:105050000E94E3C8C82F81E0B8DFAB01BC0181E04A
:105060000E94E3C8C80F81E0C23051F180E028C03F
:1050700080E0ABDFAB01BC0180E00E94E3C8C82F39
:1050800081E0A3DFAB01BC0181E00E94E3C8C80F4F
:1050900082E09BDFAB01BC0182E00E94E3C8C80F45
:1050A00083E093DFAB01BC0183E00E94E3C8C80F3B
:1050B00081E0C43029F080E003C080E001C080E0DE
:1050C000CF91089590E0FC013397EE30F10508F0A0
:1050D000A7C08827E95AFE4F8F4F0D942D54ECE559
:1050E000F3E5868D978DA0A1B1A1428D538D648D7E
:1050F000758D841B950BA60BB70B86399105A10501
:10510000B10508F48FC046A157A160A571A582A181
:1051100093A1A4A1B5A1481B590B6A0B7B0B81E09D
:10512000463951056105710508F483C080E0089592
:10513000ECE5F3E582A193A1A4A1B5A1468D578D1D
:1051400060A171A1841B950BA60BB70B8639910545
:10515000A105B10508F468C046A557A560A971A9C5
:1051600082A593A5A4A5B5A5481B590B6A0B7B0B7B
:1051700081E0463951056105710508F45AC080E0A7
:105180000895ECE5F3E582A193A1A4A1B5A1468D14
:10519000578D60A171A1841B950BA60BB70B8639A7
:1051A0009105A105B10508F441C042A953A964A91C
:1051B00075A986A597A5A0A9B1A9481B590B6A0B8B
:1051C0007B0B81E0463951056105710590F180E066
:1051D0000895ECE5F3E5868D978DA0A1B1A1428DF0
:1051E000538D648D758D841B950BA60BB70B86397B
:1051F0009105A105B105E0F042A553A564A575A5EB
:1052000086A197A1A0A5B1A5481B590B6A0B7B0BE2
:1052100081E0463951056105710558F080E0089537
:1052200080E0089581E0089581E0089581E0089587
:1052300081E00895CF9382E10E9458C1C1E0672BBD
:10524000682B692B09F4C0E082E00E9458C188E015
:10525000E6E9F3E5DF01982F1D929A95E9F7EEE96B
:10526000F3E5DF011D928A95E9F7862F90E0FC01B6
:105270003197E231F10508F0EFC08827EB59FE4F76
:105280008F4F0D942D54EC2FF0E0E153FF4D8081B2
:105290008560ECE5F3E582AF83AFE8C0EC2FF0E08A
:1052A000E153FF4D8081ECE5F3E582AF83AF83E00E
:1052B00080939E5380939F53D9C0862F03DFEC2F9A
:1052C000F0E0E153FF4D908121E0811101C020E029
:1052D000822F892BECE5F3E582AF84AF83E08093E6
:1052E0009E538093A053892F816083AF85AFBEC04A
:1052F000EC2FF0E0E153FF4D8081ECE5F3E582AF68
:1053000084AF93E090939E539093A05383AF85AF67
:1053100082E080939F538093A153A8C0862FD2DE52
:10532000EC2FF0E0E153FF4D208191E0811101C0AD
:1053300090E0892F822BECE5F3E582AF85AF93E017
:1053400090939E539093A15383AF86AF82E0809356
:105350009F538093A253822F816084AF87AF86C012
:10536000EC2FF0E0E153FF4D8081ECE5F3E582AFF7
:1053700086AF93E090939E539093A25383AF87AFF1
:1053800092E090939F539093A35384AF80939C5348
:1053900094E09093A0539093A45385AF80939D5332
:1053A00085E08093A1538093A55360C0862F8ADE49
:1053B00091E0811101C090E0892F8F70ECE5F3E559
:1053C00082AF86AF93E090939E539093A25383AFA6
:1053D00087AF82E080939F538093A35381E084AF93
:1053E00080939C5395AF90939D5340C0ECE5F3E5BB
:1053F00085E082AF84AF87E083AF85AF37C0862F6B
:1054000061DE91E0811101C090E0EC2FF0E0E1530A
:10541000FF4D8081892BECE5F3E582AF85AF83E01A
:1054200080939E538093A15391E093AF96AF84AF46
:1054300087AF1CC0EC2FF0E0E153FF4D808181600D
:10544000ECE5F3E582AF84AF83AF85AF81E0809375
:105450009F538093A1530AC0EC2FF0E0E153FF4D1E
:1054600080818560ECE5F3E582AF83AF8091965350
:1054700084700F94360581E0CF9108951F93CF93E8
:10548000DF930097E9F1EC011AAA1BAA0E94871783
:1054900087E00E9458C1162F84E00E9458C1862FD1
:1054A000612F0F940D0689E10E9458C1613071058A
:1054B0008105910521F481E00F948C1903C080E0EF
:1054C0000F948C190E94351D813031F4CE010E9459
:1054D000EE1C0E94862004C0CE010E94841CAADE1D
:1054E0000F941D1C0F941905CE010E9448210F94A2
:1054F000A81A0E94EE0F0E943F110E94BE1119824D
:10550000DF91CF911F910895CF93DF93009791F092
:10551000FC012081243071F4EC010E943620CE0180
:10552000ADDF0F9419191092BC3E63E0CE010E94CA
:105530003C141982DF91CF910895882321F081E0F6
:105540008093C13E08951092C13E08958091C13E5E
:105550000895AF92BF92CF92DF92EF92FF920F9396
:105560001F93CF93DF93DC01009709F45AC04115D4
:10557000510509F458C02115310509F456C0FA0146
:10558000C081D0E0F901008110E06115710561F082
:10559000FC017C01E60EF71E9191C90FD11D0C0F85
:1055A0001D1FEE16FF06C1F7F9017B016D01DA013F
:1055B000CC930083F601E60FF71F8CE280838BE12A
:1055C00081835B01A2E0AA0EB11CAC0CBD1C8C2F28
:1055D00082958F700F942425F50180835701F3E0A5
:1055E000AF0EB11CAC0CBD1C8C2F8F700F942425FA
:1055F000D5018C93E7012496CC0DDD1D802F82957B
:105600008F700F9424258883D7011596E601CA0F61
:10561000DB1F802F8F700F9424258883C701069687
:1056200005C0CB0103C0CB0101C0CB01DF91CF91FD
:105630001F910F91FF90EF90DF90CF90BF90AF90B0
:1056400008953F924F925F926F927F928F929F92B6
:10565000AF92BF92CF92DF92EF92FF920F931F9380
:10566000CF93DF93CDB7DEB76397CDBFDEBF7C01AD
:105670006B013A01290189E10E9458C1B62E82E0EE
:105680000E9458C1162FE114F10409F446C1C11457
:10569000D10409F444C16B3008F449C161147104A8
:1056A00009F43FC14114510409F43DC1FE01329691
:1056B000CE014296C192D1922BE0C20ED11CE817C6
:1056C000F907C1F78DE0D701D6968C93D69782E083
:1056D00090E0D4968D939C93D5978AE0D7968C933F
:1056E000F701F896EA8BFB8B41E0BE016F5F7F4FBD
:1056F000CF010E9442182981D701D4968D919C91A7
:10570000D597820F911D9C012F5F3F4FD4962D930B
:105710003C93D597F701E80FF91F2CE226ABB1E0D7
:10572000BB1590F5B12C0F2EFCE2AF2EF02D61C011
:10573000EB2DF0E0EE0FFF1F81E090E08C0F9D1F3E
:10574000E80FF91FC180D280D701D4968D919C912A
:10575000D597C696F601418550E0B6018E0D9F1D86
:105760000F942C56D60119962C91F70184A995A96E
:10577000820F911D9C012F5F3F4F24AB35ABE80F8B
:10578000F91FA6AAB39405C0B12C0F2EFCE2AF2ED0
:10579000F02D0F941A1CB81658F230C0EB2DF0E023
:1057A000EE0FFF1F81E090E08C0F9D1FE80FF91FA7
:1057B000C180D280D701D4968D919C91D597C69601
:1057C000F601418550E0B6018E0D9F1D0F942C56B9
:1057D000D60119962C91F70184A995A9820F911DE4
:1057E0009C012F5F3F4F24AB35ABE80FF91FA6AAF2
:1057F000B3940F941A1C8695B81680F21B3008F4E7
:1058000066C01C3028F01E3028F01051133010F004
:1058100010E001C011E00F2EFAEB8F2EF1E29F2E67
:10582000F02D5701F6E3AF0EB11C0F2EFCE23F2E18
:10583000F02DC12ED12CC601880F991FC80ED91E7C
:10584000CC0CDD1CCC0CDD1CC60CD71CD6011A966A
:105850008C911F928F939F928F92F70184A995A9A3
:10586000C6968E0D9F1D9F938F930F945A56F501E8
:1058700001900020E9F73197EA19FB09D701D49686
:10588000ED93FC93D597CF01C696F601418550E084
:10589000B6018E0D9F1D0F942C56D60119962C9192
:1058A000F70184A995A9820F911D9C012F5F3F4F9D
:1058B00024AB35ABE80FF91F36AA1F5F0F900F908E
:1058C0000F900F900F900F90123008F4B2CF01306C
:1058D000D9F4D701D4968D919C91D597C696820123
:1058E00001501F4FF801408150E0B2018E0D9F1D05
:1058F0000F942C56D8012C91F70184A995A9820FF9
:10590000911D84AB95AB18C0D701D496ED91FC9155
:10591000D597EE0DFF1D16AA0FC080E02EC080E0C7
:105920002CC080E02AC080E028C080E026C041145E
:10593000510409F0BBCEF9CFA7014D5A5D4FF701D5
:10594000E75AFD4F8081FA01808397012C5A3D4F21
:1059500037968081D9018C93F70164A975A96250AB
:1059600071098A899B89F5DD0296D701D4968D93BA
:105970009C93D59781E0D2968C936396CDBFDEBF82
:10598000DF91CF911F910F91FF90EF90DF90CF901B
:10599000BF90AF909F908F907F906F905F904F904F
:1059A0003F9008952F923F924F925F926F927F9215
:1059B0008F929F92AF92BF92CF92DF92EF92FF921F
:1059C0000F93CF93DF93CDB7DEB76097CDBFDEBF28
:1059D000009709F46EC06115710509F46AC09B0156
:1059E000FE013196DE01519621933193255F3F4FA1
:1059F000EA17FB07C9F76A017B011C01B12C12C031
:105A0000EB2DF0E0EE0FFF1F81E090E08C0F9D1F6B
:105A1000E80FF91F808191810E94A017882309F463
:105A200048C0B3940F941A1CB81650F30F9475190C
:105A30004B015C010F945E192B013C0184E295E45B
:105A40000E94F5CE082F81110BC09EE1890E911C9A
:105A5000A11CB11C84149504A604B70450F115C010
:105A600040E050E06AEA72E480E30E945D1D24E2B7
:105A700035E4A601B701C101E4DD46E256E46AEA75
:105A800072E482E30E945D1D0EC000E024E235E472
:105A9000A601B701C101D5DD40E050E06AEA72E439
:105AA00082E30E945D1D84E295E40E94EFCE0E9495
:105AB00087176096CDBFDEBFDF91CF910F91FF902A
:105AC000EF90DF90CF90BF90AF909F908F907F909E
:105AD0006F905F904F903F902F900895009789F0BE
:105AE0006115710571F04115510559F02115310508
:105AF00041F0FC011082FB011082FA011082F901D1
:105B0000108208952F923F924F925F926F927F92F0
:105B10008F929F92AF92BF92CF92DF92EF92FF92BD
:105B20000F931F93CF93DF93CDB7DEB72597CDBFEC
:105B3000DEBF009709F461C04115510509F45FC04B
:105B40002115310509F45DC0613BE4E07E0708F4EE
:105B50005AC02B01E0EB4E1AE4E05E0A612C712C76
:105B6000E2E04E165104610471040CF454C02C831D
:105B70003D831A018C01C12CD12C7601C3944B01B9
:105B8000A12CB12CB501A4014C195D096E097F0946
:105B9000C8010F94514C9E012F5F3F4F41E050E0F0
:105BA000BE016D5F7F4FC8010F94054981112DC063
:105BB0008B818B3191F18FEFC81AD80AE80AF80A65
:105BC000C414D504E604F704ECF225C089819A8157
:105BD0000497E8F0B10185E094E40F941629982F1A
:105BE000882341F16C817D8187E094E40F9416292C
:105BF00091E081111FC090E01DC090E01BC090E0BB
:105C000019C090E017C090E015C090E013C090E07C
:105C100011C090E00FC090E00DC09E012F5F3F4F7C
:105C200044E050E065E074E4C8010F94054988231E
:105C300069F2EFCF892F2596CDBFDEBFDF91CF91DF
:105C40001F910F91FF90EF90DF90CF90BF90AF909A
:105C50009F908F907F906F905F904F903F902F908C
:105C600008950097A9F061157105B1F0FC019C0140
:105C7000260F371F60E070E0CB0141914D3021F4D9
:105C80006F5F7F4F8F4F9F4F2E173F07B1F70895DC
:105C900060E070E0CB01089560E070E0CB01089512
:105CA0002F923F924F925F926F927F928F929F922C
:105CB000AF92BF92CF92DF92EF92FF920F931F931A
:105CC000CF93DF9300D01F92CDB7DEB7009709F4D2
:105CD00055C00115110509F453C0613B7440C0F46F
:105CE000F801108211821282138280E04CC0098177
:105CF0001A81B801C101B5DF460E571E681E791E14
:105D00000815190500F1C00ED11EE11CF11C0BC0D5
:105D10000B831C8349011A015C01C12CD12C760133
:105D2000412C512C3201B701A601C5010F94514CF1
:105D30009E012F5F3F4FA401B101C5010F9405499A
:105D40008823A9F21FC0F6E24F16510461047104C2
:105D500040F4EB81FC81108211821282138281E077
:105D600012C0F5E24F1A510861087108EB81FC81FD
:105D7000408251826282738281E005C080E003C06C
:105D800080E001C080E02496CDBFDEBFDF91CF91DF
:105D90001F910F91FF90EF90DF90CF90BF90AF9049
:105DA0009F908F907F906F905F904F903F902F903B
:105DB0000895009741F0FC01EB5AFD4F608171811D
:105DC00082819381089560E070E0CB01089500978F
:105DD00039F0FC01EB5AFD4F1082118212821382BE
:105DE0000895CF93DF93009781F12091C13E211157
:105DF0002CC0EC010F940516882339F1CE010E94C6
:105E000002970F94DE150F941B011F928F938EEB58
:105E100091E29F938F93C5E0D4E4DF93CF930F94E7
:105E20005A5609900020E9F72197AE014550544495
:105E300020E065E074E482E299E30F940C210F9076
:105E40000F900F900F900F900F90DF91CF910895CA
:105E50002115310551F0505861097109F90140834C
:105E600051836283738381E0089580E008950097F1
:105E700019F0FC01848D089580E008954F925F929F
:105E80006F927F928F929F92AF92BF92EF92FF920A
:105E90000F931F93CF93DF931F92CDB7DEB7E1141B
:105EA000F10409F465C0480159012A013B01182F8A
:105EB000C7010E947B17143031F484E10E9434C181
:105EC0009B01AC0105C085E10E9434C19B01AC017E
:105ED0002115310541055105F9F084189508A608EA
:105EE000B708880C991CAA1CBB1CD501C401880FDB
:105EF000991FAA1FBB1F880F991FAA1FBB1FBC0198
:105F0000CD01680D791D8A1D9B1D0F941154822EA1
:105F1000932EA42EB52E0EC088248A940F2EF0EE58
:105F20009F2EF02D0F2EF5EFAF2EF02D0F2EF5E05A
:105F3000BF2EF02D082D192D2A2D3B2D4BE0BE0133
:105F40006F5F7F4FC7010F949028F70101900020E9
:105F5000E9F73197EE19FF09D7011996EC931997D4
:105F600081E01B968C93682D792D8A2D9B2D04C082
:105F700060E070E080E090E00F90DF91CF911F91A2
:105F80000F91FF90EF90BF90AF909F908F907F9078
:105F90006F905F904F9008952F923F924F925F9233
:105FA0006F927F928F929F92AF92BF92CF92DF9229
:105FB000EF92FF920F931F93CF93DF93CDB7DEB78E
:105FC0002897CDBFDEBFCA01E982FA82CD82DE8288
:105FD000AB82BC826115710509F4B7C0009709F462
:105FE000B6C0EF2809F4B5C0802E912EA22EB32E94
:105FF00025EB82169104A104B10438F00F2EF4EBC6
:106000008F2E912CA12CB12CF02DDB01CD90DD90A9
:10601000ED90FC90B0E8DB1AE108F108FB01C082CA
:10602000D182E282F38221E020934732F2E08F16A0
:106030009104A104B10408F46AC0FB0127E432E32F
:106040002F83388794012150304C220F331F220FA9
:10605000331F1B01220E331E4601570100E010E0E2
:106060009801448155816681778150586109710991
:1060700044835583668377834190519061907190FA
:1060800044195509660977091416150616061706E8
:1060900034F441E0AF81B88511964C9304C0AF81D0
:1060A000B88511961C92AF81B88511965C911197B5
:1060B000BD016F5F7F4F6F8378874C91541781F0DC
:1060C000D801AA0FBB1FAA0FBB1FA80FB91F4D9263
:1060D0005D926D927C9213970F5F1F4F2F4F3F4F32
:1060E0004081518162817381C416D506E606F706A8
:1060F00014F46A017B01481559056A057B0514F4FF
:106100004A015B01E215F30509F0ABCF05C046017A
:10611000570100E010E09801A981BA810D931D9309
:106120002D933C931397ED81FE81309721F080826F
:106130009182A282B382EB81FC81309761F0C082B0
:10614000D182E282F38281E007C080E005C080E076
:1061500003C080E001C081E02896CDBFDEBFDF91A3
:10616000CF911F910F91FF90EF90DF90CF90BF9054
:10617000AF909F908F907F906F905F904F903F90E7
:106180002F9008958F929F92AF92BF92CF92DF92FD
:10619000EF92FF920F931F93FC01892BA1F16115E0
:1061A000710599F10081118122813381848195816A
:1061B000A681B781081719072A073B0744F5C08451
:1061C000D184E284F384C816D906EA06FB060CF5EE
:1061D00084849584A684B784C814D904EA04FB0493
:1061E000D4F488159905AA05BB05BCF40C151D054A
:1061F0002E053F0524F481E0FB0180830FC0FB01E5
:10620000108281E00BC080E009C080E007C080E020
:1062100005C080E003C080E001C080E01F910F91C5
:10622000FF90EF90DF90CF90BF90AF909F908F90B6
:1062300008953F924F925F926F927F928F929F92BA
:10624000AF92BF92CF92DF92EF92FF920F931F9384
:10625000CF93DF93009709F448C02115310509F465
:1062600046C0443051056105710508F442C06A0119
:106270007B01E4E0CE1AD108E108F108E1F159010F
:106280008C01912C312C812C412C512C3201E501B7
:10629000C90DD11DBE01C201880F991F880F991F1A
:1062A000800F911F6FDF882379F08881882311F098
:1062B000839401C0339483E0480E511C611C711C0F
:1062C0009394E2E0E91550F08FEF481A580A680AF3
:1062D000780A4C145D046E047F04C8F2882069F0CB
:1062E00081E0332059F080E009C080E007C080E001
:1062F00005C080E003C081E001C081E0DF91CF9163
:106300001F910F91FF90EF90DF90CF90BF90AF90D3
:106310009F908F907F906F905F904F903F900895E7
:106320002F923F924F925F926F927F928F929F92A5
:10633000AF92BF92CF92DF92EF92FF920F931F9393
:10634000CF93DF93CDB7DEB76B97CDBFDEBF782E8F
:10635000D92E662E798B19821A821B821C821D828D
:106360001E821F82188619861A861B861C861D8629
:106370001E861F86188A82E00E9458C16B3008F47E
:10638000BBC00F94531D882309F4CEC00F94421D47
:1063900080918B3C823009F0B1C084E190E40F948D
:1063A000FF4BACC08F8A988E530162010F2EF0E72D
:1063B000EF2EFFE2FF2EF02D04EB10E020E030E0A6
:1063C00047E75FE2B401832DE7DD882331F1409197
:1063D000702F5091712F6091722F7091732F24E75D
:1063E0003FE287E79FE225DF882361F08091742FE9
:1063F00090E0A0E0B0E0EF89F88D80839183A283E4
:10640000B38314C08EEF90E0A0E0B0E0EF89F88D88
:1064100080839183A283B38309C08FEF90E0A0E0D3
:10642000B0E0F40180839183A283B3833394F0E3DB
:106430008F1AFDEF9F0A84E0480E511C94E0690E0C
:10644000711CA6E03A12AECF298C3A8C6B8C862C4C
:1064500099886894552452F80F2EF5E44F2EF02DAC
:106460000F2EF2E5DF2EF02D0F2EFCE4CF2EF02DB7
:10647000AB88BC886D887E88898A9A8AF3010191ED
:106480001191219131913F01D5014D915D916D9116
:106490007D915D017401852DF1DC6531710581050A
:1064A00091051CF4F40142861AC0F10180819181AA
:1064B000A281B3810097A105B10529F4A989BA8900
:1064C0001A96CC920CC00197A105B10521F4E98977
:1064D000FA89D28604C0A989BA891A964C92539433
:1064E000BCE08B0E911CE0E32E1AEDEF3E0AF6E0C5
:1064F0005F12C2CF81E018C080E016C0272C3D2C6F
:10650000CE0101968B8B9C8BDE011996AD8BBE8BD9
:106510002C01872C9D2C6894772472F8298E3A8E52
:10652000372C6B8E3D013ECF6B96CDBFDEBFDF912A
:10653000CF911F910F91FF90EF90DF90CF90BF9080
:10654000AF909F908F907F906F905F904F903F9013
:106550002F9008951F93CF93DF93009709F4DAC02B
:10656000EC018881843069F128F4813049F082306F
:10657000C9F0D0C0883011F1893009F4A7C0CAC071
:106580008B81813009F0C6C08C81813009F0C2C096
:106590000F943B19CE010E943E2A62E0CE010E9478
:1065A0003C14B8C080917F48813029F463E0CE016B
:1065B0000E943C14AFC00E942F1CACC00E94F04E41
:1065C000A9C0CE010E94212282E00E9458C16B30F6
:1065D00040F463EC78E387E49CE30E946D18182F85
:1065E00010C00F94531D8823E1F063EC78E387E437
:1065F0009CE30E946D18182F67E57CE38CEB9DE40B
:106600008FDE113071F482E00E9458C1162F87E4AA
:106610009CE30E940A10612F84ED9FE30E942C12DC
:1066200007C083EC98E30E94AB17882309F465C088
:1066300047E55CE363EC78E3CE01B4D95EC00F9428
:10664000FE06882309F463C00F94B91A64E170E46C
:10665000CE010E9475250F94ED0659C089818111E4
:1066600059C0CE010E94E921882341F00F94B91A44
:1066700064E170E4CE010E9475254CC01AAA81E045
:106680008BAB48C08AA9882309F444C08981811151
:1066900041C0CE010E94B721882341F00F94B91A5E
:1066A00064E170E4CE010E94752534C01AAA32C09C
:1066B0000F94FE06882371F10F94B91A64E170E417
:1066C000CE010E9475250F94ED0624C0CE010E94D4
:1066D000212263EC78E387E49CE30F94440B813040
:1066E00031F083EC98E30F94990B882399F063ECD5
:1066F00078E3CE010F94C20E0DC0FE01E95CFD4FA0
:106700008081813009F49BCF823091F6BBCF8AA97A
:106710008111A4CFDF91CF911F910895CF930E9453
:1067200052C9C82F88E10E9458C1C61741F061E0E4
:1067300080E00F941B0361E081E00F941B03CF9175
:106740000895CF930E9452C9C82F88E10E9458C172
:10675000C61749F061E080E00F941B0361E081E01F
:106760000F941B0308C060E080E00F941B0360E0FF
:1067700081E00F941B03CF910895CF93DF93EC0139
:106780008091C13E882319F0E2E2F9E302C0E9E218
:10679000FAE3209729F18BE7888388E689839CE2D6
:1067A0009A8382E68B839C838CE68D838DE78E8330
:1067B0001F8221E047E050E0BE01CF010F940C2181
:1067C0000E946DB9873061F48091C13E811108C08B
:1067D00021E047E050E0BE0182E299E30F940C21F2
:1067E000DF91CF91089580918C3C0895CF92DF92F4
:1067F000FF920F931F93CF93DF931F921F92CDB7FA
:10680000DEB79FEF980F923008F045C090918C3C16
:10681000992309F443C0813019F00DEC1EE302C046
:1068200009E21AE3F82E81E6898384E78A8321E06E
:1068300042E050E0BE016F5F7F4FC8010F940C2112
:106840000F94E3190F94FA19643F71408105910583
:10685000C8F3C8010E94B7A00F94E3190F94FA1966
:10686000643F714081059105C8F38F2D0E94A4C932
:106870006C018F2D0E94A4C9FC0101900020E9F752
:106880003197AF01481B590B41F0B601C8010E9476
:1068900027A191E003C090E001C090E0892F0F9004
:1068A0000F90DF91CF911F910F91FF90DF90CF90CC
:1068B0000895EF92FF920F931F93CF93DF93CDB77D
:1068C000DEB72797CDBFDEBF7C01FB0184818D83BE
:1068D00085818E8386818F8380819181A281B3811E
:1068E00089839A83AB83BC83870180EAE81688E0BA
:1068F000F80629F460E183E00F94773314C080EB4D
:10690000E81688E0F80629F460E283E00F94773314
:1069100013C080EAE81689E0F80629F460E184E013
:106920000F94773312C0003B89E0180729F460E226
:1069300084E00F94773312C0003A8AE0180729F4F4
:1069400060E185E00F94773310C0003B8AE01807C0
:1069500029F460E285E00F94773307C0003A1B40CA
:1069600021F460E186E00F947733BE016F5F7F4FC3
:10697000C7010E944E6F2796CDBFDEBFDF91CF913A
:106980001F910F91FF90EF900895DC01892BE1F0AA
:10699000E62FE695E695E69580E2E89FF001112462
:1069A000FA5F8085677021E030E002C0220F331F5C
:1069B0006A95E2F7282381E009F480E08C93119630
:1069C0008C93119712961C920895CF93DF930097A2
:1069D00009F4A5C06D3209F0A4C03091A80621E0E9
:1069E000432F407235FF20E0FC01208331812317C3
:1069F00009F499C0EC01442309F46BC0311169C05A
:106A00000F948D150097F9F40E94A62A811119C0E0
:106A100086E0E9EDF1E2A5E0B4E401900D928A95FB
:106A2000E1F7E5E0F4E401900020E9F73197AF01E8
:106A30004550544421E065E074E482E299E30F9408
:106A40000C211A8268C0803D974008F50E94A62A52
:106A5000811119C086E0EFEDF1E2A5E0B4E4019008
:106A60000D928A95E1F7E5E0F4E401900020E9F762
:106A70003197AF014550544421E065E074E482E26F
:106A800099E30F940C210F94A1151A8244C081E060
:106A90008A830F94A1150E94A62A81113CC086E02A
:106AA000E5EEF1E2A5E0B4E401900D928A95E1F7FC
:106AB000E5E0F4E401900020E9F73197AF0145509B
:106AC000544421E065E074E482E299E30F940C21E0
:106AD00022C01A8281E090E00F94B4150E94A62A89
:106AE000811119C086E0EBEEF1E2A5E0B4E401907B
:106AF0000D928A95E1F7E5E0F4E401900020E9F7D2
:106B00003197AF014550544421E065E074E482E2DE
:106B100099E30F940C21888189838A8105C080E0E4
:106B200003C080E001C080E0DF91CF91089583EF42
:106B300097E40C94C2D608950E94A62A811117C02A
:106B400067E874E482E299E30F94B82080910945E4
:106B5000813029F547E854E469E874E482E299E376
:106B60000E94DABE87E894E40D94A920089567E8AE
:106B700074E482E299E30E94069E80910945813087
:106B800071F42FE63CE347E854E469E874E482E2F8
:106B900099E30E94F79D87E894E40D94A920089555
:106BA0000E94F591882341F01EDE811105C085E821
:106BB00091E40C94322508950E94A62A81112EC0DA
:106BC00063EA71E489E29AE30E94069E809125427D
:106BD000813021F50E94A62A811112C062E48091C1
:106BE0002239909123390E94336E4091A3415091F4
:106BF000A44121E065EA71E482E299E30F940C215B
:106C00002FE63CE343EA51E465EA71E489E29AE362
:106C10000E94F79D83EA91E40D94A9200895CF92F4
:106C2000DF92EF92FF920F931F93CF93DF930E9417
:106C3000A62A882319F002E219E302C009E21AE346
:106C400084E991E40E9432A0882349F0CCDD8111CF
:106C500006C064E971E4C8010E9418258BC28091C6
:106C6000A2418150823008F057C10E94B4A0811126
:106C700004C0B9DD882309F414C36FE470E48DEC1B
:106C80009EE30E94A99F80918041813009F072C2E9
:106C9000E0904F40F090504082E0E816F10408F494
:106CA00000C38091A241813039F4809154408F7D9E
:106CB0008C3409F0CBC00AC080915440843209F072
:106CC000C5C080915540833509F0C0C00E94A62AF6
:106CD000811156C087E0E1EFF1E2A5E0B4E4019054
:106CE0000D928A95E1F7E5E0F4E401900020E9F7E0
:106CF0003197AF014550544420E065E074E482E2EE
:106D000099E30F940C211092514010925240E114DB
:106D1000F104A1F080E090E0CFE4D0E4FC01E15B7D
:106D2000FF4B658182E299E30F9498218A819B81D0
:106D300001968A839B838E159F0580F30F94CB1A4F
:106D40001F928F9388EF91E29F938F93C5E0D4E4D5
:106D5000DF93CF930F945A5609900020E9F72197BB
:106D6000AE014550544421E065E074E482E299E3C9
:106D70000F940C210F900F900F900F900F900F9089
:106D80000F94CB1A882371F181E00E94638D8130CA
:106D900069F48FE490E40E94FF9F8FE490E40E94E6
:106DA00011A00F94A81A0E94A5A202C00E9406A3D7
:106DB000E6EEF2E4808190E0DC01AA51BD4B25852E
:106DC0003685880F991FFC01EA51FD4B41815281A4
:106DD0001F960C9161E08FE69CE30E9458250F946A
:106DE000D21B93C0E0928341F09284410F94CB1A5E
:106DF000682FC8010E9441900E94A62A811185C077
:106E00000F94CB1A1F928F938091A2411F928F9360
:106E10008EEF91E29F938F93C5E0D4E4DF93CF93FD
:106E20000F945A5609900020E9F72197AE0145507A
:106E3000544421E065E074E482E299E30F940C216C
:106E4000EDB7FEB73896EDBFFEBF5FC00E94A62A21
:106E5000811157C08091A241823049F48091544001
:106E6000843229F480915540873409F44AC086E081
:106E7000ECE1F2E2A5E0B4E401900D928A95E1F72D
:106E8000E5E0F4E401900020E9F73197AF014550C7
:106E9000544420E065E074E482E299E30F940C210D
:106EA000EFE4F0E41282138280819181892BA9F0B2
:106EB00080E090E0EF01FC01E15BFF4B658182E245
:106EC00099E30F9498218A819B8101968A839B8301
:106ED000288139818217930770F3E5E0F4E480E2BA
:106EE00090E08083918301900020E9F73197AF0112
:106EF0004550544421E065E074E482E299E30F9444
:106F00000C218FE490E40E9411A08FE490E40E9491
:106F1000FF9F0F94A81A2EC10F940F166B017C01CE
:106F20006FE470E48DEC9EE30E942D9F8091804180
:106F3000813039F0F5E6CF16D104E104F10408F40C
:106F400019C10F94261680918041813079F48FE425
:106F500090E40E9482A0882321F0E0908241F12CED
:106F600040C0E0904F40F09050403BC00F2EFFE4F7
:106F7000EF2EF0E4FF2EF02DF70181818F938081B9
:106F80008F9382E292E29F938F93C5E0D4E4DF93E4
:106F9000CF930F945A5609900020E9F72197AE013C
:106FA0004550544421E065E074E482E299E30F9493
:106FB0000C21109282410F900F900F900F900F9024
:106FC0000F90F701808191818739910530F086E932
:106FD00090E080934F4090935040E0904F40F0906D
:106FE00050400E94A62A81115DC0FF92EF9281E479
:106FF00092E29F938F93C5E0D4E4DF93CF930F94F5
:107000005A5609900020E9F72197AE0145505444A3
:1070100020E065E074E482E299E30F940C21109281
:107020005140109252400F900F900F900F900F9080
:107030000F90E114F104A1F080E090E0CFE4D0E4FF
:10704000FC01E15BFF4B658182E299E30F9498219B
:107050008A819B8101968A839B838E159F0580F38D
:107060000F94CB1A1F928F9388EF91E29F938F9387
:10707000C5E0D4E4DF93CF930F945A5609900020D3
:10708000E9F72197AE014550544421E065E074E4EE
:1070900082E299E30F940C210F900F900F900F90C4
:1070A0000F900F900F94CB1A882371F181E00E940A
:1070B000638D813069F48FE490E40E94FF9F8FE438
:1070C00090E40E9411A00F94A81A0E94A5A202C0E9
:1070D0000E9406A3E6EEF2E4808190E0DC01AA5172
:1070E000BD4B25853685880F991FFC01EA51FD4B64
:1070F000418152811F960C9161E08FE69CE30E94D2
:1071000058250F94D21B30C0E0928341F092844105
:107110000F94CB1A682FC8010E9441900E94A62AA2
:10712000811122C00F94CB1A1F928F938EE492E2AA
:107130009F938F93C5E0D4E4DF93CF930F945A5677
:1071400009900020E9F72197AE014550544421E011
:1071500065E074E482E299E30F940C210F900F90A4
:107160000F900F900F900F908FE490E40E94FF9F7C
:107170000F94A81A0F945816693C71058105910562
:1071800008F48FC00F946F160E94A62A81114AC07E
:107190008AE0E2E6F2E2A5E0B4E401900D928A957D
:1071A000E1F7E5E0F4E401900020E9F73197AF0161
:1071B0004550544420E065E074E482E299E30F9482
:1071C0000C21EFE4F0E41282138280819181892BFB
:1071D000A9F080E090E0EF01FC01E15BFF4B6581ED
:1071E00082E299E30F9498218A819B8101968A8398
:1071F0009B83288139818217930770F3E5E0F4E4DB
:1072000080E290E08083918301900020E9F731973C
:10721000AF014550544421E065E074E482E299E313
:107220000F940C2184E590E40E9490A18823A9F199
:107230008091A24181110BC0EAEAF2E481E38083EC
:1072400082E3818383E3828384E3838314C0813078
:1072500041F4EAEAF2E480E38083818382838383DA
:107260000AC0EAEAF2E481E3808382E3818383E374
:10727000828384E3838321E044E050E06AEA72E49D
:107280008DEC9EE30F940C2121E044E050E06AEA8B
:1072900072E482E299E30F940C218FE490E40E945F
:1072A000FF9FDF91CF911F910F91FF90EF90DF90A3
:1072B000CF9008958F929F92AF92BF92CF92DF921C
:1072C000EF920F931F93CF93DF93EC0180E00E9426
:1072D00034C14B015C01209709F45CC11F8EFE0193
:1072E000E05BFD4F1082CE010E940520882309F447
:1072F00051C16E0186E3C80ED11CBE01615E7F4F95
:10730000C6010E94BAF98E8F81111FC00E94A62A61
:10731000811119C08BE1ECE6F2E2A5E0B4E4019042
:107320000D928A95E1F7E5E0F4E401900020E9F799
:107330003197AF014550544421E065E074E482E2A6
:1073400099E30F940C2181E08F8F61EB76E4C60105
:107350000E9427FFFE01E15BFD4F808381EB96E4F5
:107360000E941CC88823A1F181E0FE01E05BFD4F73
:10737000808381EB96E40E94B9C70E94A62A8111FE
:1073800027C0FE01E05BFD4F80811F928F933197F4
:1073900080811F928F9387E892E29F938F9305E0FD
:1073A00014E41F930F930F945A56F8010190002094
:1073B000E9F73197AF014550544421E0B80182E22A
:1073C00099E30F940C21ADB7BEB71896ADBFBEBF01
:1073D0008F8D813039F0FE01E05BFD4F808181307F
:1073E00009F05CC00E94A62A811119C08CE1EAE96B
:1073F000F2E2A5E0B4E401900D928A95E1F7E5E0B0
:10740000F4E401900020E9F73197AF01455054446E
:1074100021E065E074E482E299E30F940C21689422
:10742000EE24E2F806EB12E2A5019401BE01685ECB
:107430007F4FCE0106960E9478578D8340E050E042
:10744000BA01CE010E94E72E8D81882309F4A2C0E3
:1074500082E00E9458C1062F8BE00E9458C121E0B3
:10746000611120E0BE016C5C7F4F44E150E4C60135
:107470000E947B50CE010E945A1C9E01265A3D4F0D
:10748000AE01475A5D4FBE016C5A7D4FCE018D5AF9
:107490009D4F0E946E2D0F94F2077CC08E010A5FF3
:1074A0001F4FB80184E190E40E9450568D838111F2
:1074B00039C0A5019401BE01685E7F4FC8010E94DA
:1074C000B2538D8340E050E0BA01CE010E94E72E16
:1074D0008D81882309F45EC082E00E9458C1062F86
:1074E0008BE00E9458C121E0611120E0BE016C5C7C
:1074F0007F4F44E150E4C6010E947B50CE010E94C0
:107500005A1C9E01265A3D4FAE01475A5D4FBE019F
:107510006C5A7D4FCE018D5A9D4F0E946E2D0F9457
:10752000F20738C08E010B5A1D4F0F2EF4E1AF2E1B
:10753000F0E4BF2EF02DF5016285738520E032E086
:10754000A601C5010E94502E015011096E01FDEAED
:10755000CF1AFDEFDF0AD5011A966D917C911B972A
:107560009801A601C5010E94822DFE01E75AFD4F38
:10757000D6018C918083C65ADD4FF80180818883C3
:10758000D5011A964D915D916D917C911D97C50124
:107590000F94514CDF91CF911F910F91EF90DF909D
:1075A000CF90BF90AF909F908F9008956DE280EC48
:1075B00098E30BDA882309F467C08091FB328823B3
:1075C00009F446C00E949B6184E0809326060F94D4
:1075D000CA1481EB96E40E9473D58FE69CE36ADEC1
:1075E0008091BF3E8823F1F00E9437D3813019F09B
:1075F000823069F017C08091BE3E882329F081EB6C
:1076000096E40E94D5D20EC00E94A8D20BC08091F1
:10761000BE3E882329F081EB96E40E9457D402C035
:107620000E9422D41092FB320F94D21B8FE69CE36F
:107630000E94F12281110F943B198FE69CE30E9476
:107640003E2A6091B23E8FE69CE30E943C141CC02F
:107650000F94D21B0F94191966E08FE69CE30E94E9
:107660003C1461E085E79CE30E941E560E949D53F6
:107670000F94392A0E94716181E08093FB3284E08B
:10768000809325060F94CA148091FB32882331F031
:107690000E94EF5F8111FCCF8091FB3208954F92E1
:1076A0005F926F927F928F929F92AF92BF92CF9292
:1076B000DF92EF92FF921F93CF93DF93CDB7DEB7A8
:1076C0002797CDBFDEBF7C011092804810E00F2EBF
:1076D000812CFBE49F2EA12CB12CF02D0F2EF5E078
:1076E000CF2EF4E4DF2EF02D0F2EF0E84F2EF5E232
:1076F0005F2E612C712CF02D111120C080E096E9D5
:10770000A0E0B0E0F70180839183A283B3838AE095
:10771000EBEBF2E2D60101900D928A95E1F7F601CA
:1077200001900020E9F73197AF014550544421E022
:10773000B60182E299E30F940C215CC0113001F58F
:1077400080EC92E1A0E0B0E0F70180839183A28316
:10775000B38389E0E5ECF2E2D60101900D928A95BF
:10776000E1F7F60101900020E9F73197AF014550AC
:10777000544421E0B60182E299E30F940C213AC00F
:107780001230E9F4D7014D925D926D927C9213977D
:1077900089E0EEECF2E2D60101900D928A95E1F7D4
:1077A000F60101900020E9F73197AF0145505444AC
:1077B00021E0B60182E299E30F940C211BC0F7018E
:1077C00080829182A282B38289E0E7EDF2E2D60163
:1077D00001900D928A95E1F7F60101900020E9F7FA
:1077E0003197AF014550544421E0B60182E299E35C
:1077F0000F940C21D70114968C9114978D831596B4
:107800008C9115978E8316968C9116978F838D91F8
:107810009D910D90BC91A02D89839A83AB83BC83ED
:1078200060E185E00F947733BE016F5F7F4F80EAA0
:107830009AE00E944E6F0F94451B08C083EF97E4B7
:107840000E94C2D6813041F00E94EB1B0F94581B5E
:10785000803A9F4098F37AC011111DC08CE0E0EE91
:10786000F2E2A5E0B4E401900D928A95E1F7E5E03B
:10787000F4E401900020E9F73197AF0145505444FA
:1078800021E065E074E482E299E30F940C2182E048
:107890008093804878C01130E9F48BE0ECEEF2E29E
:1078A000A5E0B4E401900D928A95E1F7E5E0F4E4F7
:1078B00001900020E9F73197AF014550544421E091
:1078C00065E074E482E299E30F940C2181E08093F7
:1078D000804859C01230E9F48BE0E7EFF2E2A5E00E
:1078E000B4E401900D928A95E1F7E5E0F4E40190AB
:1078F0000020E9F73197AF014550544421E065E09D
:1079000074E482E299E30F940C2183E08093804831
:107910003AC08BE0E2E0F3E2A5E0B4E401900D921E
:107920008A95E1F7E5E0F4E401900020E9F731976A
:10793000AF014550544421E065E074E482E299E3EC
:107940000F940C2184E0809380481DC01F5F143089
:1079500009F0D2CE89E0EDE0F3E2A5E0B4E40190D5
:107960000D928A95E1F7E5E0F4E401900020E9F753
:107970003197AF014550544421E065E074E482E260
:1079800099E30F940C212796CDBFDEBFDF91CF91F5
:107990001F91FF90EF90DF90CF90BF90AF909F909E
:1079A0008F907F906F905F904F900895CF92DF926D
:1079B000EF92FF920F931F93CF938FE69CE30E9469
:1079C0004F14883009F4D6C08FE69CE30E944F1410
:1079D000863009F4CFC08091CB3E9091CC3E8E345E
:1079E0009C4008F4BEC00E9434C98111B4C0C2C01A
:1079F0000F94131C81111FC00F94161C0E94A62AFD
:107A0000811119C088E1E6E1F3E2A5E0B4E4019058
:107A10000D928A95E1F7E5E0F4E401900020E9F7A2
:107A20003197AF014550544421E065E074E482E2AF
:107A300099E30F940C210F94FF1B811129C09AC068
:107A40008CE1EEE2F3E2A5E0B4E401900D928A95B8
:107A5000E1F7E5E0F4E401900020E9F73197AF01A8
:107A60004550544421E065E074E482E299E30F94C8
:107A70000C210F94A814C0E00F949714882331F0C0
:107A80000F94A814CF5FCA30B9F702C0CA30A0F370
:107A90000F9419190E949D530E94A62A811119C0A2
:107AA0008EE0ECE3F3E2A5E0B4E401900D928A9558
:107AB000E1F7E5E0F4E401900020E9F73197AF0148
:107AC0004550544421E065E074E482E299E30F9468
:107AD0000C210F94A81401E010E0C0E00F2EF3E198
:107AE000CF2EF1E2DF2EF02D0F2EF5E0EF2EF4E495
:107AF000FF2EF02D0F949714882341F10F94A814B2
:107B0000CF5F0E94A62A81111CC01F930F93DF92A2
:107B1000CF92FF92EF920F945A56F70101900020F6
:107B2000E9F73197AF014550544421E0B70182E2B3
:107B300099E30F940C210F900F900F900F900F90DE
:107B40000F900F5F1F4FC33019F0D4CFC33090F2A6
:107B50000F945B000FC00F94091C882309F46BCFAE
:107B600047CF8AEA92E40E94BD330E94A62A81117F
:107B700080CF66CFCF911F910F91FF90EF90DF9054
:107B8000CF900895F8940E94A3640F9422330F9429
:107B90007A030F94DB0360E080E00F9473040F948A
:107BA000392A0E94C09E0F94F7020E947CDD41E0BA
:107BB00060EA78E089E29AE30F946E2165E170E271
:107BC00080EA98E00E945934E0EAF8E083818F7CF3
:107BD0008061838383EA91E40F94A92061E085E8C2
:107BE00091E40E9422A041E060EA7BE08DEC9EE3FC
:107BF0000F946E216EE070E280EA9BE00E9459349F
:107C0000E0EAFBE083818F7C806183838FE490E4F2
:107C10000E94FF9F8FE490E40E9411A061E084E93C
:107C200091E40E9422A01092A2411092A94286E201
:107C300092E40F94A92041E060EA7AE080E49BE3BB
:107C40000F946E2167E070E280EA9AE00E94593456
:107C5000E0EAFAE083818F7C8061838341E060EA1F
:107C600079E082E299E30F946E2160E070E280EAAD
:107C700099E00E945934E0EAF9E083818F7C8061C9
:107C8000838387E894E40F94A9200F9432140F940F
:107C9000A1160F9445180F94E11A0F94C7160F946C
:107CA000B11C0F940A010F947D060E94670FC0E07B
:107CB00060E08C2F0F941B03CF5FC830C9F787E0BB
:107CC0008093A2007894E0E2F6E082E0868384E08C
:107CD00086830E94F0C0811116C00E94F6C10E94E6
:107CE00020C20E9470C60E940DC80E9405C90E9451
:107CF0004CC981E00E94F9C982E00E94F9C981E083
:107D00008093BD3E27C00E94E3C5882309F181E02E
:107D10008093BD3E0E94A62A81111CC08DE1EAE439
:107D2000F3E2A5E0B4E401900D928A95E1F7E5E075
:107D3000F4E401900020E9F73197AF014550544435
:107D400021E065E074E482E299E30F940C2102C023
:107D50001092BD3E0E9499C70F94F2070E94C3C5BE
:107D600081E00F94F7176DE280EC98E30E94C53430
:107D70000E94B8A264E275E483EF97E40E9436CFD4
:107D800083EF97E40E9418CA8FE69CE30E94561482
:107D900080E00F94F60581EB96E40E9473D50F9472
:107DA0002B058FE69CE386DA81E00E9470B980E0C3
:107DB0000E946AB980E00E9473B980E00E9476B99F
:107DC0000E9487170E948E330E94C49E83EF97E41F
:107DD0000E9418CA87E090E262DC0E9437D38130AB
:107DE00029F48091BE3E0E9405D925C00E9437D358
:107DF000823091F481E00E943AD38091BE3E882384
:107E000029F081EB96E40E9457D402C00E9422D44C
:107E100081E00E94ECD30FC00E9437D3833029F455
:107E200085E094E40E941CD506C00E9437D38430BC
:107E300011F40E9443D984E0809326060E9488DDD5
:107E400081E00E94F63382E00E94F6338FE69CE3E5
:107E50000E943E2A82E299E30E94E0AA0E94A30FB8
:107E600007E613E2C5E0D4E40E94973564E275E4C6
:107E700083EF97E40E94B2168FE69CE30E944316BC
:107E80008FE69CE30E94DB158FE69CE30E94F12EB7
:107E90008FE69CE30E94AA320E949C3587DB0E94F9
:107EA000D0350E940F368FE69CE30E94F51B0E949E
:107EB000B5DD0E946DB9833031F50E941E20882304
:107EC00011F10E94A62A81111EC00F94F6181F926C
:107ED0008F931F930F93DF93CF930F945A56FE0106
:107EE00001900020E9F73197AF014550544421E05B
:107EF000BE0182E299E30F940C210F900F900F9036
:107F00000F900F900F908BEC9EE30E94852466EEFD
:107F100072E48FE69CE30E94232666EE72E48FE60D
:107F20009CE30E9477260F94010740DD0FB607FC03
:107F30009BCF80E00E944A7A0E945E7AFFCFEF9248
:107F4000FF920F931F93CF93DF93009749F1611531
:107F5000710541F14115510539F18A017B01EC01AF
:107F60000F94E155F80180839183892B89F0D70123
:107F700020E030E0FE01E20FF31FE491ED932F5F6C
:107F80003F4FF801808191812817390798F302C08B
:107F900020E030E0F701E20FF31F108281E005C01E
:107FA00080E003C080E001C080E0DF91CF911F91AD
:107FB0000F91FF90EF9008950F931F93CF93DF934E
:107FC0000097C9F061157105C1F041155105B9F06F
:107FD000EA018B01FC0165917491C8010F94DA5597
:107FE000F80101900020E9F73197E01BF10BE883DD
:107FF000F98381E005C080E003C080E001C080E03B
:10800000DF91CF911F910F9108957F928F929F9250
:10801000AF92BF92CF92DF92EF92FF920F931F9396
:10802000CF93DF931F921F92CDB7DEB7009709F46D
:108030009BC06115710509F497C0D42E7B018C019A
:10804000AE014F5F5F4FBC0180E594E178DF88238C
:1080500009F48AC089819A815C012FEFA21AB20AC1
:10806000F801E80FF91F20E22083B8016A0D7B1D9B
:10807000AE014F5F5F4F89E394E161DF882309F42C
:1080800073C089819A81A80EB91EF801EA0DFB1D03
:108090008DE0808382E0A80EB11C8AE08183B80164
:1080A0006A0D7B1DAE014F5F5F4F82E294E147DFB7
:1080B000882309F459C0A981BA81AA0EBB1E4801C0
:1080C0008A0C9B1C0F2EFDE07F2EF02DF401708298
:1080D0000F2EFAE0CF2EF02DC182C5010296800F3F
:1080E000911F0E9416C1F401748ED5015E96C58E53
:1080F000DD2059F1A00FB11F8AE0EFE6F3E2019015
:108100000D928A95E1F7F7E2AF0EB11C0E9443C6CB
:10811000BC01C8018A0D9B1D0F943C560E9443C6AA
:10812000FC0101900020E9F73197E81BF90BE131E0
:10813000F10518F4E983FA8304C080E190E08983B3
:108140009A83A981BA81AA0DBB1DF801EA0FFB1F12
:108150008DE0808312968AE08183F801EA0FFB1F8D
:108160001082F701A083B1830F900F90DF91CF9120
:108170001F910F91FF90EF90DF90CF90BF90AF9045
:108180009F908F907F900895CF92DF92EF92FF9211
:108190000F931F93CF93DF931F921F92CDB7DEB73C
:1081A0006115710591F14115510579F1009769F15A
:1081B0007A016B018C0119821A82AE014F5F5F4F09
:1081C00089EF92E1BCDE882301F1C80106969F93F6
:1081D0008F9389E793E29F938F9389819A818C0D86
:1081E0009D1D9F938F930F945A56F6010190002086
:1081F000E9F73197EC19FD09D701ED93FC930F9046
:108200000F900F900F900F900F900F900F90DF91A5
:10821000CF911F910F91FF90EF90DF90CF90089535
:10822000BF92CF92DF92EF92FF920F931F93CF9363
:10823000DF931F921F92CDB7DEB7009709F482C07B
:108240006115710509F47EC06B018C0119821A82D7
:10825000DB011D921C92AE014F5F5F4FBC018DEEA2
:1082600092E16DDE882309F46DC0ECE5F3E58785C6
:108270008F9386858F9385858F9384858F9386ECE6
:108280009AE29F938F9389819A81800F911F9F9388
:108290008F930F945A56F80101900020E9F7319717
:1082A000E01BF10BE983FA83CDBFDEBFB12C0F2EAB
:1082B000FEE7EF2EF3E2FF2EF02D2DC0EB2DF0E0C8
:1082C000EE0FFF1FEE0FFF1FE45AFC4ADF015A9624
:1082D00013968C9113978F9312968C9112978F937C
:1082E00011968C918F93828D8F93FF92EF9289815B
:1082F0009A81800F911F9F938F930F945A56F80184
:1083000001900020E9F73197E01BF10BE983FA8334
:10831000B394CDBFDEBF0F941A1CB81678F2E98172
:10832000FA81E00FF11F8DE09AE080839183128241
:10833000F80101900020E9F73197E01BF10BD6011D
:10834000ED93FC930F900F90DF91CF911F910F91C0
:10835000FF90EF90DF90CF90BF900895BF92CF92A3
:10836000DF92EF92FF920F931F93CF93DF9300D092
:108370001F92CDB7DEB719821A821B821C8200972A
:1083800009F4CDC06115710509F4C9C0022FB42EDE
:108390006B017C011FEF120F123108F0B5C0AE0166
:1083A0004F5F5F4FBC0185E093E1C9DD882309F48D
:1083B000B6C01A3079F5BB2069F069817A816E0DFB
:1083C0007F1DAE014D5F5F4F86E999E0F5DD8111BC
:1083D0000EC0A5C069817A816E0D7F1DAE014D5F13
:1083E0005F4F82E799E0E8DD882309F498C069814E
:1083F0007A818B819C81680F791F69837A836E0DE6
:108400007F1DAE014D5F5F4F88EF9AE098DD8111CF
:1084100071C085C084EF800F873008F046C0BB2054
:1084200089F069817A816E0D7F1D812F90E0880F20
:10843000991FAE014D5F5F4F8C57964FBDDD811187
:1084400012C06DC069817A816E0D7F1D812F90E011
:10845000880F991FAE014D5F5F4F805A964FACDD7C
:10846000882309F45CC069817A818B819C81680FC3
:10847000791F69837A8322EF200F223058F46E0D22
:108480007F1DAE014D5F5F4F84E799E095DD81115F
:1084900031C045C06E0D7F1DAE014D5F5F4F83EE55
:1084A0009AE04DDD811126C03AC0BB2091F0698170
:1084B0007A816E0D7F1D212F30E0C901880F991F31
:1084C000AE014D5F5F4F8C57964F76DD811112C024
:1084D00026C069817A816E0D7F1D212F30E0C90190
:1084E000880F991FAE014D5F5F4F805A964F64DD34
:1084F0008823A9F029813A818B819C81820F931F67
:10850000F601808391830BC0AE014F5F5F4FBC01CA
:1085100085E093E114DD882311F010E0C6CF2496A6
:10852000CDBFDEBFDF91CF911F910F91FF90EF90F4
:10853000DF90CF90BF90089589E10E9458C181E0FB
:10854000623009F080E00895CF92DF92EF92FF92BF
:108550001F93CF93DF9300D01F92CDB7DEB7198260
:108560001A821B821C82009709F453C061157105A1
:1085700009F44FC0142F6B017C01AE014F5F5F4FB8
:10858000BC0185E093E1DBDC882309F442C01730AD
:1085900089F01930E1F0113039F569817A816E0D79
:1085A0007F1DAE014D5F5F4F82E89AE0C8DC81110C
:1085B00027C02FC069817A816E0D7F1DAE014D5F8E
:1085C0005F4F81E29AE0BBDC81111AC022C0698151
:1085D0007A816E0D7F1DAE014D5F5F4F80EC99E09B
:1085E000AEDC81110DC015C069817A816E0D7F1DD1
:1085F000AE014D5F5F4F82E89AE0A1DC882349F02D
:1086000029813A818B819C81820F931FF60180839F
:1086100091832496CDBFDEBFDF91CF911F91FF9054
:10862000EF90DF90CF900895EF92FF920F931F93FA
:10863000CF93DF931F921F92CDB7DEB719821A82B4
:10864000009751F16115710539F17B018C0187E1CA
:108650000E9458C1662351F0AE014F5F5F4FB801D1
:108660008EE893E16CDC81110AC016C0AE014F5F49
:108670005F4FB80181E193E162DC882369F0898171
:108680009A81F801E80FF91F2DE020832AE0218369
:108690000296F701808391830F900F90DF91CF9125
:1086A0001F910F91FF90EF900895EF92FF920F931B
:1086B0001F93CF93DF931F921F92CDB7DEB7009722
:1086C00009F47EC04115510509F47CC0F22E8A01DF
:1086D000E62EAE014F5F5F4FB8016EDC811102C024
:1086E00019821A8283E0E81629F18E1538F091E09C
:1086F000E91659F082E0E81699F03AC094E0E916DC
:1087000019F185E0E81651F133C0E1EBF6E4019090
:108710000020E9F73197E15BF64461EB76E42BC08A
:10872000E8ECF6E401900020E9F7E95CF64468EC37
:1087300076E421C0EFEDF6E401900020E9F7E05E79
:10874000F6446FED76E417C0E6EFF6E40190002002
:10875000E9F7E75FF64466EF76E40DC0EDE0F7E495
:1087600001900020E9F7EE50F7446DE077E403C094
:1087700061EB76E4E0E0EF3008F0EEE0CB018E0F45
:10878000911DFC01108289819A81800F911F0F94A5
:108790003C56F80101900020E9F73197E01BF10BFE
:1087A000FF2091F0C8018E0F911DFC018CE29DE02D
:1087B000808391838AE090E08283938381E005C087
:1087C00080E003C080E001C081E00F900F90DF9156
:1087D000CF911F910F91FF90EF9008958F929F92EC
:1087E000AF92BF92CF92DF92EF92FF920F931F93BF
:1087F000CF93DF931F921F92CDB7DEB73091BE3E6D
:10880000311104C0FB011082118236C00097A1F122
:10881000672B91F14115510579F1022F4A016C0145
:108820000F2EFCEDEF2EF9E1FF2EF02D11E0202FA1
:10883000A601612FC70139DF8823A9F0F601019055
:108840000020E9F731975F01AC18BD089E012F5F4A
:108850003F4FA501B601C4010F94514A89819A8105
:10886000A816B90631F41F5FF2E0EF0EF11C1630C6
:10887000F1F6C4010F94FF4B0F900F90DF91CF9151
:108880001F910F91FF90EF90DF90CF90BF90AF902E
:108890009F908F9008958F929F92AF92BF92DF9298
:1088A000EF92FF920F931F93CF93DF93CDB7DEB775
:1088B0002597CDBFDEBF009709F497C44115510538
:1088C00009F495C4D22E7A01162FAE014F5F5F4F87
:1088D000B70172DB811102C019821A82163109F0C8
:1088E0006DC00E9472F54B015C01672B682B692BF0
:1088F000E1F486E10E9458C120E13EE040E050E012
:108900000F9411545F934F933F932F9389E893E211
:108910009F938F9389819A818E0D9F1D9F938F9333
:108920000F945A56CDBFDEBF49C486E10E9458C19C
:10893000992324F586E10E9458C120E13EE040E001
:1089400050E00F941154CA01B9010F948926BF92C7
:10895000AF929F928F929F938F937F936F9384E8B0
:1089600093E29F938F9389819A818E0D9F1D9F9390
:108970008F930F945A56CDBFDEBF20C486E10E946C
:1089800058C1BF92AF929F928F9220E13EE040E0AB
:1089900050E00F9411545F934F933F932F9385E8CA
:1089A00093E29F938F9389819A818E0D9F1D9F9350
:1089B0008F930F945A56CDBFDEBF00C4123060F4BF
:1089C000812F0E94BDC129813A81BC01C701820F5C
:1089D000931F0F943C56F2C3163081F486E00E9438
:1089E00058C18B019C0189819A814BE0BE016B5F6C
:1089F0007F4F8E0D9F1D0F94E226E0C3153081F44A
:108A000085E00E9458C18B019C0189819A814BE0CD
:108A1000BE016B5F7F4F8E0D9F1D0F942E28CEC31E
:108A2000123009F06EC082E00E9458C163317105B6
:108A30008105910524F061E070E080E090E0013074
:108A400009F049C029813A812E0D3F1DDC01CB017F
:108A50000197A109B109880F991FAE014D5F5F4FC2
:108A6000B9018D5A974FA8DA8130F9F4F7010190D6
:108A70000020E9F73197EE19FF09E983FA8382E0D4
:108A80000E9458C19F938F937F936F938EE893E2D8
:108A90009F938F9389819A818E0D9F1D9F938F93B2
:108AA0000F945A56CDBFDEBF89C382E00E9458C1E1
:108AB0009F938F937F936F938FE893E29F938F930E
:108AC00089819A818E0D9F1D9F938F930F945A5683
:108AD000CDBFDEBF73C382E00E9458C19F938F93C6
:108AE0007F936F9387EC9AE29F938F9389819A810A
:108AF0008E0D9F1D9F938F930F945A56CDBFDEBF4F
:108B00005DC31B3059F08DEE810F823038F089EE55
:108B1000810F823018F01A3109F05CC0812F0E9459
:108B200058C14B015C01011113C0BF92AF929F92DB
:108B30006F9387EC9AE29F938F9389819A818E0D30
:108B40009F1D9F938F930F945A56CDBFDEBF36C3A0
:108B5000672B682B692BF9F469817A816E0D7F1D73
:108B6000AE014D5F5F4F8FE498E0E9D9811126C3D4
:108B70001F921F921F921F9287EC9AE29F938F93EE
:108B800089819A818E0D9F1D9F938F930F945A56C2
:108B9000CDBFDEBF13C369817A816E0D7F1DAE012B
:108BA0004D5F5F4F8CE498E0CAD9811107C3BF9233
:108BB000AF929F928F9287EC9AE29F938F938981D5
:108BC0009A818E0D9F1D9F938F930F945A56CDBF00
:108BD000DEBFF4C2173009F05CC087E00E9458C1C4
:108BE0004B015C01011113C0BF92AF929F926F9332
:108BF00087EC9AE29F938F9389819A818E0D9F1DB6
:108C00009F938F930F945A56CDBFDEBFD7C2672B69
:108C1000682B692BF9F469817A816E0D7F1DAE0195
:108C20004D5F5F4F88E498E08AD98111C7C21F92D7
:108C30001F921F921F9287EC9AE29F938F938981D4
:108C40009A818E0D9F1D9F938F930F945A56CDBF7F
:108C5000DEBFB4C269817A816E0D7F1DAE014D5FAA
:108C60005F4F84E498E06BD98111A8C2BF92AF92A4
:108C70009F928F9287EC9AE29F938F9389819A813A
:108C80008E0D9F1D9F938F930F945A56CDBFDEBFBD
:108C900095C2143009F05CC084E00E9458C14B01B9
:108CA0005C01011113C0BF92AF929F926F9387EC4A
:108CB0009AE29F938F9389819A818E0D9F1D9F9336
:108CC0008F930F945A56CDBFDEBF78C2672B682BA7
:108CD000692BF9F469817A816E0D7F1DAE014D5FBC
:108CE0005F4F8DE398E02BD9811168C21F921F92CC
:108CF0001F921F9287EC9AE29F938F9389819A81AA
:108D00008E0D9F1D9F938F930F945A56CDBFDEBF3C
:108D100055C269817A816E0D7F1DAE014D5F5F4F37
:108D200084E398E00CD9811149C2BF92AF929F921F
:108D30008F9287EC9AE29F938F9389819A818E0D0F
:108D40009F1D9F938F930F945A56CDBFDEBF36C29F
:108D5000133009F0ABC083E00E9458C14B015C01A5
:108D6000011113C0BF92AF929F926F9387EC9AE26A
:108D70009F938F9389819A818E0D9F1D9F938F93CF
:108D80000F945A56CDBFDEBF19C291E089169104E7
:108D9000A104B10461F182E088169104A104B10438
:108DA00009F445C081149104A104B10409F05FC025
:108DB00069817A816E0D7F1DAE014D5F5F4F88E244
:108DC00098E0BDD88111FAC11F921F921F921F9285
:108DD00087EC9AE29F938F9389819A818E0D9F1DD4
:108DE0009F938F930F945A56CDBFDEBFE7C1698121
:108DF0007A816E0D7F1DAE014D5F5F4F8FE198E070
:108E00009ED88111DBC11F921F921F9281E08F9328
:108E100087EC9AE29F938F9389819A818E0D9F1D93
:108E20009F938F930F945A56CDBFDEBFC7C1698100
:108E30007A816E0D7F1DAE014D5F5F4F8AE198E034
:108E40007ED88111BBC11F921F921F9282E08F9327
:108E500087EC9AE29F938F9389819A818E0D9F1D53
:108E60009F938F930F945A56CDBFDEBFA7C16981E0
:108E70007A816E0D7F1DAE014D5F5F4F88E298E0F5
:108E80005ED881119BC1BF92AF929F928F9287EC67
:108E90009AE29F938F9389819A818E0D9F1D9F9354
:108EA0008F930F945A56CDBFDEBF88C1193109F098
:108EB000AEC089E10E9458C14B015C01011113C091
:108EC000BF92AF929F926F9387EC9AE29F938F939A
:108ED00089819A818E0D9F1D9F938F930F945A566F
:108EE000CDBFDEBF6BC191E089169104A104B1042E
:108EF00061F182E088169104A104B10409F446C02E
:108F000081149104A104B10409F061C069817A81DE
:108F10006E0D7F1DAE014D5F5F4F86E198E00FD86B
:108F200081114CC11F921F921F921F9287EC9AE2EF
:108F30009F938F9389819A818E0D9F1D9F938F930D
:108F40000F945A56CDBFDEBF39C169817A816E0D4B
:108F50007F1DAE014D5F5F4F80E198E00E949F3F13
:108F600081112CC11F921F921F9281E08F9387EC79
:108F70009AE29F938F9389819A818E0D9F1D9F9373
:108F80008F930F945A56CDBFDEBF18C169817A8185
:108F90006E0D7F1DAE014D5F5F4F88E098E00E942F
:108FA0009F3F81110BC11F921F921F9282E08F93EE
:108FB00087EC9AE29F938F9389819A818E0D9F1DF2
:108FC0009F938F930F945A56CDBFDEBFF7C0698130
:108FD0007A816E0D7F1DAE014D5F5F4F86E198E097
:108FE0000E949F3F8111EAC0BF92AF929F928F92E1
:108FF00087EC9AE29F938F9389819A818E0D9F1DB2
:109000009F938F930F945A56CDBFDEBFD7C01231B6
:1090100009F05EC082E10E9458C14B015C01011160
:1090200013C0BF92AF929F926F9387EC9AE29F9387
:109030008F9389819A818E0D9F1D9F938F930F949B
:109040005A56CDBFDEBFBAC0672B682B692B01F51E
:1090500069817A816E0D7F1DAE014D5F5F4F87EF95
:1090600097E00E949F3F8111A9C01F921F921F92FB
:109070001F9287EC9AE29F938F9389819A818E0D3C
:109080009F1D9F938F930F945A56CDBFDEBF96C0FE
:1090900069817A816E0D7F1DAE014D5F5F4F8FEE4E
:1090A00097E00E949F3F811189C0BF92AF929F922B
:1090B0008F9287EC9AE29F938F9389819A818E0D8C
:1090C0009F1D9F938F930F945A56CDBFDEBF76C0DE
:1090D000153109F05EC085E10E9458C14B015C0169
:1090E000011113C0BF92AF929F926F9387EC9AE2E7
:1090F0009F938F9389819A818E0D9F1D9F938F934C
:109100000F945A56CDBFDEBF59C0672B682B692B11
:1091100001F569817A816E0D7F1DAE014D5F5F4F54
:1091200083E098E00E949F3F811148C01F921F92E8
:109130001F921F9287EC9AE29F938F9389819A8165
:109140008E0D9F1D9F938F930F945A56CDBFDEBFF8
:1091500035C069817A816E0D7F1DAE014D5F5F4F15
:109160008EEF97E00E949F3F811128C0BF92AF927F
:109170009F928F9287EC9AE29F938F9389819A8135
:109180008E0D9F1D9F938F930F945A56CDBFDEBFB8
:1091900015C0812F0E9458C19F938F937F936F9327
:1091A00087EC9AE29F938F9389819A818E0D9F1D00
:1091B0009F938F930F945A56CDBFDEBFF701019056
:1091C0000020E9F73197EE19FF09DD2091F0C70182
:1091D0008E0F911DFC018CE29DE0808391838AE0DB
:1091E00090E08283938381E005C080E003C080E04B
:1091F00001C081E02596CDBFDEBFDF91CF911F91E9
:109200000F91FF90EF90DF90BF90AF909F908F9065
:1092100008956F927F928F929F92AF92BF92CF925A
:10922000DF92EF92FF920F931F93CF93DF931F92E2
:109230001F92CDB7DEB70097B1F1672BA1F14115B1
:10924000510589F1802E922E3A016C010F2EFBE818
:10925000EF2EFBE1FF2EF02D10E0082D292DA601A9
:10926000612FC70118DB8823A9F0F60101900020C7
:10927000E9F731975F01AC18BD089E012F5F3F4FA2
:10928000A501B601C3010F94514A89819A81A8169C
:10929000B90631F41F5F82E0E80EF11C1C31E9F6DB
:1092A000C3010F94FF4B0F900F90DF91CF911F914F
:1092B0000F91FF90EF90DF90CF90BF90AF909F9075
:1092C0008F907F906F9008958F929F92AF92BF92F0
:1092D000DF92EF92FF920F931F93CF93DF931F9232
:1092E0001F92CDB7DEB7009709F48FC061157105E5
:1092F00009F48BC04B017C010E9443C69F938F935E
:1093000085E993E29F938F93FF92EF920F945A56C1
:10931000F70101900020E9F73197AF014E195F097D
:109320004231510510F041E150E09E012F5F3F4F67
:10933000B701C4010F94514A0F900F900F900F90F6
:109340000F900F90D12C0F2EF3ECAF2EF9E2BF2E21
:10935000F02D8D2D0E9434C19F938F937F936F9337
:10936000BF92AF92FF92EF920F945A56F70101907D
:109370000020E9F731978F010E191F099E012F5F19
:109380003F4FA801B701C4010F94514ACDBFDEBFC2
:1093900089819A810817190731F4D39496E1D9127B
:1093A000D8CF11E001C011E00F2EF5E9AF2EF3E2A6
:1093B000BF2EF02D812F0E94A4C99F938F93BF923F
:1093C000AF92FF92EF920F945A56F701019000204E
:1093D000E9F73197AF014E195F094231510510F09D
:1093E00041E150E09E012F5F3F4FB701C4010F9450
:1093F000514A1F5F0F900F900F900F900F900F909A
:109400001330C1F6C4010F94FF4B0F900F90DF9102
:10941000CF911F910F91FF90EF90DF90BF90AF9091
:109420009F908F9008952F923F924F925F926F92EC
:109430007F928F929F92AF92BF92CF92DF92EF92E4
:10944000FF920F931F93CF93DF93CDB7DEB7E197D2
:10945000CDBFDEBF91E09BA76115710509F4B7C3CD
:109460004115510509F4B5C38A017B0189AB0F94FD
:10947000D21B29A9213089F4A8016CEF72E3CE0137
:109480000B960E94C354182F86E08BA70F94A00858
:109490006DA77EA78FA798AB1AC0A8016CEF72E3E7
:1094A000CE010B960E943855182F0F94A0086DA777
:1094B0007EA78FA798AB82E00F941907862FAE0185
:1094C000445D5F4FBE01655D7F4F0E9466221123A0
:1094D00009F481C341E0BE01675F7F4FC7010E946D
:1094E000054049855A85CA01A0E0B0E089839A8386
:1094F000AB83BC839E01275F3F4FB701CE010B9624
:109500000F94514ACE010B960F94FF4BBE01655F3D
:109510007F4FC701D9DE0DE0D7010C931AE01196F9
:109520001C939E01275F3F4F42E050E0B701CE0100
:109530000B960F94514ACE010B960F94FF4BECEF14
:10954000F2E3018B128B9E01275F3F4F43E150E016
:10955000BF01CE010B960F94514ACE010B960F948A
:10956000FF4BB9A9B1113DC30F94F5080F94DE0864
:1095700038C301E021E0A701612FC6018CD98823FF
:1095800081F0F70101900020E9F73197AF014E1902
:109590005F099E01275F3F4FB701CE010B960F94E5
:1095A000514AE2E0CE0ED11C1F5F133011F70F2E8F
:1095B000FDE9CF2EFBE1DF2EF02D19E001E021E0E7
:1095C000A701612FC60167D9882381F0F7010190B7
:1095D0000020E9F73197AF014E195F099E01275F1F
:1095E0003F4FB701CE010B960F94514AF2E0CF0ED8
:1095F000D11C1F5F1B3011F70F2EF2E18F2E912C23
:10960000A12CB12CF02D28E182169104A104B10403
:1096100051F401E021E0A70169E18DEB9BE13BD929
:1096200081110EC030C001E021E0A701682DC40106
:10963000880F991F8557944E2ED98823C1F007C0F3
:109640000F2EF9E18F2E912CA12CB12CF02DF701CA
:1096500001900020E9F73197AF014E195F099E0193
:10966000275F3F4FB701CE010B960F94514A33E06D
:10967000830E911CA11CB11C4AE184169104A10423
:10968000B10408F4C0CFCE010B960F94FF4B89E0D4
:109690000E9458C16F31710581059105C0F4DC014C
:1096A000CB01072E7CE0880F991FAA1FBB1F7A955C
:1096B000D1F7702D89839A83AB83BC8380E090E1DE
:1096C000A0E0B0E08D839E83AF83B88717C0DC0134
:1096D000CB01072E79E0880F991FAA1FBB1F7A952F
:1096E000D1F7702D89839A83AB83BC8380E092E0AD
:1096F000A0E0B0E08D839E83AF83B88789819A8193
:10970000AB81BC812DA53EA54FA558A928173907C7
:109710004A075B07A1F1AE01475F5F4FB70184EBDA
:1097200099E00E949F3F813081F4F7010190002071
:10973000E9F73197AF014E195F099E01275F3F4F4F
:10974000B701CE010B960F94514ACE010B960F94A0
:10975000FF4BCE010B960F94464C39A931113DC2F7
:109760000F946C098FE69CE30E94F12281110F9403
:109770003B198FE69CE30E943E2A80E03AC2AE018C
:10978000475F5F4FB70188EA99E00E949F3F8130B1
:1097900081F4F70101900020E9F73197AF014E19EC
:1097A0005F099E01275F3F4FB701CE010B960F94D3
:1097B000514A48A94F935FA55F938EA58F939DA5AE
:1097C0009F9388858F938F818F938E818F938D81C7
:1097D0008F9389E993E29F938F93FF92EF920F9477
:1097E0005A56F70101900020E9F73197AF014E1961
:1097F0005F099E01275F3F4FB701CE010B960F9483
:10980000514A88E290E089879A8768E2C7010E94FE
:109810001AAA482F50E060E070E049835A836B83B6
:109820007C83682F70E0C7010F947228CDBFDEBF24
:109830008823C9F049815A819E01275F3F4FB701B4
:10984000CE010B960F94514A8DE0F70180838AE098
:1098500081839E01275F3F4F42E050E0B701CE0178
:109860000B960F94514ABE016F5F7F4FC7010E9454
:10987000144349815A819E01275F3F4FB701CE01B2
:109880000B960F94514A6BE370E0C7010E946DA9DB
:10989000A0E0B0E089839A83AB83BC830E94A62AB0
:1098A00081110EC0F70101900020E9F73197AF0157
:1098B0004E195F0920E0B70182E299E30F940C2171
:1098C00049815A816B817C81411551056105710582
:1098D000C1F09E01275F3F4FB701CE010B960F9459
:1098E000514A8DE0D7018C938AE011968C939E01AA
:1098F000275F3F4F42E050E0B701CE010B960F9437
:10990000514ACE010B960F94FF4B0E945759198272
:109910001A821B821C822DA53EA54FA558A9232B78
:10992000242B252B09F433C180E090E0DC010F2EBD
:10993000F2ED2F2EF3E23F2EF02D0F2EF4EA8F2EB4
:10994000F3E29F2EF02D880F991FAA1FBB1FBC01A9
:10995000CD017E5F8F4F9F4F0E945F590E94EA5B4F
:109960008111FCCF80E091E0EBEFF2E4DF019C019C
:109970001D9221503040E1F76F010F2EFBEFAF2E0B
:10998000F3E4BF2EF02D8F010E942EA9D8018D93F4
:109990009D938D01AA16BB06B9F70E942A5A0F940F
:1099A000392ACE010B960F94FF4B412C512C3201DA
:1099B000F601619171916F01AE014B5F5F4F8BA515
:1099C0000E945015882309F496C088858F938F8153
:1099D0008F938E818F938D818F9389819A81AB81B3
:1099E000BC81840D951DA61DB71DBF93AF939F939A
:1099F0008F939F928F92FF92EF920F945A56F70196
:109A000001900020E9F73197AF014E195F099E01DF
:109A1000275F3F4FB701CE010B960F94514A182F85
:109A2000CDBFDEBF882309F48CC00E94A62A811115
:109A300026C089819A81AB81BC81840D951DA61DAC
:109A4000B71DBF93AF939F938F931F921F934EEABF
:109A500053E25F934F93FF92EF920F945A56F701A0
:109A600001900020E9F73197AF014E195F0920E01E
:109A7000B70182E299E30F940C21CDBFDEBFF7015D
:109A800001900020E9F73197AF014E195F099E015F
:109A9000275F3F4FB701CE010B960F94514A182F05
:109AA0000E94A62A81114DC089819A81AB81BC8117
:109AB000840D951DA61DB71DBF93AF939F938F93E4
:109AC0001F921F93EFEBF3E2FF93EF93FF92EF925E
:109AD0000F945A56F70101900020E9F73197AF0132
:109AE0004E195F0920E0B70182E299E30F940C213F
:109AF000CDBFDEBF26C00E94A62A811122C0898167
:109B00009A81AB81BC81840D951DA61DB71DBF93A5
:109B1000AF939F938F933F922F92FF92EF920F9468
:109B20005A56F70101900020E9F73197AF014E191D
:109B30005F0920E0B70182E299E30F940C21CDBFC9
:109B4000DEBF9FEF491A590A690A790AA0E84A1646
:109B500051046104710409F02BCFCE010B960F94D0
:109B6000FF4B89819A81AB81BC8180589F4FAF4F59
:109B7000BF4F89839A83AB83BC832DA53EA54FA598
:109B800058A982179307A407B50708F4DCCECE01C5
:109B90000B960F94FF4BCE010B960F94464C1092F0
:109BA0000D338CEF92E30E94175639A9311117C07B
:109BB0000F946C098FE69CE30E94F12281110F94AF
:109BC0003B198FE69CE30E943E2A81E012C080E0B0
:109BD00010C080E00EC080E00CC080E00AC081E0D0
:109BE00008C00F2EFBE8CF2EFBE1DF2EF02D10E09A
:109BF000C0CCE196CDBFDEBFDF91CF911F910F9119
:109C0000FF90EF90DF90CF90BF90AF909F908F909C
:109C10007F906F905F904F903F902F900895CF92DC
:109C2000DF92EF92FF920F931F93CF93DF931F92D8
:109C30001F92CDB7DEB7009709F457C061157105C3
:109C400009F453C07B018C01AE014F5F5F4FBC0133
:109C500080E594E10E949F3F882309F446C08981F2
:109C60009A816C012FEFC21AD20AF801E80FF91F8E
:109C700020E22083B8016C0D7D1DAE014F5F5F4F68
:109C800089E394E10E949F3F882379F189819A8139
:109C9000C80ED91EF801EC0DFD1D8DE0808382E019
:109CA000C80ED11C8AE08183B8016C0D7D1DAE0108
:109CB0004F5F5F4F8BE094E10E949F3F8823A9F0A4
:109CC00089819A81C80ED91EF801EC0DFD1D8DE029
:109CD000808322E0C20ED11C8AE08183F801EC0D62
:109CE000FD1D1082F701C082D1820F900F90DF918D
:109CF000CF911F910F91FF90EF90DF90CF9008953B
:109D0000EF92FF920F931F93CF93DF93CDB7DEB700
:109D1000A297CDBFDEBF009709F451C06115710550
:109D200009F44FC07B018C0160E0CE01039615D78A
:109D3000882309F44BC0B701C80171DFF7014081E6
:109D400051819E012F5F3F4FB801CE0103960F94C2
:109D5000514ACE0103960F94FF4BF70120813181C8
:109D600089819A812817390771F5BE016D5F7F4F90
:109D7000C801AADAA701B80183EC9BE10E949F3FCA
:109D8000813099F4F701408151819E012F5F3F4F4F
:109D9000B801CE0103960F94514AF7012081318119
:109DA00089819A812817390781F4CE0103960F948F
:109DB000464C81E012D70F94D21B81E007C080E0AF
:109DC00005C080E003C080E001C080E0A296CDBF66
:109DD000DEBFDF91CF911F910F91FF90EF9008951B
:109DE0000F931F93CF93DF931F921F92CDB7DEB7D0
:109DF0000F94D21B8091B13E823009F462C028F4E6
:109E0000882359F0813081F1D6C0843009F485C0AF
:109E100008F464C08A30E1F0CEC060E084EF9FE3D4
:109E20007FD5811107C06091B23E8FE69CE30E940E
:109E30003C14C9C00F943201811104C081E08093A9
:109E4000B13EC1C08AE08093B13E0F94E319BBC01C
:109E50000F94FA196C3D75408105910508F4B3C063
:109E600081E08093B13EAFC040E063EA7CE385EAE5
:109E70009CE30E9405400FE61CE3F80144A955A9A4
:109E80009E012F5F3F4F65EA7CE384EF9FE30F94D1
:109E9000514A84EF9FE30F94FF4BF80124A935A9A1
:109EA00089819A812817390741F01092B13E60915B
:109EB000B23EC8010E943C1486C082E08093B13E4D
:109EC00082C000E021E044EF5FE363EA7CE385EADF
:109ED0009CE39FD983E08093B13E75C043EA5CE385
:109EE00065EA7CE383EC9BE10E949F3F813069F44B
:109EF0004091A33C5091A43C9E012F5F3F4F65EAE7
:109F00007CE384EF9FE30F94514A84EF9FE30F9427
:109F1000464C84E08093B13E56C00E9437D38823DC
:109F200081F10F942D1B8823C9F00E941E208823E5
:109F300009F449C08FE69CE30E94F12281110F943D
:109F40003B198FE69CE30E943E2A1092B13E60913D
:109F5000B23E8FE69CE30E943C1435C08FE69CE342
:109F60000E94F12281110F943B198FE69CE30E941D
:109F70003E2A1092B13E61E08FE69CE30E943C14C1
:109F800022C00F947519672B682B692BE1F48FE6BB
:109F90009CE30E94F12281110F943B198FE69CE310
:109FA0000E943E2A1092B13E6091B23E8FE69CE341
:109FB0000E943C1408C01092B13E6091B23E8FE600
:109FC0009CE30E943C140F900F90DF91CF911F9162
:109FD0000F9108959F92AF92BF92CF92DF92EF922E
:109FE000FF920F931F93CF93DF9300D0CDB7DEB7CF
:109FF000009709F471C06115710509F46DC0A42EB4
:10A000006B017C018EE0EDEDF3E2D70101900D9242
:10A010008A95E1F7F70101900020E9F73197EE19F1
:10A02000FF09E983AF0155279E012E5F3F4FB7011E
:10A03000C6010F94514AB12C0F2EFCE29F2EF02D39
:10A040008B2D0E94B3C88B019C0148E0BE016F5F5D
:10A050007F4FC7010F94902882E08B1550F08981C3
:10A06000F701E80FF11D90828F5FF701E80FF11DF6
:10A070001082F70101900020E9F73197EE19FF09EE
:10A08000E983AF0155279E012E5F3F4FB701C601FF
:10A090000F94514A898190E02A813B81821793076E
:10A0A00021F4B394E4E0BE12CBCFAA2081F08DE07E
:10A0B000F70180838AE0818382E089839E012E5F9D
:10A0C0003F4F42E050E0B701C6010F94514AC6012C
:10A0D0000F94FF4B0F94D21B2396CDBFDEBFDF91B1
:10A0E000CF911F910F91FF90EF90DF90CF90BF9095
:10A0F000AF909F9008959F92AF92BF92CF92DF92C0
:10A10000EF92FF920F931F93CF93DF931F921F92B3
:10A11000CDB7DEB7009709F4E1C06115710509F408
:10A12000DFC04115510509F4DDC0902E122F5A01F0
:10A130006B017C010F94D21B41E0B601C7010E9464
:10A140000540F601408151819E012F5F3F4FB701CD
:10A15000C5010F94514AC5010F94FF4BF6012081B0
:10A16000318189819A812817390709F0BDC08DE0B6
:10A17000EBEEF3E2D70101900D928A95E1F7F7013A
:10A1800001900020E9F73197AF014E195F0955277B
:10A190009E012F5F3F4FB701C5010F94514AC50182
:10A1A0000F94FF4BB501C7018FD88DE0F701808375
:10A1B0008AE081839E012F5F3F4F42E050E0B7016C
:10A1C000C5010F94514AC5010F94FF4B41E0B50101
:10A1D000C70100DFA601B7018FE69CE30E94C440DF
:10A1E000F601408151819E012F5F3F4FB701C501AC
:10A1F0000F94514AC5010F94FF4BF6012081318124
:10A2000089819A812817390709F070C0B601C70102
:10A210000E941041F601408151819E012F5F3F4F06
:10A22000B701C5010F94514AC5010F94FF4BF601C8
:10A230002081318189819A812817390709F058C016
:10A2400001E021E0A501B601C7010E94094921E012
:10A25000A501B601C7010E94EE430E949C428823DB
:10A2600031F0492DB601C7010E94A44206C0292D34
:10A27000412FB601C7010E94AE41F60140815181D4
:10A280009E012F5F3F4FB701C5010F94514AC50191
:10A290000F94FF4BF6012081318189819A81281723
:10A2A000390741F5B601C7010E941443F601408108
:10A2B00051819E012F5F3F4FB701C5010F94514A55
:10A2C000C5010F94FF4B81E0F60140815181298146
:10A2D0003A814217530779F080E00DC080E00BC04F
:10A2E00080E009C080E007C080E005C080E003C0D6
:10A2F00080E001C080E00F900F90DF91CF911F911F
:10A300000F91FF90EF90DF90CF90BF90AF909F9014
:10A3100008952F923F924F925F926F927F928F9209
:10A320009F92AF92BF92CF92DF92EF92FF920F93E4
:10A330001F93CF93DF93CDB7DEB7A897CDBFDEBF16
:10A340004115510509F4D7C12115310509F4D5C1CD
:10A350006115710509F4D3C1280169011A017B0156
:10A3600088A70F94D21BA6016CEF72E3CE0107966B
:10A37000A7D6882309F4C5C141E0BE016B5F7F4FBA
:10A38000C1010E9405404D815E819E012B5F3F4FC0
:10A39000B101CE0107960F94514ACE0107960F9452
:10A3A000FF4BBE01695F7F4FC1010E9464491DE000
:10A3B000F10110830AE001839E012B5F3F4F42E0D1
:10A3C00050E0B101CE0107960F94514ACE01079695
:10A3D0000F94FF4BECEFF2E3118B028B9E012B5F8E
:10A3E0003F4F43E150E0BF01CE0107960F94514A21
:10A3F000CE0107960F94FF4B0F2EFBE8CF2EFBE10B
:10A40000DF2EF02D10E001E021E0A101612FC60157
:10A410000E944B44882381F0F10101900020E9F76C
:10A420003197AF01421953099E012B5F3F4FB10194
:10A43000CE0107960F94514AF2E0CF0ED11C1F5F58
:10A44000133009F70F2EFDE9CF2EFBE1DF2EF02DA3
:10A4500019E001E021E0A101612FC6010E944B44F7
:10A46000882381F0F10101900020E9F73197AF01D5
:10A47000421953099E012B5F3F4FB101CE01079650
:10A480000F94514A22E0C20ED11C1F5F1B3009F706
:10A490000F2EF2E18F2E912CA12CB12CF02D88E102
:10A4A00088169104A104B10491F401E021E0A10116
:10A4B00069E18DEB9BE10E944B44811116C00F2E88
:10A4C000FCE18F2E912CA12CB12CF02D31C001E09C
:10A4D00021E0A101682DC401880F991F8557944E72
:10A4E0000E944B448823C1F007C00F2EF9E18F2E44
:10A4F000912CA12CB12CF02DF10101900020E9F755
:10A500003197AF01421953099E012B5F3F4FB101B3
:10A51000CE0107960F94514A93E0890E911CA11C1D
:10A52000B11CEAE18E169104A104B10408F4B7CF7E
:10A530001F92F8A5FF9388EF93E29F938F933F922A
:10A540002F920F945A56F10101900020E9F73197AC
:10A55000AF01421953099E012B5F3F4FB101CE015C
:10A5600007960F94514ACE0107960F94FF4B612C2A
:10A57000712C0F900F900F900F900F900F9041142F
:10A5800051046104710409F4A7C0870175016401D5
:10A59000812C912C5401F80141915191619171915B
:10A5A0008F019E012F5F3F4F88A50E94282F88238F
:10A5B00009F482C08C818F938B818F938A818F93D2
:10A5C00089818F93BF92AF929F928F9284EA93E298
:10A5D0009F938F933F922F920F945A56F1010190BF
:10A5E0000020E9F73197AF01421953099E012B5F13
:10A5F0003F4FB101CE0107960F94514A8FA3CDBFB3
:10A60000DEBF9FA1992309F457C00E94A62A811199
:10A610001FC0FF92EF92DF92CF921F92EFA1EF93B4
:10A620008EEA93E29F938F933F922F920F945A5604
:10A63000F10101900020E9F73197AF014219530968
:10A6400020E0B10182E299E30F940C21CDBFDEBF7F
:10A65000F10101900020E9F73197AF014219530948
:10A660009E012B5F3F4FB101CE0107960F94514AD7
:10A670008FA30E94A62A81111FC0FF92EF92DF9242
:10A68000CF921F929FA19F93EFEBF3E2FF93EF9383
:10A690003F922F920F945A56F10101900020E9F752
:10A6A0003197AF014219530920E0B10182E299E3E9
:10A6B0000F940C21CDBFDEBF9FEF891A990AA90A1A
:10A6C000B90AEFEFCE1ADE0AEE0AFE0A84149504E8
:10A6D000A604B70408F45FCFCE0107960F94FF4B92
:10A6E000CE0107960F94464C10920D338CEF92E3F7
:10A6F0009ED281E007C080E005C080E003C080E01A
:10A7000001C080E0A896CDBFDEBFDF91CF911F9141
:10A710000F91FF90EF90DF90CF90BF90AF909F9000
:10A720008F907F906F905F904F903F902F90089503
:10A7300008958091113308950895109211338091F6
:10A740001033882331F01092103384E190E40D949B
:10A75000464C089584E190E40D94464C0895809110
:10A7600010330895CF92DF92EF92FF921F93CF9311
:10A77000DF93CDB7DEB76897CDBFDEBF6C017B013D
:10A7800084E1E3E0F4E2DE01159601900D928A95F2
:10A79000E1F7DA01C9010196A11DB11D883E23E050
:10A7A0009207A105B1050CF460C01F921F921F9281
:10A7B00081E08F9384EE90E29F938F93CE01019678
:10A7C0009F938F930F945A568981898B8A818A8BA4
:10A7D0008B818B8B80E38D838AE38E83CDBFDEBF3D
:10A7E000E114F10459F0D701FE0138969E01245F6F
:10A7F0003F4F8D918193E217F307D9F710E346E0BD
:10A80000BE016B5F7F4F84E190E40F94B34799EFF3
:10A81000980F9230C8F48B89893399F48A898933E7
:10A8200061F48989893321F41092103380E03CC0AF
:10A830008F5F898B1A8B1B8BE2CF1B8B8F5F8A8B71
:10A84000DECF8F5F8B8BDBCF882321F0109210330C
:10A8500080E02AC081E080931033BE01695F7F4FA2
:10A86000C6010F943C5681E01FC0BF93AF939F93E6
:10A870008F9384EE90E29F938F93CE0101969F93E6
:10A880008F930F945A568981898B8A818A8B8B8109
:10A890008B8B80E38D838AE38E83CDBFDEBFE11493
:10A8A000F10409F0A0CFAACF6896CDBFDEBFDF913B
:10A8B000CF911F91FF90EF90DF90CF90089580E0AF
:10A8C0000F947901882361F08250823030F58091B5
:10A8D0001133882311F1109211331092103308951F
:10A8E00080911133811119C081E0809311338EE280
:10A8F00092E0E2E1F3E3DF019C011D922150304040
:10A90000E1F7BF0180E00F9495478B3019F4109266
:10A910001033089581E08093103308958AE00895FC
:10A92000CF93DF93CDB7DEB76097CDBFDEBF009783
:10A9300019F120E329832AE32A832BE0E7E1F4E2FB
:10A94000DE01139601900D922A95E1F7613041F4F2
:10A9500041E0BE016F5F7F4F0F94B347982F07C050
:10A960004AE0BE016F5F7F4F0F94B347982F81E09D
:10A97000992319F080E001C080E06096CDBFDEBF72
:10A98000DF91CF910895DF92EF92FF920F931F9383
:10A99000CF93DF93CDB7DEB76497CDBFDEBF8C0119
:10A9A00084E1E2E2F4E2DE01119601900D928A95D3
:10A9B000E1F70115110509F449C06115710509F4A4
:10A9C00047C080E389838AE38A834115510559F0A2
:10A9D000DA01FE0134969E01285F3F4F9D919193CD
:10A9E000E217F307D9F77B010F2EF0E3DF2EF02DEE
:10A9F00046E0BE016F5F7F4FC8010F94B34799EFE8
:10AA0000980F9230A8F49F85993379F48E85893315
:10AA100041F48D858933F1F08F5F8D87DE86DF8687
:10AA2000E7CFDF868F5F8E87E3CF9F5F9F87E0CF83
:10AA3000811112C081E1FE013396D70101900D9280
:10AA40008A95E1F7F701118A81E007C080E005C02F
:10AA500080E003C080E001C080E06496CDBFDEBF2F
:10AA6000DF91CF911F910F91FF90EF90DF900895AC
:10AA7000DF92EF92FF920F931F93CF93DF93CDB7A7
:10AA8000DEB76497CDBFDEBF8C0184E1E6E3F4E27C
:10AA9000DE01119601900D928A95E1F701151105DD
:10AAA00009F449C06115710509F447C080E3898341
:10AAB0008AE38A834115510559F0DA01FE01349683
:10AAC0009E01285F3F4F9D919193E217F307D9F7BD
:10AAD0007B010F2EF0E3DF2EF02D46E0BE016F5F0D
:10AAE0007F4FC8010F94B34799EF980F9230A8F4A5
:10AAF0009F85993379F48E85893341F48D85893327
:10AB0000F1F08F5F8D87DE86DF86E7CFDF868F5F90
:10AB10008E87E3CF9F5F9F87E0CF811112C081E1D5
:10AB2000FE013396D70101900D928A95E1F7F70166
:10AB3000118A81E007C080E005C080E003C080E0AA
:10AB400001C080E06496CDBFDEBFDF91CF911F9141
:10AB50000F91FF90EF90DF9008950F931F93CF9385
:10AB6000DF93CDB7DEB76097CDBFDEBF009761F151
:10AB70008C0180E389838AE38A838BE0EAE4F4E250
:10AB8000DE01139601900D928A95E1F7613049F448
:10AB900041E0BE016F5F7F4FC8010F94B347982F0C
:10ABA0000EC041E060E0CE0103960F94234E4AE0D0
:10ABB000BE016F5F7F4FC8010F94B347982F81E0AC
:10ABC000992319F080E001C080E06096CDBFDEBF20
:10ABD000DF91CF911F910F910895CF93DF93CDB760
:10ABE000DEB76097CDBFDEBF9BE0EAE4F4E2DE01B2
:10ABF000119601900D929A95E1F7813041F441E070
:10AC000061E0CE0101960F94234E982F07C041E0DA
:10AC100060E0CE0101960F94234E982F81E09111B0
:10AC200080E06096CDBFDEBFDF91CF9108950097A1
:10AC300021F041E061E00D94234E08951F93CF93DE
:10AC4000DF93CDB7DEB76497CDBFDEBF009701F1CC
:10AC5000162FBC0180E389838AE38A83CE010396A1
:10AC60000F943C56113041F441E061E0CE01019671
:10AC70000F94234E982F07C041E060E0CE0101966B
:10AC80000F94234E982F81E0992319F080E001C0A2
:10AC900080E06496CDBFDEBFDF91CF911F91089514
:10ACA000EF92FF920F931F93CF93DF93CDB7DEB751
:10ACB0006497CDBFDEBF6115710589F1009789F1F9
:10ACC0008B017C0180E389838AE38A83CE0103962A
:10ACD0000F943C5643E0BE016F5F7F4FC7010F9456
:10ACE000B347873069F460E0C801A8DF982F882354
:10ACF000D9F043E0BE016F5F7F4FC7010F94B347A8
:10AD0000811111C0F7014285538564857585C7019E
:10AD10000F94514C91E0882339F090E005C090E009
:10AD200003C090E001C090E0892F6496CDBFDEBFE4
:10AD3000DF91CF911F910F91FF90EF900895CF93E6
:10AD4000DF93CDB7DEB76097CDBFDEBF0097C1F010
:10AD500020E329832AE32A832AE0E5E5F4E2DE0101
:10AD6000139601900D922A95E1F741E0BE016F5FC5
:10AD70007F4F0F94B34791E0882319F090E001C012
:10AD800090E0892F6096CDBFDEBFDF91CF9108950F
:10AD90003F924F925F926F927F928F929F92AF926B
:10ADA000BF92CF92DF92EF92FF920F931F93CF93B8
:10ADB000DF93CDB7DEB76197CDBFDEBF61157105FB
:10ADC00009F470C0009709F46FC04115510509F4EA
:10ADD0006DC03FEF320F383008F06AC0322E7A0172
:10ADE0008C01FB01138A41E00F94B347811162C0CB
:10ADF000F8014285538564857585483EF3E05F0719
:10AE00006105710508F458C0413B84E058076105AD
:10AE1000710508F053C0C32CD12C5601E6E0AE0EEC
:10AE2000B11C25010B2C000C660877084419550944
:10AE300066097709C8010F94514C811141C0A501E1
:10AE400060E070E0CE0103960F9435569E012F5FAF
:10AE50003F4FA501BE016D5F7F4FC8010F940549AB
:10AE6000C8010F94464CFE01EC0DFD1D12868E01AB
:10AE70000D5F1F4F812C912C5401A601B801C70111
:10AE80000F941F56892BF1F0FFEF8F1A9F0AAF0A1C
:10AE9000BF0A0F5F1F4F481459046A047B0468F708
:10AEA00080E011C080E00FC080E00DC080E00BC0EA
:10AEB00080E009C080E007C081E005C080E003C0F9
:10AEC00080E001C081E06196CDBFDEBFDF91CF9110
:10AED0001F910F91FF90EF90DF90CF90BF90AF90B8
:10AEE0009F908F907F906F905F904F903F900895CC
:10AEF0004F925F926F927F92AF92BF92CF92DF920A
:10AF0000EF92FF920F931F93CF93DF93CDB7DEB7EE
:10AF10006897CDBFDEBF680114E1E3E0F4E2DE0133
:10AF2000159601900D921A95E1F7009709F491C0DA
:10AF3000C114D10409F48FC0EFEFEE0DE83008F032
:10AF40008CC0860129013A015B016C01283E83E037
:10AF50003807410551050CF482C01F921F921F92C1
:10AF600081E08F9384EE90E29F938F93CE010196C0
:10AF70009F938F930F945A568981898B8A818A8BEC
:10AF80008B818B8B80E38D838AE38E83CDBFDEBF85
:10AF9000A114B10459F0D501FE0138969E01245F39
:10AFA0003F4F8D918193E217F307D9F70F2EF0E30E
:10AFB000FF2EF02D46E0BE016B5F7F4F84E190E4F1
:10AFC0000F94B34799EF980F923090F52E2DA8016A
:10AFD000BE016B5F7F4F84E190E4DADE882379F075
:10AFE00060E0C6012BDE882351F04AE0BE016B5FB2
:10AFF0007F4F84E190E40F94B3478823F9F09B8955
:10B00000993399F48A89893361F48989893321F4E0
:10B010001092103380E042C08F5F898BFA8AFB8ADE
:10B02000C9CFFB8A8F5F8A8BC5CF9F5F9B8BC2CFB7
:10B03000882321F01092103380E030C081E08093AB
:10B040001033BE01695F7F4FC6010F943C5681E00B
:10B0500025C080E023C080E021C080E01FC07F9237
:10B060006F925F922F9384EE90E29F938F93CE0125
:10B0700001969F938F930F945A568981898B8A8169
:10B080008A8B8B818B8B80E38D838AE38E83CDBF0C
:10B09000DEBFA114B10409F07ECF88CF6896CDBF82
:10B0A000DEBFDF91CF911F910F91FF90EF90DF9066
:10B0B000CF90BF90AF907F906F905F904F9008952A
:10B0C000DF92EF92FF920F931F93CF93DF93CDB751
:10B0D000DEB76497CDBFDEBF8C0184E1EFE5F4E21B
:10B0E000DE01119601900D928A95E1F70115110587
:10B0F00009F449C06115710509F447C080E38983EB
:10B100008AE38A834115510559F0DA01FE0134962C
:10B110009E01285F3F4F9D919193E217F307D9F766
:10B120007B010F2EF0E3DF2EF02D46E0BE016F5FB6
:10B130007F4FC8010F94B34799EF980F9230A8F44E
:10B140009F85993379F48E85893341F48D858933D0
:10B15000F1F08F5F8D87DE86DF86E7CFDF868F5F3A
:10B160008E87E3CF9F5F9F87E0CF811112C081E17F
:10B17000FE013396D70101900D928A95E1F7F70110
:10B18000118A81E007C080E005C080E003C080E054
:10B1900001C080E06496CDBFDEBFDF91CF911F91EB
:10B1A0000F91FF90EF90DF900895809140350895C2
:10B1B0000895089581E080934035089510924035B8
:10B1C0000895CF92DF92EF92FF920F931F93662321
:10B1D000B9F081111DC0C12CD12C760100E010E620
:10B1E0002AEE30E040E06CE170E280EB98E00F94F2
:10B1F0002D346CE170E280EB98E00F94773408C056
:10B20000811106C06CE170E280EB98E00F948D3400
:10B210001F910F91FF90EF90DF90CF900895CF9303
:10B22000DF931F921F92CDB7DEB780914135909189
:10B230004235A0914335B0914435072E75E1B6955E
:10B24000A795979587957A95D1F7702D61E0B9DF2D
:10B2500087ED8A8341E050E0BE016E5F7F4F80EB57
:10B2600098E00F94483441E050E0BE016F5F7F4F9B
:10B2700080EB98E00F945F3489818823A4F7809154
:10B28000413590914235A0914335B0914435072E18
:10B2900075E1B695A795979587957A95D1F7702D15
:10B2A00060E08FDF0F900F90DF91CF91089580EBDA
:10B2B00098E00F94F6331092453581E008951F937E
:10B2C000CF93DF93CDB7DEB72C97CDBFDEBF61152F
:10B2D000710520E28207910508F0A1C0DC01CB01D5
:10B2E0008093413590934235A0934335B0934435D4
:10B2F00080914535811193DF10924535809141351C
:10B3000090914235A0914335B0914435072E75E1B7
:10B31000B695A795979587957A95D1F7702D61E0A9
:10B3200050DF82ED8C8741E050E0BE01645F7F4FCB
:10B3300080EB98E00F9448348091413590914235EC
:10B34000A0914335B0914435AC01BD01032E39E0E5
:10B3500076956795579547953A95D1F7302D032EF9
:10B360003AE0440F551F661F771F3A95D1F7302DED
:10B370009170AA27BB27842B952BA62BB72B8983EB
:10B380009A83AB83BC838B818D8341E050E0BE0107
:10B390006B5F7F4F80EB98E00F9448348A818E83F7
:10B3A00041E050E0BE016A5F7F4F80EB98E00F9470
:10B3B000483489818F8341E050E0BE01695F7F4F4F
:10B3C00080EB98E00F94483415E5188741E050E091
:10B3D000BE01685F7F4F80EB98E00F944834198777
:10B3E00041E050E0BE01675F7F4F80EB98E00F9433
:10B3F00048341A8741E050E0BE01665F7F4F80EB22
:10B4000098E00F9448341B8741E050E0BE01655F2F
:10B410007F4F80EB98E00F94483481E001C080E0DA
:10B420002C96CDBFDEBFDF91CF911F910895052EE1
:10B4300059E0660F771F881F991F5A95D1F7502D35
:10B440006115710520E28207910510F438CF089547
:10B4500080E008958091413590914235A091433527
:10B46000B09144350097A105B10569F00197A10994
:10B47000B109072E75E1B695A795979587957A95A9
:10B48000D1F7702D01C080E060E09BDE1092453561
:10B490000895CF93DF93CDB7DEB72897CDBFDEBF3A
:10B4A0006115710520E28207910508F078C0DC0182
:10B4B000CB018093413590934235A0934335B093AF
:10B4C0004435809145358111AADE10924535809131
:10B4D000413590914235A0914335B0914435072EC6
:10B4E00075E1B695A795979587957A95D1F7702DC3
:10B4F00061E067DE82E8888741E050E0BE01685F76
:10B500007F4F80EB98E00F944834809141359091C3
:10B510004235A0914335B0914435AC01BD01032EB5
:10B5200039E076956795579547953A95D1F7302D3F
:10B53000032E3AE0440F551F661F771F3A95D1F747
:10B54000302D9170AA27BB27842B952BA62BB72BC8
:10B5500089839A83AB83BC838B818D8341E050E0E8
:10B56000BE016B5F7F4F80EB98E00F9448348A8177
:10B570008E8341E050E0BE016A5F7F4F80EB98E030
:10B580000F94483489818F8341E050E0BE01695FA8
:10B590007F4F80EB98E00F94483481E001C080E059
:10B5A0002896CDBFDEBFDF91CF910895CF93DF9373
:10B5B0001F92CDB7DEB78091413590914235A09171
:10B5C0004335B0914435AC01BD01517066277727F2
:10B5D000452B462B472B31F1198241E050E0BE014B
:10B5E0006F5F7F4F80EB98E00F9448348091413536
:10B5F00090914235A0914335B09144350196A11DFB
:10B60000B11D8093413590934235A0934335B0935B
:10B610004435AC01BD01517066277727452B462B79
:10B62000472BD1F60097A105B10569F00197A10953
:10B63000B109072E75E1B695A795979587957A95E7
:10B64000D1F7702D01C080E060E0BBDD81E0809328
:10B6500045350F90DF91CF9108950F931F93CF93AE
:10B66000DF931F92CDB7DEB7809145358823B1F0C7
:10B67000109245358091413590914235A0914335E6
:10B68000B0914435BC01CD01052E59E096958795C2
:10B69000779567955A95D1F7502DC9DE41E050E076
:10B6A000BE016F5F7F4F80EB98E00F945F34809115
:10B6B000413590914235A0914335B0914435AC016C
:10B6C000BD014F5F5F4F6F4F7F4F409341355093A8
:10B6D000423560934335709344358A019B01117064
:10B6E00022273327012B022B032BA1F4452B462BBA
:10B6F000472B51F0072E75E1B695A795979587953D
:10B700007A95D1F7702D01C080E060E05ADD81E0CC
:10B710008093453589810F90DF91CF911F910F91D3
:10B7200008950F931F93CF93DF931F92CDB7DEB78A
:10B73000182F80914535882349F0609141357091EB
:10B7400042358091433590914435A3DE198341E021
:10B7500050E0BE016F5F7F4F80EB98E00F9448345C
:10B760008091413590914235A0914335B091443557
:10B77000AC01BD014F5F5F4F6F4F7F4F409341352D
:10B780005093423560934335709344358A019B0151
:10B79000117022273327012B022B032BA1F4452BF9
:10B7A000462B472B51F0072E75E1B695A795979537
:10B7B00087957A95D1F7702D01C080E060E001DDBA
:10B7C00081E08093453581E00F90DF91CF911F910B
:10B7D0000F910895CF93DF931F921F92CDB7DEB7DD
:10B7E00080914535882309F440C08091413590917E
:10B7F0004235A0914335B0914435072E75E1B69599
:10B80000A795979587957A95D1F7702D61E0D9DC4A
:10B8100087ED8A8341E050E0BE016E5F7F4F80EB91
:10B8200098E00F94483441E050E0BE016F5F7F4FD5
:10B8300080EB98E00F945F348091413590914235D0
:10B84000A0914335B0914435072E75E1B695A79583
:10B85000979587957A95D1F7702D60E0B2DC898154
:10B860008095881F8827881F01C080E00F900F9067
:10B87000DF91CF910895CF93DF93EC01803C28E0D6
:10B88000920729F468E083E00F94773310C0803C7E
:10B8900029E0920729F468E084E00F94773307C029
:10B8A000803C9A4021F468E085E00F9477338881EA
:10B8B00080618883DF91CF910895EF92FF920F937B
:10B8C0001F93CF937C01C42FB901A80100E010E6BB
:10B8D0002AEE30E00E949166882344F0F7018081CF
:10B8E000CC0FCC0FCC70837FC82BC083CF911F911E
:10B8F0000F91FF90EF90089580E0089591E08111FD
:10B9000001C090E09093344081E0809344200895FA
:10B910000F931F930CE51EE52FE130E048E855E357
:10B9200061E082E00E941477811105C068E87CE53F
:10B9300082E00E9464781F910F910895CF93DF9366
:10B9400010926B3510926C350F94A334811104C0A2
:10B9500010928435D0E012C08150809384352ADC67
:10B96000D82F882359F0C0E060E08C2F0F94B934B1
:10B97000CF5F809184358C17B8F7CADF8D2FDF91A8
:10B98000CF910895C5CF08950F931F9302EC1CE546
:10B990002DE030E048E450E260E081E80E94147756
:10B9A000811105C064EC7CE581E80E9464781F91F8
:10B9B0000F91089580916C35882341F082E00E94B8
:10B9C0003D786AED7CE582E00C946478089580917E
:10B9D0006C35882341F081E80E943D7867EE7CE574
:10B9E00081E80C94647808958091502090915120C2
:10B9F000A0915220B0915320892B8A2B8B2B59F088
:10BA000080919435882324F481E80E943D7803C016
:10BA100082E00E943D7880918C3590918D35A09187
:10BA20008E35B0918F3580934C2090934D20A0930C
:10BA30004E20B0934F20A8CF0895E0E7F5E382E1D0
:10BA4000DF011D928A95E9F780EF80838AE0878382
:10BA50000895DF92EF92FF920F931F93CF93DF939E
:10BA6000D82EC62FD72F122F032FF42EE52EE5DF69
:10BA700081E080935420E0E7F5E3D282E382F48210
:10BA800005831683D487C587DF91CF911F910F91CE
:10BA9000FF90EF90DF90089520E030E0A90160E092
:10BAA00074E285E0D6CF08950F931F9320919435CB
:10BAB00042276CF00091502010915120209152208B
:10BAC00030915320061717072807390720F4E4DFC1
:10BAD0008BDF80E001C081E01F910F91089520E08D
:10BAE00030E0A90160E070E084E0B3CF08950F93E7
:10BAF0001F93262F30E00DE91DE5AC0161E081E8E0
:10BB00000E941477811102C0EADF6EDF1F910F914E
:10BB1000089520E030E0A90160E078E286E099CF66
:10BB2000089520E030E0A90160E07AE382E091CF5F
:10BB3000089583DF109254200895CF93DF938111ED
:10BB400011C0EB01F6DFE8E4F0E280859185A28583
:10BB5000B3858C1B9D0BA109B10980879187A287B2
:10BB6000B38742DFDF91CF9108951F93CF93DF9387
:10BB7000D82F84E1E0E5F5E3DF011D928A95E9F72E
:10BB8000DD2331F090919F35E8E5F5E318E005C03D
:10BB900090919B35E4E5F5E314E0809199358F733E
:10BBA0008C3111F08F3339F48CE180838AE081830A
:10BBB00085E08383145FC12F911708F4C92F8C2F60
:10BBC00090E0A0E0B0E040E8BC01CD016DDF88234B
:10BBD00009F1809195350F94C034811102C020E0A5
:10BBE00001C020E8DD2361F0E0E5F5E3812F90E07E
:10BBF000029798278927982780839183238306C0FB
:10BC0000E0E5F5E38FEF810F808322836C2F80E5E1
:10BC100095E36DDFDF91CF911F910895CF93C82FEA
:10BC200081110FC0809195350F94C034882349F05D
:10BC300020E030E0A90160E077E287E00ADFD4DEAF
:10BC400039C0A6E6B5E3E8E8F5E3818913968C935D
:10BC50001397828912968C931297838911968C93ED
:10BC6000119784898C93A4E6B5E3868911968C9309
:10BC7000119787898C936091643570916535CB01FC
:10BC8000A0E0B0E0BC01CD01052E59E0660F771FA2
:10BC9000881F991F5A95D1F7502DC11102C040E05D
:10BCA00001C040E801DF882329F0C0936A3581E0B4
:10BCB00080936B35CF9108950F931F93CF93DF93AC
:10BCC000811132C16F31710569F48091883590918D
:10BCD0008935A0918A35B0918B3585359345A2443D
:10BCE000B34431F081E080936C3564DE70DE1CC1BA
:10BCF000E8E8F5E395859F709587809184358917ED
:10BD000018F4CADE71DE10C1E8E8F5E3408551851C
:10BD10006285738540935020509351206093522048
:10BD200070935320478550E04B35510508F0EEC025
:10BD3000FA018827E958FE4F8F4F0D942D54C0917A
:10BD40009B35C33108F0C2E18C2F90E0A0E0B0E059
:10BD500040E8BC01CD01A8DE882309F4E5C06C2FC2
:10BD600080E795E3C4DEE0C0C0919B35C53208F0A2
:10BD7000C4E28C2F90E0A0E0B0E040E8BC01CD012F
:10BD800093DE882309F4D0C080919835837021F424
:10BD9000D0919935DD2319F07FDE26DEC5C0809174
:10BDA00095350F94C7348111D0E800E210E2F80114
:10BDB000D183809195350F94CE3420E1FC013196EA
:10BDC000A0E3B0E201900D922A95E1F7F801808995
:10BDD000882309F4A4C0823209F4A3C0E1E3F0E2AD
:10BDE00081E09191992309F49DC0923209F49AC09F
:10BDF0008F5F8031B1F708C0E82FF0E0E05EFF4DC3
:10BE0000908B8F5F8031C1F76C2F80E290E26FDE04
:10BE10008BC080E0AADE88C081E0A7DE85C0892FC4
:10BE20000F94A534823039F0833019F0811105C0A8
:10BE300006C06FDE05C075DE03C051DE01C079DECD
:10BE4000D3DD72C040E868E070E080E090E02CDE76
:10BE5000882309F469C068E475E3809195350F94EF
:10BE6000AC34823041F0833019F0811107C009C031
:10BE700050DEBADD59C055DEB7DD56C030DEB4DD68
:10BE800053C0E8E4F5E380E090E0A2E0B0E0848312
:10BE90009583A683B78380819181A281B3815A2F34
:10BEA0004B2F60E070E0982789279827A0E0B0E04A
:10BEB000DC0199278827842B952BA62BB72B808311
:10BEC0009183A283B38368E0CF0111DE2DC08091FE
:10BED0009B3581FF06C08095682F6170892F0F9474
:10BEE000B93427DE81DD20C080919B35811102C0ED
:10BEF00020DE01C0D1DD78DD17C01BDE75DD14C08A
:10BF000081E08CDE11C080E089DE0EC020E030E0F0
:10BF1000A90160E070E285E09CDD66DD05C080E09F
:10BF200001C080E090E268CFDF91CF911F910F9127
:10BF3000089510926B3542C9089580913D40882341
:10BF4000F4F480768032D9F580913E408E3FC9F579
:10BF500080914340909144400197A9F580913F40E2
:10BF600090914040892B89F5EDE3F0E484E895E376
:10BF70008087918781E090E082879387089580761B
:10BF8000803229F580913E408F3F19F580914340E2
:10BF900090914440892BF9F480913F40909140402A
:10BFA000892BD9F410926C3510926B3582E00E9487
:10BFB000D27781E80E94D277ABDC81E0089580E0FF
:10BFC000089580E0089580E0089580E0089580E07D
:10BFD000089580E0089580E0089580E00895CF936B
:10BFE000C0916B35CC23A9F110926B3580916A35E5
:10BFF000882389F02091643530916535409166350C
:10C0000050916735609168357091693580919535AB
:10C010000F94D63410C0209164353091653540912D
:10C0200066355091673560916835709169358091BA
:10C0300095350F94FA34823041F0833021F081112C
:10C0400006C077DD05C065DD03C06BDD01C047DDDF
:10C05000CBDC8C2FCF910895EF92FF920F931F931B
:10C06000CF93DF93982F80914420882309F448C010
:10C07000109244202115310511F0890102C00EE70C
:10C080001CE5911102C082E001C081E8E9017A015A
:10C09000AB01970160E00E941477811104C091E028
:10C0A000909344202DC0CD2BD9F480914420882337
:10C0B000E1F380913440811122C0E8E4F0E2808510
:10C0C0009185A285B3858E199F09A109B109808741
:10C0D0009187A287B3879091344081E0892710C06F
:10C0E000E8E4F0E240855185628573854E195F0969
:10C0F00061097109408751876287738701C080E0B9
:10C10000DF91CF911F910F91FF90EF900895E091F3
:10C11000AD35F091AE350190F081E02D2281338173
:10C120002E0F3F1FFC014081E40FF11DE217F307C2
:10C13000A0F481818430A1F0861306C014C08181EF
:10C140008430A1F08617A9F08081E80FF11DE21775
:10C15000F307A8F380E090E0089580E090E0089570
:10C1600080E090E008958E2F9F2F089580E090E06A
:10C1700008958E2F9F2F089580913F408F770C94C4
:10C180002F7608959091AF35992381F1E091AD35E7
:10C19000F091AE350190F081E02D9481891740F542
:10C1A000E093AB35F093AC35228133812E0F3F1FE6
:10C1B000E217F307F8F49181943061F492818913C6
:10C1C00009C09381961306C0E093AB35F093AC356C
:10C1D00081E008959081E90FF11DE217F30758F30C
:10C1E000E093AB35F093AC3580E0089580E008959E
:10C1F00080E0089580E00895EF92FF921F93CF931F
:10C20000DF93C82F60E0BEDF182F882381F1A09153
:10C21000AD35B091AE35EC2FF0E0EE0FFF1F12966A
:10C220008D919C911397E80FF91FE080F180D70161
:10C230001696ED91FC9117971995682F8C2FA2DF18
:10C24000182F8823A1F0C091AB35D091AC3565E0B3
:10C25000CE015DDFEC01892B21F08A810E942178DB
:10C26000F6CFD7011296ED91FC9113971995812F76
:10C27000DF91CF911F91FF90EF9008951F93CF937F
:10C28000DF93182F7FDF882341F1C091AB35D09128
:10C29000AC3565E0CE013BDFEC01892B49F04C81E8
:10C2A0005D816B818A810E943C768111F2CF15C03D
:10C2B000A091AD35B091AE35E12FF0E0EE0FFF1F4C
:10C2C00012968D919C911397E80FF91F0190F081C0
:10C2D000E02D0190F081E02D1995DF91CF911F9114
:10C2E00008950C94C7750895CF938091AF35882336
:10C2F000C1F0E091AD35F091AE350190F081E02DC7
:10C300008481882371F0C0E08C2F76DFCF5FE091CD
:10C31000AD35F091AE350190F081E02D8481C817E4
:10C3200098F31092AF3581E090E08093B035909310
:10C33000B135CF9108950E949375D6CF0895CF93CC
:10C340008091AF35882349F1A091AD35B091AE35DC
:10C35000ED91FC91119784818823F9F0C0E0EC2FD6
:10C36000F0E0EE0FFF1F12968D919C911397E80F4E
:10C37000F91F0190F081E02D0084F185E02D3097C8
:10C3800009F01995CF5FA091AD35B091AE35ED9123
:10C39000FC9111978481C81710F3CF9108950F93E2
:10C3A0001F93CF93DF93EDE3F0E412861386148698
:10C3B000158616861786808188230CF060C220912E
:10C3C0004340309144402115310509F05DC24FC210
:10C3D0008F7109F097C090913E40963081F098306F
:10C3E00009F485C091118EC02230310509F0FBC1DE
:10C3F00062E070E080EB95E30E9435764EC280915A
:10C400003F4090914040292F33272230310589F059
:10C410002330310579F12130310509F0A6C1809131
:10C42000622090916320DC016C9170E00E9435766F
:10C430004FC0E0916220F09163202189821708F0BB
:10C44000D2C19927880F991F880F991FE091642006
:10C45000F0916520E80FF91F80819181FC016281D4
:10C4600073810E943576E0914540F091464082E02C
:10C4700081832EC099278130910599F058F0823040
:10C48000910509F406C2039709F078C13CE0E3E79F
:10C49000F4E20AC064E070E088EC90E20E94357635
:10C4A00017C0EEEBF0E239E0A2EAB0E220E08191C1
:10C4B00090E08D939D932F5F2317C8F3632F660F32
:10C4C0006E5F6093A02070E080EA90E20E94357673
:10C4D000EDE3F0E486819781228533858217930707
:10C4E00008F0DBC18093474090934840D6C121308B
:10C4F000310509F078C161E070E08FEA95E30E94B0
:10C500003576CBC18130E9F590913E409A30C9F53E
:10C510002130310509F037C18091AF35882309F406
:10C5200032C1C0914140D09142400091AD3510914F
:10C53000AE35D801ED91FC918481C81708F023C174
:10C5400060E08C2F1FDE882309F418C1CE019927E3
:10C55000880F991FD8011296ED91FC911397E80F5F
:10C56000F91F0190F081E02D86819781FC011995DA
:10C570008093AA3561E070E08AEA95E30E943576FF
:10C580008CC1823009F0FAC080913E408111EFC029
:10C590002230310509F027C1809141400E94C476C4
:10C5A00090E08093A8359093A93562E070E088EA26
:10C5B00095E30E94357671C18F7109F084C0909126
:10C5C0003E40933009F4D5C018F49130A1F07BC0FF
:10C5D000953019F0993039F176C0809143409091AF
:10C5E0004440892B09F0FFC08CEB90E680934940D2
:10C5F00090934A4052C18091434090914440892B8E
:10C6000009F0F1C080913F4090914040019709F0BE
:10C61000EAC08091B0359091B1358D7F8093B0356F
:10C620009093B1353AC18091434090914440892B19
:10C6300009F0D9C00E943276882309F49FC0209166
:10C640003F40309140403327E0916220F0916320D9
:10C65000818990E08217930708F490C045DE8091AD
:10C660003F40909140408093AF35882309F415C135
:10C6700099278150904C880F991F880F991FE0913E
:10C680006420F0916520E80FF91FE093AD35F09339
:10C69000AE350190F081E02D8481882309F4FDC03E
:10C6A000C0E060E08C2FEADD882309F467C0CF5F2B
:10C6B000E091AD35F091AE350190F081E02D8481AF
:10C6C000C81778F3EAC08130E9F490913E409B307E
:10C6D000C9F48091434090914440892B09F053C0A4
:10C6E0008091AF35882309F44EC0EDE3F0E4C481B6
:10C6F000D2818C2F81DD882309F440C06D2F8C2FCF
:10C70000BDDD3AC08230D1F580913E40813019F0D4
:10C710008330A1F030C08091434090914440892BF8
:10C7200009F061C080913F4090914040892B09F011
:10C730005AC0809141400E94DF761EC080914340E4
:10C7400090914440892B09F04EC080913F409091D8
:10C750004040892B09F047C0CDE3D0E48C810E9492
:10C76000D2778C810E943D7807C080E005C080E0D0
:10C7700003C080E001C080E0811190C080913D4005
:10C780008F71813081F58091AF35882309F471C0B4
:10C790000091414010914240C091AD35D091AE35ED
:10C7A000E881F9818481081708F065C060E0802F76
:10C7B000E9DC8823C1F0F801FF27CF01880F991F1A
:10C7C000EA81FB81E80FF91FC081D181EE81FF81F1
:10C7D0001995682F802FD6DC882329F0EC81FD8104
:10C7E000199581115BC080913D408F71823009F0B5
:10C7F00044C08091AF358823B1F1A091AD35B0919F
:10C80000AE35ED91FC9111978481882371F1C0E0E0
:10C81000EC2FF0E0EE0FFF1F12968D919C91139775
:10C82000E80FF91F00811181D8011696ED91FC9156
:10C8300017971995682F8C2FA5DC882379F1D801DB
:10C840001496ED91FC9115971995811127C0CF5F32
:10C85000A091AD35B091AE35ED91FC9111979481D9
:10C86000C917B0F21BC080E019C080E017C080E09B
:10C8700015C080E013C080E011C080E00FC0982F89
:10C88000907609F07BCF98CE982F907609F076CFEE
:10C890009FCD33E0EAEBF0E207CE81E0DF91CF916C
:10C8A0001F910F9108958038910558F1672B21F45D
:10C8B000873C910571F41CC08F3F910509F0F8F495
:10C8C0009C01220F331FF901E05CF84D80819181BA
:10C8D0000895E2E4F8E221E030E0419151918417BB
:10C8E000950741F02F5F3F4F20383105B1F702C067
:10C8F00020E030E020583F4FC9019927089580E09B
:10C9000090E008958136910589F0E2E6F6E240E094
:10C9100050E04F5F5F4F219131912115310591F02A
:10C9200028173907B1F7892B19F40AC040E050E005
:10C93000440F551FFA01E058FB4D80819181089505
:10C9400080E090E0089543E050E060E880E096E009
:10C950000F94CF3343E050E064E080E296E00F9420
:10C96000CF3343E050E062E080E296E00F94CF33B3
:10C9700040E058E160E280EA96E00F94CF3341E076
:10C9800050E062E080EA96E00F94CF3343E050E05D
:10C9900060E180E896E00F94CF3343E050E060E13F
:10C9A00080E496E00F94CF3341E050E061E080E412
:10C9B00096E00F94CF3341E050E062E080E496E0EF
:10C9C0000F94CF3341E050E060E280E696E00F94B0
:10C9D000CF3341E050E062E080E096E00F94CF3347
:10C9E00043E050E062E080E696E00F94CF3340E011
:10C9F00050E061E080EA96E00F94CF3340E050E0F1
:10CA000061E080E096E00F94CF3340E050E068E0D2
:10CA100080E096E00F94CF3341E050E060E480E0A6
:10CA200096E00F94CF3340E058E161E080E896E073
:10CA30000F94CF3340E050E061E080E096E00F9447
:10CA4000CF3340E050E060E280E096E00F94CF33D7
:10CA500040E050E064E080E096E00F94CF3340E0A7
:10CA600050E061E080EA96E00F94CF3343E050E07D
:10CA700060E880E496E00F94CF3343E050E060E25A
:10CA800080E496E00F94CF3340E050E060E480E42F
:10CA900096E00F94CF3341E050E060E880E896E004
:10CAA0000F94CF3341E050E060E280E896E00F94CD
:10CAB000CF3340E050E060E480E896E00F94CF335D
:10CAC00043E050E068E080E496E00F94CF3340E02C
:10CAD00050E064E080E496E00F94CF3343E050E010
:10CAE00068E080E696E00F94CF3340E050E064E0E9
:10CAF00080E696E00F94CF3343E050E068E080E8B2
:10CB000096E00F94CF3340E050E064E080E896E098
:10CB10000F94CF3343E050E068E080EA96E00F9452
:10CB2000CF3340E050E064E080EA96E00F94CF33EA
:10CB300040E058E160E480EA96E00F94CF3340E0B3
:10CB400058E160E180E696E00F94CF3340E058E191
:10CB500061E080E296E00F94CF3343E050E060E87C
:10CB600080E496E00F94CF3343E050E060E280E44D
:10CB700096E00F94CF3340E050E060E480E496E02C
:10CB80000F94CF3343E050E060E880EA96E00F94E2
:10CB9000CF3343E050E060E880E496E00F94CF3379
:10CBA00043E050E060E280E496E00F94CF3340E051
:10CBB00050E060E480E496E00F94CF3343E050E02F
:10CBC00068E080E296E00F94CF3341E050E062E00D
:10CBD00080E896E00F94CF3340E050E061E080E6DB
:10CBE00096E00F94CF3340E050E060E180E096E0C3
:10CBF0000D94CF3308951F920F920FB60F92112408
:10CC00000BB60F928F939F93EF93FF93E5E3F0E4BE
:10CC100080819181019680839183FF91EF919F9113
:10CC20008F910F900BBE0F900FBE0F901F90189515
:10CC30001F920F920FB60F9211240BB60F92CF9244
:10CC4000DF92EF92FF920F931F932F933F934F9397
:10CC50005F936F937F938F939F93AF93BF93EF9364
:10CC6000FF93E5E3F0E48081918122813381821793
:10CC70009307F0F121E020930204E0913B40F09112
:10CC80003C403097A9F16091080470910904A0E03C
:10CC9000B0E0DC0199278827AB0160E070E08C01EF
:10CCA0009D01042B152B262B372BC901B801A5E3B9
:10CCB000B0E412960D911C91139720E030E098019A
:10CCC000112700271496CD90DC901597E12CF12CBC
:10CCD0000C291D292E293F29061717072807390770
:10CCE00030F0C901B8016F5F7F4F8F4F9F4F19958B
:10CCF000FF91EF91BF91AF919F918F917F916F9134
:10CD00005F914F913F912F911F910F91FF90EF9065
:10CD1000DF90CF900F900BBE0F900FBE0F901F9023
:10CD20001895CF92DF92EF92FF920F931F93CF93BC
:10CD3000DF93EC016A017B01DB01CA010197A109C4
:10CD4000B109BC01CD01600F711F821F931FA701A4
:10CD500096010F94EF532138310541055105F8F440
:10CD6000213460F4213260F4213160F4293060F420
:10CD7000253060F4233060F490E80BC093E009C0E4
:10CD800092E007C092E805C091E003C091E801C0BD
:10CD900090E088818C77892B888381E001C08FEFB8
:10CDA000DF91CF911F910F91FF90EF90DF90CF9087
:10CDB00008951F920F920FB60F9211240BB60F9287
:10CDC0002F933F934F935F936F937F938F939F9393
:10CDD000AF93BF93EF93FF93E091F835F091F9355E
:10CDE000309709F01995FF91EF91BF91AF919F9105
:10CDF0008F917F916F915F914F913F912F910F9004
:10CE00000BBE0F900FBE0F901F9018951F920F92A0
:10CE10000FB60F9211240BB60F922F933F934F939F
:10CE20005F936F937F938F939F93AF93BF93EF9392
:10CE3000FF93E091F635F091F735309709F01995A9
:10CE4000FF91EF91BF91AF919F918F917F916F91E2
:10CE50005F914F913F912F910F900BBE0F900FBE9E
:10CE60000F901F9018951F920F920FB60F921124DA
:10CE70000BB60F922F933F934F935F936F937F93D4
:10CE80008F939F93AF93BF93EF93FF93E091F4350C
:10CE9000F091F535309709F01995FF91EF91BF9119
:10CEA000AF919F918F917F916F915F914F913F9142
:10CEB0002F910F900BBE0F900FBE0F901F901895E3
:10CEC0001F920F920FB60F9211240BB60F922F9351
:10CED0003F934F935F936F937F938F939F93AF9302
:10CEE000BF93EF93FF93E091F235F091F3353097D4
:10CEF00009F01995FF91EF91BF91AF919F918F919B
:10CF00007F916F915F914F913F912F910F900BBE49
:10CF10000F900FBE0F901F9018951F920F920FB693
:10CF20000F9211240BB60F922F933F934F935F9361
:10CF30006F937F938F939F93AF93BF93EF93FF93E1
:10CF4000E091F035F091F135309709F01995FF91A6
:10CF5000EF91BF91AF919F918F917F916F915F9171
:10CF60004F913F912F910F900BBE0F900FBE0F90DE
:10CF70001F9018951F920F920FB60F9211240BB6A7
:10CF80000F922F933F934F935F936F937F938F9362
:10CF90009F93AF93BF93EF93FF93E091EE35F091A2
:10CFA000EF35309709F01995FF91EF91BF91AF914F
:10CFB0009F918F917F916F915F914F913F912F91B1
:10CFC0000F900BBE0F900FBE0F901F9018951F92E1
:10CFD0000F920FB60F9211240BB60F922F933F931F
:10CFE0004F935F936F937F938F939F93AF93BF9371
:10CFF000EF93FF93E091EC35F091ED35309709F028
:10D000001995FF91EF91BF91AF919F918F917F9172
:10D010006F915F914F913F912F910F900BBE0F90A9
:10D020000FBE0F901F9018951F920F920FB60F9280
:10D0300011240BB60F922F933F934F935F936F93EF
:10D040007F938F939F93AF93BF93EF93FF93E09161
:10D05000EA35F091EB35309709F01995FF91EF9192
:10D06000BF91AF919F918F917F916F915F914F9100
:10D070003F912F910F900BBE0F900FBE0F901F90FE
:10D0800018951F920F920FB60F9211240BB60F92A4
:10D090002F933F934F935F936F937F938F939F93C0
:10D0A000AF93BF93EF93FF93E091E835F091E935AB
:10D0B000309709F01995FF91EF91BF91AF919F9132
:10D0C0008F917F916F915F914F913F912F910F9031
:10D0D0000BBE0F900FBE0F901F9018951F920F92CE
:10D0E0000FB60F9211240BB60F922F933F934F93CD
:10D0F0005F936F937F938F939F93AF93BF93EF93C0
:10D10000FF93E091E635F091E735309709F01995F6
:10D11000FF91EF91BF91AF919F918F917F916F910F
:10D120005F914F913F912F910F900BBE0F900FBECB
:10D130000F901F9018951F920F920FB60F92112407
:10D140000BB60F922F933F934F935F936F937F9301
:10D150008F939F93AF93BF93EF93FF93E091E43549
:10D16000F091E535309709F01995FF91EF91BF9156
:10D17000AF919F918F917F916F915F914F913F916F
:10D180002F910F900BBE0F900FBE0F901F90189510
:10D190001F920F920FB60F9211240BB60F922F937E
:10D1A0003F934F935F936F937F938F939F93AF932F
:10D1B000BF93EF93FF93E091E235F091E335309721
:10D1C00009F01995FF91EF91BF91AF919F918F91C8
:10D1D0007F916F915F914F913F912F910F900BBE77
:10D1E0000F900FBE0F901F9018951F920F920FB6C1
:10D1F0000F9211240BB60F922F933F934F935F938F
:10D200006F937F938F939F93AF93BF93EF93FF930E
:10D21000E091E035F091E135309709F01995FF91F3
:10D22000EF91BF91AF919F918F917F916F915F919E
:10D230004F913F912F910F900BBE0F900FBE0F900B
:10D240001F9018951F920F920FB60F9211240BB6D4
:10D250000F922F933F934F935F936F937F938F938F
:10D260009F93AF93BF93EF93FF93E091DE35F091DF
:10D27000DF35309709F01995FF91EF91BF91AF918C
:10D280009F918F917F916F915F914F913F912F91DE
:10D290000F900BBE0F900FBE0F901F9018951F920E
:10D2A0000F920FB60F9211240BB60F922F933F934C
:10D2B0004F935F936F937F938F939F93AF93BF939E
:10D2C000EF93FF93E091DC35F091DD35309709F075
:10D2D0001995FF91EF91BF91AF919F918F917F91A0
:10D2E0006F915F914F913F912F910F900BBE0F90D7
:10D2F0000FBE0F901F9018951F920F920FB60F92AE
:10D3000011240BB60F922F933F934F935F936F931C
:10D310007F938F939F93AF93BF93EF93FF93E0918E
:10D32000DA35F091DB35309709F01995FF91EF91DF
:10D33000BF91AF919F918F917F916F915F914F912D
:10D340003F912F910F900BBE0F900FBE0F901F902B
:10D3500018951F920F920FB60F9211240BB60F92D1
:10D360002F933F934F935F936F937F938F939F93ED
:10D37000AF93BF93EF93FF93E091D835F091D935F8
:10D38000309709F01995FF91EF91BF91AF919F915F
:10D390008F917F916F915F914F913F912F910F905E
:10D3A0000BBE0F900FBE0F901F9018951F920F92FB
:10D3B0000FB60F9211240BB60F922F933F934F93FA
:10D3C0005F936F937F938F939F93AF93BF93EF93ED
:10D3D000FF93E091D635F091D735309709F0199544
:10D3E000FF91EF91BF91AF919F918F917F916F913D
:10D3F0005F914F913F912F910F900BBE0F900FBEF9
:10D400000F901F9018951F920F920FB60F92112434
:10D410000BB60F922F933F934F935F936F937F932E
:10D420008F939F93AF93BF93EF93FF93E091D43586
:10D43000F091D535309709F01995FF91EF91BF9193
:10D44000AF919F918F917F916F915F914F913F919C
:10D450002F910F900BBE0F900FBE0F901F9018953D
:10D460001F920F920FB60F9211240BB60F922F93AB
:10D470003F934F935F936F937F938F939F93AF935C
:10D48000BF93EF93FF93E091D235F091D33530976E
:10D4900009F01995FF91EF91BF91AF919F918F91F5
:10D4A0007F916F915F914F913F912F910F900BBEA4
:10D4B0000F900FBE0F901F9018951F920F920FB6EE
:10D4C0000F9211240BB60F922F933F934F935F93BC
:10D4D0006F937F938F939F93AF93BF93EF93FF933C
:10D4E000E091D035F091D135309709F01995FF9141
:10D4F000EF91BF91AF919F918F917F916F915F91CC
:10D500004F913F912F910F900BBE0F900FBE0F9038
:10D510001F9018951F920F920FB60F9211240BB601
:10D520000F922F933F934F935F936F937F938F93BC
:10D530009F93AF93BF93EF93FF93E091CE35F0911C
:10D54000CF35309709F01995FF91EF91BF91AF91C9
:10D550009F918F917F916F915F914F913F912F910B
:10D560000F900BBE0F900FBE0F901F9018951F923B
:10D570000F920FB60F9211240BB60F922F933F9379
:10D580004F935F936F937F938F939F93AF93BF93CB
:10D59000EF93FF93E091CC35F091CD35309709F0C2
:10D5A0001995FF91EF91BF91AF919F918F917F91CD
:10D5B0006F915F914F913F912F910F900BBE0F9004
:10D5C0000FBE0F901F9018951F920F920FB60F92DB
:10D5D00011240BB60F922F933F934F935F936F934A
:10D5E0007F938F939F93AF93BF93EF93FF93E091BC
:10D5F000CA35F091CB35309709F01995FF91EF912D
:10D60000BF91AF919F918F917F916F915F914F915A
:10D610003F912F910F900BBE0F900FBE0F901F9058
:10D6200018951F920F920FB60F9211240BB60F92FE
:10D630002F933F934F935F936F937F938F939F931A
:10D64000AF93BF93EF93FF93E091C835F091C93545
:10D65000309709F01995FF91EF91BF91AF919F918C
:10D660008F917F916F915F914F913F912F910F908B
:10D670000BBE0F900FBE0F901F9018951F920F9228
:10D680000FB60F9211240BB60F922F933F934F9327
:10D690005F936F937F938F939F93AF93BF93EF931A
:10D6A000FF93E091C635F091C735309709F0199591
:10D6B000FF91EF91BF91AF919F918F917F916F916A
:10D6C0005F914F913F912F910F900BBE0F900FBE26
:10D6D0000F901F9018951F920F920FB60F92112462
:10D6E0000BB60F922F933F934F935F936F937F935C
:10D6F0008F939F93AF93BF93EF93FF93E091C435C4
:10D70000F091C535309709F01995FF91EF91BF91D0
:10D71000AF919F918F917F916F915F914F913F91C9
:10D720002F910F900BBE0F900FBE0F901F9018956A
:10D730001F920F920FB60F9211240BB60F922F93D8
:10D740003F934F935F936F937F938F939F93AF9389
:10D75000BF93EF93FF93E091C235F091C3353097BB
:10D7600009F01995FF91EF91BF91AF919F918F9122
:10D770007F916F915F914F913F912F910F900BBED1
:10D780000F900FBE0F901F9018951F920F920FB61B
:10D790000F9211240BB60F922F933F934F935F93E9
:10D7A0006F937F938F939F93AF93BF93EF93FF9369
:10D7B000E091C035F091C135309709F01995FF918E
:10D7C000EF91BF91AF919F918F917F916F915F91F9
:10D7D0004F913F912F910F900BBE0F900FBE0F9066
:10D7E0001F9018951F920F920FB60F9211240BB62F
:10D7F0000F922F933F934F935F936F937F938F93EA
:10D800009F93AF93BF93EF93FF93E091BE35F09159
:10D81000BF35309709F01995FF91EF91BF91AF9106
:10D820009F918F917F916F915F914F913F912F9138
:10D830000F900BBE0F900FBE0F901F9018951F9268
:10D840000F920FB60F9211240BB60F922F933F93A6
:10D850004F935F936F937F938F939F93AF93BF93F8
:10D86000EF93FF93E091BC35F091BD35309709F00F
:10D870001995FF91EF91BF91AF919F918F917F91FA
:10D880006F915F914F913F912F910F900BBE0F9031
:10D890000FBE0F901F9018951F920F920FB60F9208
:10D8A00011240BB60F922F933F934F935F936F9377
:10D8B0007F938F939F93AF93BF93EF93FF93E091E9
:10D8C000BA35F091BB35309709F01995FF91EF917A
:10D8D000BF91AF919F918F917F916F915F914F9188
:10D8E0003F912F910F900BBE0F900FBE0F901F9086
:10D8F00018951F920F920FB60F9211240BB60F922C
:10D900002F933F934F935F936F937F938F939F9347
:10D91000AF93BF93EF93FF93E091B835F091B93592
:10D92000309709F01995FF91EF91BF91AF919F91B9
:10D930008F917F916F915F914F913F912F910F90B8
:10D940000BBE0F900FBE0F901F9018951F920F9255
:10D950000FB60F9211240BB60F922F933F934F9354
:10D960005F936F937F938F939F93AF93BF93EF9347
:10D97000FF93E091B635F091B735309709F01995DE
:10D98000FF91EF91BF91AF919F918F917F916F9197
:10D990005F914F913F912F910F900BBE0F900FBE53
:10D9A0000F901F9018951F920F920FB60F9211248F
:10D9B0000BB60F922F933F934F935F936F937F9389
:10D9C0008F939F93AF93BF93EF93FF93E091B43501
:10D9D000F091B535309709F01995FF91EF91BF910E
:10D9E000AF919F918F917F916F915F914F913F91F7
:10D9F0002F910F900BBE0F900FBE0F901F90189598
:10DA00001F920F920FB60F9211240BB60F922F9305
:10DA10003F934F935F936F937F938F939F93AF93B6
:10DA2000BF93EF93FF93E091B235F091B335309708
:10DA300009F01995FF91EF91BF91AF919F918F914F
:10DA40007F916F915F914F913F912F910F900BBEFE
:10DA50000F900FBE0F901F901895CF93CFB7F894EB
:10DA6000282F392F211588E0380749F461E083E039
:10DA70000F94773364E083E00F9477334FC0203402
:10DA800088E0380749F462E083E00F94773364E07C
:10DA900083E00F94773342C0211589E0380749F4B9
:10DAA00061E084E00F94773364E084E00F9477338F
:10DAB00035C0203489E0380749F462E084E00F94EF
:10DAC000773364E084E00F94773328C021158AE02F
:10DAD000380749F461E085E00F94773364E085E02E
:10DAE0000F9477331BC020348AE0380749F462E092
:10DAF00085E00F94773364E085E00F9477330EC0B0
:10DB000021153B4049F461E086E00F94773364E0EF
:10DB100086E00F94773302C0CFBF01C0CFBFCF9153
:10DB20000895CF93CFB7F894282F392F211588E087
:10DB3000380749F461E083E00F94833364E083E0C5
:10DB40000F9483334FC0203488E0380749F462E0F3
:10DB500083E00F94833364E083E00F94833342C007
:10DB6000211589E0380749F461E084E00F9483339C
:10DB700064E084E00F94833335C0203489E03807B3
:10DB800049F462E084E00F94833364E084E00F940E
:10DB9000833328C021158AE0380749F461E085E025
:10DBA0000F94833364E085E00F9483331BC02034EB
:10DBB0008AE0380749F462E085E00F94833364E03B
:10DBC00085E00F9483330EC021153B4049F461E09A
:10DBD00086E00F94833364E086E00F94833302C0C1
:10DBE000CFBF01C0CFBFCF910895811528E0920724
:10DBF00029F46093F8357093F9350895803428E05E
:10DC0000920729F46093EC357093ED3508958115F2
:10DC100029E0920729F46093E4357093E53508957F
:10DC2000803429E0920729F46093D8357093D93570
:10DC3000089581152AE0920729F46093D0357093F6
:10DC4000D135089580342AE0920729F46093C435D1
:10DC50007093C535089581159B4021F46093BC35C0
:10DC60007093BD350895FC01918195FFFDCF6083D0
:10DC700080E090E008954F925F926F927F928F9232
:10DC80009F92AF92BF92EF92FF920F931F93CF9309
:10DC90007C014A015B0128013901FC01848182FF7A
:10DCA00016C0D901C801689412F8B695A795979542
:10DCB00087951694D1F7B901A801032E36E1769520
:10DCC0006795579547953A95D1F7302D15C0D901ED
:10DCD000C801689413F8B695A795979587951694FB
:10DCE000D1F7B901A801032E37E1769567955795CD
:10DCF00047953A95D1F7302D88159905AA05BB05AA
:10DD000008F4A6C084169506A606B70608F4A2C0B5
:10DD1000F701848182FD04C0880C991CAA1CBB1CDD
:10DD2000C301B201A50194010F94EF532F3F3105B8
:10DD30004105510508F490C08FEF90E0A0E0B0E0FD
:10DD4000C9EF05C0281739074A075B0758F0880F45
:10DD5000991FAA1FBB1FCD3F0CF48160CF5FC73056
:10DD600089F74FC0CC230CF04CC0D501C401880FFB
:10DD7000991FAA1FBB1F880F991FAA1FBB1F880FBF
:10DD8000991FAA1FBB1F481A590A6A0A7B0ACE3F6D
:10DD9000F4F48DEF9FEF8C1B9109C7FD939504C0A0
:10DDA000440C551C661C771C8A95D2F7D501C4011A
:10DDB000B695A79597958795BC01CD01640D751D06
:10DDC000861D971DA50194010F94EF5337C083E082
:10DDD0008C0FA501940104C0220F331F441F551F4F
:10DDE0008A95D2F7DA01C901B695A79597958795D7
:10DDF000BC01CD01640D751D861D971D0F94EF5359
:10DE00001DC083E08C0FA501940104C0220F331FB5
:10DE1000441F551F8A95D2F7DA01C901B695A79517
:10DE200097958795BC01CD01640D751D861D971DC5
:10DE30000F94EF532150310941095109832F8F70FD
:10DE4000C295C07FC82BF701C783268381E018C025
:10DE500080E016C080E014C0D501C401880F991F6E
:10DE6000AA1FBB1F880F991FAA1FBB1F880F991FCE
:10DE7000AA1FBB1F481A590A6A0A7B0AC9EF89CF31
:10DE8000CF911F910F91FF90EF90BF90AF909F9017
:10DE90008F907F906F905F904F9008950F931F9396
:10DEA000CF93DF93EC018B01009709F41EC1803CF6
:10DEB000910529F460E180E00F94773316C1C11514
:10DEC00084E0D80729F464E080E00F9477330DC133
:10DED000C038E1E0DE0729F462E080E00F94773398
:10DEE00004C1C115F1E0DF0729F461E080E00F947F
:10DEF0007733FBC0C03883E0D80729F461E081E0C4
:10DF00000F947733F2C0C039E3E0DE0729F461E013
:10DF100082E00F947733E9C0C115F2E0DF0729F4FE
:10DF200062E081E00F947733E0C0C03482E0D8072C
:10DF300029F462E082E00F947733D7C0C032E3E087
:10DF4000DE0729F464E082E00F947733CEC0C11578
:10DF5000F8E0DF0729F461E083E00F947733C5C070
:10DF6000C11589E0D80729F461E084E00F94773384
:10DF7000BCC0C115EAE0DE0729F461E085E00F943A
:10DF80007733B3C0C115FBE0DF0729F461E086E019
:10DF90000F947733AAC0C03488E0D80729F462E030
:10DFA00083E00F947733A1C0C034E9E0DE0729F4A1
:10DFB00062E084E00F94773398C0C034FAE0DF0762
:10DFC00029F462E085E00F9477338FC0C03988E090
:10DFD000D80729F464E083E00F94773386C0C03912
:10DFE000E9E0DE0729F464E084E00F9477337DC034
:10DFF000C039FAE0DF0729F464E085E00F94773355
:10E0000074C0C0398BE0D80729F464E086E00F942F
:10E0100077336BC0C03CE8E0DE0729F468E083E0BA
:10E020000F94773362C0C03CF9E0DF0729F468E061
:10E0300084E00F94773359C0C03C8AE0D80729F4B4
:10E0400068E085E00F94773350C0C03AE8E0DE071F
:10E0500029F460E183E00F94773347C0C03AF9E0D8
:10E06000DF0729F460E184E00F9477333EC0C03AC3
:10E070008AE0D80729F460E185E00F94773335C052
:10E08000C03AEBE0DE0729F460E186E00F947733D5
:10E090002CC0C03BF8E0DF0729F460E283E00F9476
:10E0A000773323C0C03B89E0D80729F460E284E0DD
:10E0B0000F9477331AC0C03BEAE0DE0729F460E230
:10E0C00085E00F94773311C0C038F4E0DF0729F4FE
:10E0D00060E483E00F94773308C0C03A84E0D80747
:10E0E00021F460E485E00F9477338D818F738D8305
:10E0F000F80195818481892B9681911198E0892B73
:10E100008D83F801408151816281738100E010E6C6
:10E110002AEE30E0CE01AFDD9C8198609C839C812B
:10E1200090619C83DF91CF911F910F910895CF92C1
:10E13000DF92EF92FF920F931F93CF93DF93EC0147
:10E14000D901C801B695A79597958795481759079E
:10E150006A077B0778F46A017B01CC0CDD1CEE1C9E
:10E16000FF1CC901B801A70196010F94EF5321507C
:10E17000310902C020E030E0832F8F708F832E831F
:10E18000DF91CF911F910F91FF90EF90DF90CF9093
:10E190000895EF92FF920F931F93CF93DF93EC01BB
:10E1A0007B01009709F4B9C1803C910529F460E135
:10E1B00080E00F947733B1C18115944029F464E075
:10E1C00080E00F947733A9C1C03881E0D80729F4E3
:10E1D00062E080E00F947733A0C1C115E1E0DE0773
:10E1E00029F461E080E00F94773397C1C038F3E001
:10E1F000DF0729F461E081E00F9477338EC1C039E5
:10E2000033E0D30729F461E082E00F94773385C1CE
:10E21000C11582E0D80729F462E081E00F947733DA
:10E220007CC1C034E2E0DE0729F462E082E00F94B2
:10E23000773373C1C032F3E0DF0729F464E082E092
:10E240000F9477336AC1C11538E0D30729F461E030
:10E2500083E00F94773361C1C11589E0D80729F4B1
:10E2600061E084E00F94773358C1C115EAE0DE071E
:10E2700029F461E085E00F9477334FC1C115FBE0CD
:10E28000DF0729F461E086E00F94773346C1C0349C
:10E2900038E0D30729F462E083E00F9477333DC17F
:10E2A000C03489E0D80729F462E084E00F94773322
:10E2B00034C1C034EAE0DE0729F462E085E00F945F
:10E2C00077332BC1C039F8E0DF0729F464E083E03D
:10E2D0000F94773322C1C03939E0D30729F464E0C1
:10E2E00084E00F94773319C1C0398AE0D80729F444
:10E2F00064E085E00F94773310C1C039EBE0DE07AE
:10E3000029F464E086E00F94773307C1C03CF8E05D
:10E31000DF0729F468E083E00F947733FEC0C03C48
:10E3200039E0D30729F468E084E00F947733F5C02F
:10E33000C03C8AE0D80729F468E085E00F94773381
:10E34000ECC0C03AE8E0DE0769F460E183E00F94D6
:10E350007733E0EAF8E084818F7E8483F7012481BB
:10E36000225053C0C03AF9E0DF0729F460E184E0AD
:10E370000F947733D2C0C03A3AE0D30729F460E172
:10E3800085E00F947733C9C0C03A8BE0D80729F4F1
:10E3900060E186E00F947733C0C0C03BE8E0DE0761
:10E3A00029F460E283E00F947733B7C0C03BF9E013
:10E3B000DF0729F460E284E00F947733AEC0C03BFE
:10E3C0003AE0D30729F460E285E00F947733A5C0E3
:10E3D000C03884E0D80729F460E483E00F947733F1
:10E3E0009CC0C03AE4E0DE0729F460E485E00F94C5
:10E3F000773393C08C818F7E8C83FB0124812250E4
:10E40000CE01C03AF8E0DF0731F480914E0684FD7A
:10E410008CC011E18BC0803B38E0930779F0803AE3
:10E42000E9E09E0731F430916E0634FD82C019E1B7
:10E4300010C0803BF9E09F0789F001C015E1803AE8
:10E440003AE0930731F480918E0684FD74C011E2A6
:10E4500012C0803BEAE09E0759F001C01DE1803AFE
:10E460009B4049F48091AE0684FD04C019E203C0CC
:10E4700015E201C01DE2E12FE695E695E69530E252
:10E48000E39FF0011124FA5F177081E090E0012E04
:10E4900002C0880F991F0A94E2F78183223010F09E
:10E4A00040E001C040E4DF015096A10FB11D3FB72D
:10E4B000F8942C9127702C939C91942B9C933FBFA4
:10E4C00085838D81806C8D83F70184818D7F813080
:10E4D00021F48D8182608D8303C08D818D7F8D833A
:10E4E000F7018581882321F08D8184608D8303C0AD
:10E4F0008D818B7F8D83F701408151816281738192
:10E5000000E010E62AEE30E0CE0111DE8C8188605A
:10E510008C838C8180618C8310C08C818F7E8C83F6
:10E52000F70124812250CE0176CF15E180EA98E0F0
:10E5300080CF1DE18ECF15E29ECFDF91CF911F914D
:10E540000F91FF90EF9008950F93E8ECF4E0808135
:10E550008F7D808380818F7D8083E8EFF6E302E00A
:10E5600005931092FA361092FB3600E2069300E40F
:10E570000693E0EFF6E300E2069300E40693EDE392
:10E58000F0E4148615861686178612861386109276
:10E59000E3360F9108950F9385E08093E336E9EF1A
:10E5A000F6E304E00593E1EFF6E304E005930F9151
:10E5B00008950F9383E08093E3361092FA36109219
:10E5C000FB36E8EFF6E302E006930F910895E09141
:10E5D0004940F0914A40309709F0199508950F93FA
:10E5E000CF93DF938091E336833019F4F0DFACDF13
:10E5F0005EC08091DF369091E036C0914740D09167
:10E600004840C81BD90B71F52091E1363091E236B4
:10E61000820F931F8093E1369093E236209143401E
:10E62000309144408217930721F08091FA35882376
:10E6300041F084E08093E336E0EFF6E302E00693F6
:10E6400036C0E0914B40F0914C40309799F01995CD
:10E65000882381F01092DF361092E036C091474057
:10E66000D0914840C034D10528F01092FA35C0E46A
:10E67000D0E003C081E08093FA35E4EEF6E3C68B88
:10E68000D78B8091DF369091E036209145403091D4
:10E690004640280F391F208F318FC80FD91FC093D4
:10E6A000DF36D093E036E8EFF6E302E00693DF9141
:10E6B000CF910F910895FC018181E82FE7708E2F93
:10E6C00090E0FC013197E730F105D8F48827EE524D
:10E6D000FE4F8F4F0D942D5480E190E0089580E21D
:10E6E00090E0089580E490E0089580E890E0089537
:10E6F00080E091E0089580E092E008958FEF93E04C
:10E70000089588E090E00895282F2F7030E0220FC0
:10E71000331F082E000C990B8827990F881F992703
:10E72000820F931F02979C01220F331F220F331F6A
:10E73000220F331F820F931F8558994C08950F9312
:10E74000CF938091CC0480FF63C081E08093CC04A0
:10E75000E0EFF6E300E80693E8EFF6E300E806935F
:10E760008093CA04E0EFF6E300E106938091E3367C
:10E77000882329F08350823008F429DFE5DE809178
:10E78000F2369091F336089709F044C088E0EFE93B
:10E79000F6E3ADE3B0E401900D928A95E1F7E8EC81
:10E7A000F4E08081806280838081806280830E9427
:10E7B000CF61C82F811103C0EEDEC1E02CC0809173
:10E7C0003D4088236CF41092E1361092E2361092AC
:10E7D000DF361092E03682E08093E33600DF1BC024
:10E7E0008091434090914440892B11F4E2DE13C0A4
:10E7F0001092E1361092E2361092DF361092E03637
:10E8000081E08093E336E0EFF6E302E0069303C095
:10E81000C0E001C0C1E08C2FCF910F9108958F927D
:10E820009F92AF92BF92DF92EF92FF920F931F934E
:10E83000CF93DF93D82E68DF8C01CD2DCF70D0E041
:10E84000CE01880F991FCD2D0D2C000CDD0BCC2790
:10E85000DD0FCC1FDD27C80FD91FCE01880F991FF0
:10E86000880F991F880F991F9C012051394C7901FD
:10E87000C90121DF4C01DD200CF07BC0FE01EE0F51
:10E88000FF1FEE0FFF1FEE0FFF1FEC51F94C228907
:10E890003389D80115968D919C911697820F931FFD
:10E8A00015968D939C93169713962D913C911497E2
:10E8B0008217930709F447C0281B390B2115B4E0D0
:10E8C0003B0740F02FEF33E0C901B4010F94C85368
:10E8D000281B390BF801808181FF0AC0C901B401EE
:10E8E0000F94C85341E0892B09F040E0842F01C008
:10E8F00080E0D8019C9180FB91F99C93FE01EE0F82
:10E90000FF1FEE0FFF1FEE0FFF1FEC51F94C128A95
:10E91000138A2687378711962D913C911297159669
:10E920008D919C911697820F931FCC0FDD1FCC0FFA
:10E93000DD1FCC0FDD1FCC50D94C88839983F701A4
:10E9400002E00693E4C0D8018C9181FFCDC08D7F99
:10E950008C93CC0FDD1FCC0FDD1FCC0FDD1FCC51F6
:10E96000D94C1A8A1B8A1E861F86F70102E006937D
:10E97000CEC0FE01EE0FFF1FEE0FFF1FEE0FFF1FB9
:10E98000EC51F94CA684B784D8018C9182FF1BC04E
:10E990001196ED91FC91129715962D913C91169739
:10E9A00013968D919C911497B4010F94C853B0E4C1
:10E9B000DB9EB001112465547A4CAC01CF01820F6B
:10E9C000931F0F942C56F801258136812A0D3B1D8B
:10E9D00025833683838194818217930768F4858326
:10E9E0009683CC0FDD1FCC0FDD1FCC0FDD1FCC516C
:10E9F000D94C8A899B8978C0FE01EE0FFF1FEE0F6C
:10EA0000FF1FEE0FFF1FEC51F94C42895389A416EA
:10EA1000B50609F069C02817390709F465C0AC01CB
:10EA2000421B530B9A01211554E0350748F02FEF94
:10EA300033E0C901B4010F94C853281B390B06C039
:10EA4000C901B4010F94C853281B390BFE01EE0F06
:10EA5000FF1FEE0FFF1FEE0FFF1FEC51F94C168644
:10EA600017862815390500F5D8018C9184608C93A0
:10EA7000B0E4DB9EC001112485549A4CFE01EE0FD8
:10EA8000FF1FEE0FFF1FEE0FFF1FEC50F94C8083AE
:10EA90009183CC0FDD1FCC0FDD1FCC0FDD1FCC51C0
:10EAA000D94C8A8A9B8A1CC0F80141815281858198
:10EAB0009681840F951FFE01EE0FFF1FEE0FFF1FC3
:10EAC000EE0FFF1FEC50F94C80839183CC0FDD1FBC
:10EAD000CC0FDD1FCC0FDD1FCC51D94C2A8B3B8BCB
:10EAE000F70102E0069313C0D8018C9180FF0FC09C
:10EAF0008E7F8C931796ED91FC911897309739F093
:10EB000015966D917C9116974D2D80E01995DF91AA
:10EB1000CF911F910F91FF90EF90DF90BF90AF903A
:10EB20009F908F900895CF93CFB7F894E1ECF4E0E5
:10EB300080818E7F80831092C00410820F94C63330
:10EB400010922437CFBFCF9108959FB7F89481E0FA
:10EB500080932437EAECF4E080E4808380E28083D1
:10EB6000E1ECF4E0808181608083A9ECB4E08C91D9
:10EB700082608C93E8ECF4E08081806480838C91E7
:10EB800081608C938081806880839FBF0895CF933C
:10EB9000DF93C0E6D0E0188280E30F948E33E0EC80
:10EBA000F4E080818064808381E08883CFB7F8942B
:10EBB000E4EEF6E31586158A158E15A215A615AA9C
:10EBC000EBE7F6E380818E7F8083E4E8F6E38081E3
:10EBD0008E7F8083EDE8F6E380818E7F8083E6E997
:10EBE000F6E380818E7F80836AE170E082E00F949B
:10EBF00088518F3F19F08093FA0403C08FE180930E
:10EC0000FA046BE170E082E00F9488518F3F19F0B5
:10EC10008093FB0403C08FE18093FB04E0ECF4E0FD
:10EC20008081826080838081806880838081806130
:10EC3000808380EF96E386839783808180628083E0
:10EC40008FEF8093C504E8ECF4E0808181608083DD
:10EC5000109224377ADFCFBFDF91CF910895809350
:10EC6000C30408958091C3040895EDE3F0E4808720
:10EC70009187628773870895282F2F7030E0220FC5
:10EC8000331F082E000C990B8827990F881F99278E
:10EC9000820F931FFC01EE0FFF1FEE0FFF1FEE0F01
:10ECA000FF1FEC51F94C2585207C09F069C0637089
:10ECB000613011F018F404C060EC03C060E801C0DA
:10ECC00060E440385105E9F050F440325105A9F0B4
:10ECD00040345105A1F040315105D9F40CC0411523
:10ECE00022E0520791F04F3F23E0520781F0411597
:10ECF000514079F408C021E00DC022E00BC023E0B0
:10ED000009C024E007C025E005C026E003C027E0D5
:10ED100001C020E0FC01EE0FFF1FEE0FFF1FEE0F02
:10ED2000FF1FEC51F94C158636E03487262B2587DA
:10ED3000FC01EE0FFF1FEE0FFF1FEE0FFF1FEC5148
:10ED4000F94C2585207C203C69F4FC01EE0FFF1F67
:10ED5000EE0FFF1FEE0FFF1FEC51F94C25852770BA
:10ED6000273081F0880F991F880F991F880F991FEE
:10ED7000FC01EC51F94C85858062858781E008951E
:10ED800080E0089581E00895E82FEF70F0E0EE0F45
:10ED9000FF1F082E000C990B8827990F881F9927B1
:10EDA000E80FF91FEE0FFF1FEE0FFF1FEE0FFF1F03
:10EDB000EC51F94C858582FB882780F90895282F2E
:10EDC0002F7030E0A901440F551F282F082E000C8A
:10EDD000330B2227330F221F3327240F351FF9014E
:10EDE000EE0FFF1FEE0FFF1FEE0FFF1FEC51F94C50
:10EDF000958592FF17C0220F331F220F331F220F5A
:10EE0000331FF901EC51F94C95859B7F95877CDC8C
:10EE1000FC01808180FF06C08E7F80830780F085A3
:10EE2000E02D199581E008958F929F92AF92BF9245
:10EE3000CF92DF92EF92FF920F931F93CF93DF93C6
:10EE4000982E862E6A0179015FDC5C01292DC92D7F
:10EE5000CF70D0E0CE01880F991FC92D092C000C6E
:10EE6000DD0BCC27DD0FCC1FDD27C80FD91FFE011E
:10EE7000EE0FFF1FEE0FFF1FEE0FFF1FEC51F94CBF
:10EE80008585807C09F47EC0FE01EE0FFF1FEE0F2A
:10EE9000FF1FEE0FFF1FEC51F94C8585807C803CF5
:10EEA00061F0FE01EE0FFF1FEE0FFF1FEE0FFF1FC1
:10EEB000EC51F94C858582FD67C08FB7F894F50158
:10EEC000908190FF03C08FBF80E05FC0F50190810B
:10EED000916090838FBFC182D282E382F4821582D7
:10EEE000168207831087811006C091E0E114F104B7
:10EEF00019F090E001C091E0F501808190FB81F96B
:10EF00008B7F808322235CF4CC0FDD1FCC0FDD1FB1
:10EF1000CC0FDD1FCC51D94C1A8A1B8A2FC0FE01A1
:10EF2000EE0FFF1FEE0FFF1FEE0FFF1FEC51F94C0E
:10EF30008585807C803CB1F4CE01880F991F880FB5
:10EF4000991F880F991F8051994CB5DBBC01C701EF
:10EF50000F94C853892B31F0F50180818E7F808317
:10EF600080E013C0CC0FDD1FCC0FDD1FCC0FDD1FE9
:10EF7000CC51D94C1E861F861A8A1B8A892D4FDCDC
:10EF800081E003C080E001C080E0DF91CF911F915C
:10EF90000F91FF90EF90DF90CF90BF90AF909F9038
:10EFA0008F900895FF920F931F93CF93DF93182FA5
:10EFB000C82FCF70D0E0CE01880F991FC12F012E2E
:10EFC000000CDD0BCC27DD0FCC1FDD27C80FD91FB0
:10EFD000812F9ADBDC01FE01EE0FFF1FEE0FFF1FFA
:10EFE000EE0FFF1FE051F94C02E005938C9180FF7A
:10EFF00022C08E7F8C931796ED91FC9118973097D5
:10F00000D1F011235CF4CC0FDD1FCC0FDD1FCC0F32
:10F01000DD1FCC51D94C6A897B890AC0CC0FDD1F1A
:10F02000CC0FDD1FCC0FDD1FCC51D94C6E857F85F9
:10F03000412F81E01995DF91CF911F910F91FF90A2
:10F040000895CF93C82FAEDFEC2FEF70F0E0EE0FF6
:10F05000FF1F8C2FCC0F990B8827990F881F99279A
:10F06000E80FF91FEE0FFF1FEE0FFF1FEE0FFF1F40
:10F07000EC51F94C1586CF9108950F93E82FEF705E
:10F08000F0E0EE0FFF1F282F082E000C330B222775
:10F09000330F221F3327E20FF31FEE0FFF1FEE0F78
:10F0A000FF1FEE0FFF1FDF01AC51B94C1D969C9165
:10F0B0001D9794601D969C93E051F94C01E00693D6
:10F0C00071DF81E00F9108950F931F93CF93DF932A
:10F0D0008B01C82FCF70D0E0CC0FDD1F282F082E5A
:10F0E000000C330B2227330F221F3327C20FD31FED
:10F0F0000BDBCC0FDD1FCC0FDD1FCC0FDD1FCC5188
:10F10000D94C2D8522FF0AC0FC01208120FD0AC0B8
:10F11000216020830783108781E005C0F8011995DD
:10F1200081E001C080E0DF91CF911F910F910895A0
:10F130001F920F920FB60F9211240BB60F920F93DE
:10F140002F933F934F935F936F937F938F939F93EF
:10F15000AF93BF93EF93FF938091CB04882344F444
:10F1600080E88093CA040E949F610E94D55887C09E
:10F170008091CB0482FF20C084E08093CA048091F8
:10F18000F83686FF7CC08091CC0481FD78C0D7DA48
:10F19000811175C08091E336813011F40ADA6FC0B5
:10F1A000843009F06CC0E9EFF6E304E00593E1EF89
:10F1B000F6E304E0059363C08091CB0481FF5AC05D
:10F1C00082E08093CA048091F03686FF58C0809117
:10F1D000CC0481FD54C0B3DA811151C08091E33673
:10F1E000823041F484E08093E336E0EFF6E302E01E
:10F1F000069345C0833009F042C0E9EFF6E304E02E
:10F200000593E1EFF6E304E0059339C080E18093D4
:10F21000CA0481E0C7DE81E8C5DE0E9474611092F5
:10F22000C304E4EEF6E3158696E0948783E48587CD
:10F23000158A948B858B8FE996E3808B918B84D98B
:10F240001EC08091CB0486FF08C080E48093CA046E
:10F25000109224370E94D85812C08091CB0485FFA9
:10F260000EC080E28093CA0481E0809324370E941C
:10F27000D95805C08091CB0484FFE3CFC7CFFF915D
:10F28000EF91BF91AF919F918F917F916F915F911E
:10F290004F913F912F910F910F900BBE0F900FBE8A
:10F2A0000F901F9018951F920F920FB60F92112476
:10F2B0000BB60F920F931F932F933F934F935F9330
:10F2C0006F937F938F939F93AF93BF93CF93DF936E
:10F2D000EF93FF938091CC0481FD03C030DA81115C
:10F2E000C2C082E08093CC048091C5048195880FD0
:10F2F000E0EFF6E3E81BF10920813181205F36431E
:10F30000369527953695279536952795822F86959C
:10F3100020FD02C090E001C090E8890FE82FEF7057
:10F32000F0E0EE0FFF1F282F082E000C330B2227D2
:10F33000330F221F3327E20FF31FDF01AA0FBB1F7A
:10F34000AA0FBB1FAA0FBB1FAC51B94C1C969C91B6
:10F3500095FF89C0EE0FFF1FEE0FFF1FEE0FFF1F7F
:10F36000E051F94C00E20693811178C08091E336B8
:10F37000843019F42CD9E8D876C00091F236109177
:10F38000F3368091474090914840C091DF36D0914C
:10F39000E03698012C0F3D1F8217930718F48C015B
:10F3A0000C1B1D0B8091454090914640A8016FE9D0
:10F3B00076E38C0F9D1F0F942C56C00FD11FC09366
:10F3C000DF36D093E0360034110569F48091E136E0
:10F3D0009091E2368C0F9D1F209143403091444024
:10F3E0008217930780F0EDE3F0E4C287D3870684A9
:10F3F000F785E02D309729F01995811102C0CBD8FF
:10F4000032C0D7D830C08091474090914840C8174B
:10F41000D907F9F4E0914B40F0914C40309711F44A
:10F42000BAD821C01995811102C0B5D81CC020914D
:10F43000E1363091E2368091DF369091E036820FEE
:10F44000931F8093E1369093E2361092DF3610924C
:10F45000E036E0EFF6E302E0069305C0803811F4F1
:10F46000BED801C0DCD9FF91EF91DF91CF91BF9160
:10F47000AF919F918F917F916F915F914F913F914C
:10F480002F911F910F910F900BBE0F900FBE0F90F9
:10F490001F9018959091800024E0829FB001112464
:10F4A0006C7392709160692B80E890E00F94295101
:10F4B000E0E8F0E0828180FDFDCF0895609180005A
:10F4C0006C73636080E890E00F942951E0E8F0E00D
:10F4D000828180FDFDCF0895CF92DF92EF92FF925F
:10F4E000CF93DF93EC016B01E12CF12C60E070E62F
:10F4F0008AEE90E0A70196010F94EF53CA01B9017B
:10F500002FEF3FEF40E050E00F94EF53211531050E
:10F5100029F481E08C8321E030E02DC022303105D8
:10F5200028F482E08C8322E030E025C024303105CD
:10F5300028F483E08C8324E030E01DC028303105BE
:10F5400028F484E08C8328E030E015C020343105B5
:10F5500028F485E08C8320E430E00DC02F3F310596
:10F5600009F028F486E08C8320E031E004C087E0D5
:10F570008C8320E034E040E050E060E070E68AEE0A
:10F5800090E00F94EF53CA01B901A70196010F94BF
:10F59000EF532D833E832436310518F41C821D82DF
:10F5A0001E82DF91CF91FF90EF90DF90CF90089572
:10F5B0000F931F93CF93DF93EC018901862F90E087
:10F5C0008730910508F08BC0FC018827E752FE4F79
:10F5D0008F4F0D942D5480E098E088839983E0E468
:10F5E000F6E0308181E090E02FEF240F02C0880F19
:10F5F000991F2A95E2F7832B808371C080E498E0FD
:10F6000088839983E0E4F6E0308181E090E023E0B4
:10F61000240F02C0880F991F2A95E2F7832B80835D
:10F620005EC080E099E088839983E0E6F6E030816F
:10F6300081E090E02FEF240F02C0880F991F2A95D8
:10F64000E2F7832B80834BC080E499E08883998321
:10F65000E0E6F6E0308181E090E023E0240F02C094
:10F66000880F991F2A95E2F7832B808338C080E0AA
:10F670009AE088839983E0E8F6E0308181E090E0C9
:10F680002FEF240F02C0880F991F2A95E2F7832BD2
:10F69000808325C080E49AE088839983E0E8F6E0DF
:10F6A000308181E090E023E0240F02C0880F991F91
:10F6B0002A95E2F7832B808312C080E09BE0888349
:10F6C0009983E0EAF6E0308181E090E02FEF240FAB
:10F6D00002C0880F991F2A95E2F7832B80834A8303
:10F6E000423061F018F4413031F010C0433049F03D
:10F6F000443051F00BC080E18B8308C080E28B83E3
:10F7000005C080E48B8302C080E88B838881998167
:10F710000E942D6DE881F9818181887F83608183DA
:10F720001D821E821C82E881F9818081807F808316
:10F73000B801CE01D1DEDF91CF911F910F910895D5
:10F74000CF93DF93EC012D813E81A62FB0E00F9483
:10F75000355424E630E040E050E00F94EF538A81C6
:10F76000E881F981E6FD17C0823061F018F481303C
:10F7700031F01BC0833049F0843051F016C020AF07
:10F7800031AF13C022AF33AF10C024AF35AF0DC0BF
:10F7900026AF37AF0AC0813019F0823021F005C0A2
:10F7A00020AF31AF02C022AF33AF8D819E81E8819F
:10F7B000F98186A397A38B81E881F981E6FD04C0D6
:10F7C0009181892B818304C091818073892B8183EE
:10F7D000E881F9818081807F9C81892B8083DF9102
:10F7E000CF910895CF93DF93EC014115510509F4B2
:10F7F00043C0AAEAB2E420E030E0922FF901E159D7
:10F80000FB4EE491ED932F5F3F4F27303105A9F771
:10F81000FA01DE01CAEAD2E480818B8381818C8384
:10F82000F901E655FD4B8CE28083E2E0E90FF0E060
:10F83000E655FD4B6083C4E0C90F9D5FE92FF0E002
:10F84000E655FD4B8DE78083D0E0FE01E655FD4B8C
:10F85000108221E0AE016AEA72E4CD010F940C211E
:10F860000E94A62A811108C021E0AE016AEA72E472
:10F8700082E299E30F940C21DF91CF9108954F928A
:10F880005F926F927F928F929F92AF92BF92DF9220
:10F89000EF92FF920F931F93CF93DF931F92CDB7F9
:10F8A000DEB77C014115510509F466C188E0898302
:10F8B000AAEAB2E420E030E0922FF901E159FB4ED0
:10F8C000E491ED932F5F3F4F27303105A9F7FA01FF
:10F8D000162FAAEAB2E4808113968C931397818144
:10F8E00014968C9302E0090FF901E655FD4B8CE26A
:10F8F0008083623088F5862F0F9410088823B1F03A
:10F90000812F0F94D5079F938F931F921F9380E4AD
:10F9100099E29F938F93E02FF0E0E655FD4BFF9324
:10F92000EF930F945A56CDBFDEBF08C1812F0E94BE
:10F93000BDC19F938F931F921F9380E499E29F9381
:10F940008F93E02FF0E0E655FD4BFF93EF930F947C
:10F950005A56CDBFDEBFF2C0663109F078C086E1ED
:10F960000F9419072B013C010E94A3FE4B015C017F
:10F97000672B682B692BF1F4C301B20120E13EE053
:10F9800040E050E00F9411545F934F933F932F93B7
:10F990001F9286E18F9387E499E29F938F93E02FE4
:10F9A000F0E0E655FD4BFF93EF930F945A56CDBF11
:10F9B000DEBFC4C0802F0E9458C1992334F5C30113
:10F9C000B20120E13EE040E050E00F941154CA0142
:10F9D000B9010F948926BF92AF929F928F929F9305
:10F9E0008F937F936F931F9286E18F938FE499E2B9
:10F9F0009F938F93E02FF0E0E655FD4BFF93EF933D
:10FA00000F945A56CDBFDEBF99C0BF92AF929F925E
:10FA10008F92C301B20120E13EE040E050E00F943C
:10FA200011545F934F933F932F931F9286E18F93CF
:10FA30008CE599E29F938F93E02FF0E0E655FD4B24
:10FA4000FF93EF930F945A56CDBFDEBF77C0663059
:10FA500071F5E02FF0E0E655FD4B86E38083689476
:10FA6000DD24D2F8D90E9D5FE92FF0E0E655FD4B7D
:10FA70008CE2808386E00F9419078B019C018D2D09
:10FA800090E04BE0BE016F5F7F4F86559D4B0F941A
:10FA9000E226E981ED0DAE2FB0E0A655BD4B8DE716
:10FAA0008C93EF5FF0E0E655FD4B108247C0653068
:10FAB00071F5E02FF0E0E655FD4B85E38083689417
:10FAC000DD24D2F8D90E9D5FE92FF0E0E655FD4B1D
:10FAD0008CE2808385E00F9419078B019C018D2DAA
:10FAE00090E04BE0BE016F5F7F4F86559D4B0F94BA
:10FAF0002E28E981ED0DAE2FB0E0A655BD4B8DE768
:10FB00008C93EF5FF0E0E655FD4B108217C0862F17
:10FB10000F9419079F938F937F936F931F921F9357
:10FB200087E499E29F938F93802F90E086559D4BB9
:10FB30009F938F930F945A56CDBFDEBFEAEAF2E44B
:10FB400001900020E9F73197EA5AF244E983AF01C6
:10FB5000552721E06AEA72E4C7010F940C210E9444
:10FB6000A62A811109C0498150E021E06AEA72E4C5
:10FB700082E299E30F940C210F90DF91CF911F91B6
:10FB80000F91FF90EF90DF90BF90AF909F908F907C
:10FB90007F906F905F904F900895AC016115710553
:10FBA00071F1E8E7F4E1AAEAB2E422EB32E49491DD
:10FBB0009D933196A217B307D1F7FB01CA01AAEAB8
:10FBC000B2E4208113962C931397218114962C93E1
:10FBD000149718961C92189721E048E050E0BD0158
:10FBE0000F940C210E94A62A811109C021E048E04F
:10FBF00050E06AEA72E482E299E30D940C210895E0
:10FC0000EF92FF920F931F93CF93DF938C016115B7
:10FC1000710509F47FC04115510509F47BC0E6E682
:10FC2000F4E1AAEAB2E4C2EBD2E494919D93319656
:10FC3000AC17BD07D1F7FA017B01CAEAD2E4808193
:10FC40008B8381818C831F922F9388E699E29F9307
:10FC50008F9382EB92E49F938F930F945A5609905F
:10FC60000020E9F72197CA5AD244F70181810F9009
:10FC70000F900F900F900F900F90811115C0808101
:10FC80001F928F9386E791E29F938F93DD27C6554E
:10FC9000DD4BDF93CF930F945A560F900F900F9038
:10FCA0000F900F900F9016C01F928F93F7018081D5
:10FCB0001F928F9383E791E29F938F93DD27C65521
:10FCC000DD4BDF93CF930F945A56EDB7FEB73896BE
:10FCD000EDBFFEBFEAEAF2E401900020E9F73197B8
:10FCE000EA5AF244EF01DD2721E0AE016AEA72E44C
:10FCF000C8010F940C210E94A62A81110BC0025248
:10FD0000194341F021E0AE016AEA72E482E299E32C
:10FD10000F940C21DF91CF911F910F91FF90EF90E5
:10FD20000895CF93DF93EC014115510509F43FC0CD
:10FD3000662361F0E8E7F4E1AAEAB2E490E02491F6
:10FD40002D939F5F31969730D1F70BC0EFE6F4E12A
:10FD5000AAEAB2E490E024912D939F5F3196973008
:10FD6000D1F7DA01CE01EAEAF2E42C91238311966D
:10FD70002C9124832CE227833CE43087218720E3E5
:10FD800022872DE72387148621E04CE050E0BF0155
:10FD90000F940C210E94A62A811109C021E04CE099
:10FDA00050E06AEA72E482E299E30F940C21DF9159
:10FDB000CF910895EF92FF920F931F93CF93DF930C
:10FDC00000D01F92CDB7DEB70097C9F1663071053C
:10FDD000C0F1FC0120812035B1F521812C32A9F53B
:10FDE00024812C32A1F57A018C010B5F1F4FAB01EE
:10FDF000455051099E012F5F3F4FB8018CE20F948F
:10FE0000B926882349F149815A814B5F5F4F498365
:10FE10005A8346305105E8F045509E012D5F3F4F13
:10FE200060E0C8010F9441258823B1F08B819C814B
:10FE30008C31910580F4F701808381E00DC080E072
:10FE40000BC080E009C080E007C080E005C080E012
:10FE500003C080E001C080E02496CDBFDEBFDF910B
:10FE6000CF911F910F91FF90EF900895CF92DF9265
:10FE7000EF92FF920F931F93CF93DF93CDB7DEB72F
:10FE80002C97CDBFDEBF009709F431C166307105F4
:10FE900008F42FC1FC012081203509F02CC12181FB
:10FEA0002C3209F02AC124812C3209F028C17B01AF
:10FEB0008C016C01F5E0CF0ED11CAB01455051090E
:10FEC0009E012F5F3F4FB6018CE20F94B926982F09
:10FED000882309F423C149815A814B5F5F4F4983CD
:10FEE0005A834630510508F40CC145509E012D5FE0
:10FEF0003F4F60E0C6010F944125982F882309F4F5
:10FF00000DC12B813C812C31310508F0FCC04981A9
:10FF10005A81DA011196AE15BF0508F0F6C02C31F2
:10FF2000310508F0F4C0F9018827E052FE4F8F4FE9
:10FF30000D942D54C8018A0F9B1FFC0160816D3206
:10FF400041F4FA013296EE15FF0508F0E2C040E0F8
:10FF500002C0FD0141E02631310559F46E2D6E1BC2
:10FF60009E01275F3F4FC8018E0F9F1F0E940FF514
:10FF700012C02630310541F46E2D6A1BAE01475F79
:10FF80005F4F0E94DCF707C06E2D6A1BAE01475F12
:10FF90005F4F0E94F8F8882309F4BDC049855A854F
:10FFA0006B857C858B810E94ACC6982F882309F4D1
:10FFB000B5C049855A856B857C858B810F942C074C
:10FFC00091E0ACC04E2D4A1B9E012B5F3F4F60E07D
:10FFD000C8018A0F9B1F0F94CC25982F882309F402
:10FFE0009DC04D815E816F81788549875A876B8777
:10FFF0007C878B810E94ACC6982F882309F48EC021
:020000021000EC
:1000000089859A85AB85BC858B309105A105B105A5
:1000100049F48FE69CE30E94372F982F882309F438
:100020007DC00CC00C97A105B10544F08FE69CE3A0
:100030000E94372F982F882309F470C049855A856C
:100040006B857C858B810F942C0791E067C04E2DCA
:100050004A1B9E012B5F3F4F60E0C8018A0F9B1F28
:100060000F94CC25982F882309F458C04D815E81C8
:100070006F81788549875A876B877C878B810E943F
:10008000ACC6982F882349F049855A856B857C85B5
:100090008B810F942C0791E041C02B813C81A901F9
:1000A0004C50510946305105C8F549855A856B8534
:1000B0007C85452B462B472B89F540E050E0BA0163
:1000C000822F0F942C0791E029C0C7018A1B9B0B3C
:1000D000899718F56E2D6A1B422FC8018A0F9B1F46
:1000E0000F94970791E0811119C090E017C090E03C
:1000F00015C090E013C090E011C090E00FC090E0F8
:100100000DC090E00BC090E009C090E007C090E007
:1001100005C090E003C090E001C090E0892F2C96CC
:10012000CDBFDEBFDF91CF911F910F91FF90EF9078
:10013000DF90CF9008950F931F93CF93DF931F927B
:100140001F92CDB7DEB7009741F16630710538F1E7
:10015000FC012081203529F521812C3221F52481D3
:100160002C3219F58C01AB0145505109BC016B5F74
:100170007F4F9E012F5F3F4F8CE20F94B92688235B
:10018000B9F089819A810596069788F081E0F80197
:100190009581963469F080E00BC080E009C080E072
:1001A00007C080E005C080E003C080E001C080E0BF
:1001B0000F900F90DF91CF911F910F910895EF92C3
:1001C000FF920F931F93CF93DF9300D000D0CDB752
:1001D000DEB7009709F453C06630710508F451C0CA
:1001E000FC012081203509F04EC021812C3209F01C
:1001F0004CC024812C3209F04AC07B018C01AB0138
:1002000045505109BC016B5F7F4F9E012F5F3F4FEF
:100210008CE20F94B926882309F442C089819A811F
:100220009C012B5F3F4F29833A832630310588F1AB
:10023000F8012581263479F506968E159F0568F517
:100240004E2D481B9E012D5F3F4F60E0800F911F98
:100250000F94CC25882321F16B817C818D819E8137
:100260008B019C010150110921093109073E1340FE
:1002700021053105A0F40E9441C281E011C080E057
:100280000FC080E00DC080E00BC080E009C080E0BE
:1002900007C080E005C080E003C080E001C080E0CE
:1002A0002696CDBFDEBFDF91CF911F910F91FF90BA
:1002B000EF9008950F931F93CF93DF93EC01611597
:1002C000710509F444C0AAEAB2E420E030E0922FBC
:1002D000F901E159FB4EE491ED932F5F3F4F273039
:1002E0003105A9F7FB01AAEAB2E4808113968C9349
:1002F0001397818114968C931497F901E655FD4B61
:100300008CE280839E5FE92FF0E0E655FD4B86E4AA
:100310009DE7808391831282FD0101900020E9F71F
:100320003197EA5AF2448F01112721E0A801BD015B
:10033000CE010F940C210E94A62A811108C021E051
:10034000A8016AEA72E482E299E30F940C21DF913A
:10035000CF911F910F910895FC01892B61F06530B9
:10036000710558F08081803551F481E091819C3293
:1003700039F080E0089580E0089580E0089580E0FD
:100380000895009799F06330710590F0FC01208189
:10039000203581F421812C3279F424812C3271F4BE
:1003A00085818354823060F080E0089580E0089574
:1003B00080E0089580E0089580E0089580E0089549
:1003C00081E00895009791F06330710588F0FC0199
:1003D0002081203579F421812C3271F424812C3252
:1003E00069F485818F3461F080E0089580E008959C
:1003F00080E0089580E0089580E0089580E0089509
:1004000081E00895009791F06330710588F0FC0158
:100410002081203579F421812C3271F424812C3211
:1004200069F48581873561F080E0089580E0089562
:1004300080E0089580E0089580E0089580E00895C8
:1004400081E00895CF92DF92EF92FF920F931F9376
:10045000CF93DF934115510509F4AFC0009709F41C
:10046000AEC06630710508F4ACC0FC0120812035B7
:1004700009F0A9C021812C3209F0A7C024812C32B7
:1004800009F0A5C08581873509F0A3C0EA018FE690
:100490009CE30E944F14883009F49DC08FE69CE3D2
:1004A0000E944F14863009F498C00F9419190E94C5
:1004B000AA5361E085E79CE30E941E560F945408FE
:1004C0000E94351D813079F582E00E9466C16B0182
:1004D0007C01DD24EE24FF24B701A60182E00F9405
:1004E0002C07B701A60182E00E944EC10E94A62AF5
:1004F000811119C084E1ECE6F9E2A5E0B4E40190D1
:100500000D928A95E1F7E5E0F4E401900020E9F727
:100510003197AF014550544420E065E074E482E235
:1005200099E30F940C21CE010E94841C80E00E946C
:1005300034C19B01AC016894EE24E2F806EB12E2B0
:10054000BE01685E7F4FCE0106960E9478578D836C
:1005500040E050E0BA01CE010E94E72E8D81882351
:1005600051F182E00E9458C1062F8BE00E9458C1D1
:1005700021E0611120E044E150E4BE016C5C7F4F5A
:10058000CE01C6960E947B50CE010E945A1C9E014D
:10059000265A3D4FAE01475A5D4FBE016C5A7D4F02
:1005A000CE018D5A9D4F0E946E2D0E94A13368E0AE
:1005B000CE010E943C148D8111C080E00FC080E00C
:1005C0000DC080E00BC080E009C080E007C080E083
:1005D00005C080E003C080E001C080E0DF91CF91E2
:1005E0001F910F91FF90EF90DF90CF900895CF92E1
:1005F000DF92EF92FF920F93CF93DF934115510556
:1006000009F4B0C0009709F4AFC06630710508F472
:10061000ADC0FC012081203509F0AAC021812C3217
:1006200009F0A8C024812C3209F0A6C0EA01858116
:10063000833409F493C0843409F0A0C00E94F6C149
:100640000F94F2078FE69CE30E944F14883009F460
:1006500097C08FE69CE30E944F14863009F492C045
:100660000F9419190E94AA5361E085E79CE30E9448
:100670001E560F9454080E94351D813079F582E092
:100680000E9466C16B017C01DD24EE24FF24B701CA
:10069000A60182E00F942C07B701A60182E00E9418
:1006A0004EC10E94A62A811119C084E1ECE6F9E24C
:1006B000A5E0B4E401900D928A95E1F7E5E0F4E459
:1006C00001900020E9F73197AF014550544420E0F4
:1006D00065E074E482E299E30F940C2180E00E94CB
:1006E00034C19B01AC01BE01685E7F4FCE0106960E
:1006F0000E94B2538D8340E050E0BA01CE010E94C7
:10070000E72E8D81882341F182E00E9458C1062F97
:100710008BE00E9458C121E0611120E044E150E4E7
:10072000BE016C5C7F4FCE01C6960E947B50CE010D
:100730000E945A1C9E01265A3D4FAE01475A5D4FFA
:10074000BE016C5A7D4FCE018D5A9D4F0E946E2D79
:1007500068E0CE010E943C148D8115C00F94F20711
:1007600081E011C080E00FC080E00DC080E00BC0D0
:1007700080E009C080E007C080E005C080E003C0E1
:1007800080E001C080E0DF91CF910F91FF90EF906A
:10079000DF90CF900895BF92CF92DF92EF92FF92B9
:1007A0000F931F93CF93DF931F92CDB7DEB76115E1
:1007B000710509F464C0DB017C01EAEAF2E48BE72D
:1007C000808380E781838CE282839C91938311965E
:1007D0009C91948385839FE49683878380E00E9425
:1007E000B3C88B019C0148E0BE016F5F7F4F82EB75
:1007F00092E40F949028E981E85FD12C0F2EFCE25F
:10080000BF2EF02DCC24C394CE0EF0E0E655FD4B68
:10081000B082D3948D2D0E94B3C88B019C018C2D86
:1008200090E048E0BE016F5F7F4F86559D4B0F946F
:100830009028E981EC0D83E0D812E4CF81E08E0F9F
:10084000F0E0E655FD4B9DE79083482F50E0FA011C
:10085000E655FD4B1082898321E06AEA72E4C70104
:100860000F940C210E94A62A811109C0498150E0F1
:1008700021E06AEA72E482E299E30F940C210F907E
:10088000DF91CF911F910F91FF90EF90DF90CF906C
:10089000BF900895CF93DF9341155105A9F10097BB
:1008A000A9F165307105A0F1FC012081203591F599
:1008B00021812C3289F52281263481F5EA01848157
:1008C0008235E9F0833531F0843451F50E9420C23D
:1008D00081E027C00F941919BE016C5C7F4FCE01D7
:1008E000C6960E94804E8FE69CE30E94F122811101
:1008F0000F943B19CE010E943E2A8D8112C0CA017D
:10090000C6960E94FDFD0DC080E00BC080E009C0CE
:1009100080E007C080E005C080E003C080E001C047
:1009200080E0DF91CF910895FC01892B79F066304A
:10093000710570F08081833569F481818C3261F4B6
:1009400081E094819C3249F080E0089580E0089530
:1009500080E0089580E0089580E008950F93CF939C
:10096000DF93009709F476C06630710508F474C00F
:10097000FC016081633509F071C061816C3209F05E
:100980006FC064816C3209F06DC04115510509F4E6
:100990006BC02115310509F469C08581813309F0E7
:1009A00067C0B901EA01F9011082CA010E94D8208A
:1009B000882309F45FC0CE010E94B92081112BC0A9
:1009C000CE010E943E2A61E0CE010E94692764E0C8
:1009D000CE010E943C1461E0CE010E94AA2019823F
:1009E0000E9487A2E6EEF2E4808190E0DC01AA5149
:1009F000BD4B25853685880F991FFC01EA51FD4BBB
:100A0000418152811F960C9161E08FE69CE30E9428
:100A1000582581E032C00E94A62A81112DC083E1B1
:100A2000E0E8F9E2AAEAB2E401900D928A95E1F7D2
:100A3000EAEAF2E401900020E9F73197AF014A5A5F
:100A4000524421E06AEA72E482E299E30F940C21B5
:100A500081E013C080E011C080E00FC080E00DC0D5
:100A600080E00BC080E009C080E007C080E005C0E6
:100A700080E003C081E001C081E0DF91CF910F9160
:100A800008950F93CF93DF93009709F45EC166300A
:100A9000710508F45CC1DC012C91233509F059C1C2
:100AA00011962C9111972C3209F055C114962C9166
:100AB00014972C3209F051C14115510509F44FC169
:100AC0001596EC918E2F90E0FC01F097E534F1053E
:100AD00008F047C1EA018827E450FE4F8F4F0D947C
:100AE0002D54CA010E944F14843031F0CE010E946F
:100AF0004F14893009F037C1CE010E943620CE0153
:100B00000F940B0BCE010E943E2A0F94191960E03E
:100B10008FE69CE30E94692763E0CE010E943C14AB
:100B200019820E9474A2E6EEF2E4808190E0DC017A
:100B3000AA51BD4B25853685880F991FFC01EA51C6
:100B4000FD4B418152811F960C9161E08FE69CE341
:100B50000E94582591E016C1CA010E94B92088233D
:100B600009F403C181E0898360E0CE010E943E1553
:100B700060E0CE010E942C150E94A62A8111F7C0C8
:100B800080E1E3E9F9E2AAEAB2E401900D928A95E4
:100B9000E1F7EAEAF2E401900020E9F73197AF01CA
:100BA0004A5A524421E06AEA72E482E299E30F94DD
:100BB0000C2191E0E7C0CA010E94B920882309F402
:100BC000D8C060E0CE010E943E1560E0CE010E94D8
:100BD0002C15FE01ED5AFD4FDE01A75ABD4F8C9139
:100BE0008083319611968C91808319820E94A62A67
:100BF0008111C1C080E1E3EAF9E2AAEAB2E401901E
:100C00000D928A95E1F7EAEAF2E401900020E9F713
:100C10003197AF014A5A524421E06AEA72E482E213
:100C200099E30F940C2191E0ADC0CA010E94B92054
:100C3000982F882309F4A6C0CE010E94062891E0CF
:100C40008111A0C090E09EC0CA010E94B9208823F3
:100C500029F0CE010E949027982F94C00E9405C9C8
:100C600091E090C0CA010E94B920982F882309F40E
:100C700089C00F94191960E08FE69CE30E946927F0
:100C800069E0CE010E943C141982CE010F941B0B27
:100C9000CE010E94EE1CCE010F94B50F0F941D1CC7
:100CA00061E0CE010E94AA2091E06CC0CA010E94BE
:100CB0004F14893009F061C064E170E4CE010F94F3
:100CC000520FCE010F94120B843109F058C0CE019F
:100CD0000F941B0BCE010F94B50F0F941D1C91E0C8
:100CE00051C0CA010E944F14893009F04AC0CE0198
:100CF0000F940B0BCE010E943E2A61E0CE010E94B0
:100D0000692764E0CE010E943C1461E0CE010E949C
:100D1000AA2019820E9487A2E6EEF2E4808190E088
:100D2000DC01AA51BD4B25853685880F991FFC0132
:100D3000EA51FD4B418152811F960C9161E08FE693
:100D40009CE30E94582591E01DC090E01BC090E0FC
:100D500019C090E017C090E015C090E013C090E07B
:100D600011C090E00FC091E00DC091E00BC091E088
:100D700009C091E007C091E005C090E003C091E098
:100D800001C090E0892FDF91CF910F910895FC0170
:100D9000892B61F06630710558F080818D3451F4F3
:100DA00081E091819C3239F080E0089580E00895DF
:100DB00080E0089580E00895FC01892B61F06630A1
:100DC000710558F08081823551F481E091819C3227
:100DD00039F080E0089580E0089580E0089580E093
:100DE0000895FC01892B61F06530710558F0808110
:100DF0008A3551F481E091819C3239F080E0089588
:100E000080E0089580E0089580E00895CF92DF9219
:100E1000EF92FF920F931F93CF93DF93CDB7DEB77F
:100E20002897CDBFDEBF009709F457C06530710524
:100E300008F455C0FC0120812A3509F052C02181F7
:100E40002C3209F050C07B018C016C01F2E0CF0E16
:100E5000D11CAB01425051099E012F5F3F4FB6019B
:100E60008CE20F94B926882309F446C049815A813F
:100E70004E5F5F4F49835A8343305105B0F1425072
:100E80009E012D5F3F4F60E0C6010F9441258823EE
:100E900099F18B819C81039750F589819A81019604
:100EA0008E159F0530F54E2D481B9E012B5F3F4F41
:100EB00060E0800F911F0F94CC258823E9F06D81AD
:100EC0007E818F819885623071058105910598F446
:100ED0008B810E94FEDD81E00FC080E00DC080E0CC
:100EE0000BC080E009C080E007C080E005C080E062
:100EF00003C080E001C080E02896CDBFDEBFDF9157
:100F0000CF911F910F91FF90EF90DF90CF900895B8
:100F10002F923F924F925F926F927F928F929F9209
:100F2000AF92BF92CF92DF92EF92FF920F931F93F7
:100F3000CF93DF93CDB7DEB76397CDBFDEBF8C0114
:100F4000F62E81E08D830115110509F423C38093EA
:100F5000CE2089E10E9458C1672B682B692B09F0CC
:100F600025C30F943201B82E811103C0F11020C3A4
:100F700085C38FE69CE30E942B21B82E882309F4B9
:100F80007DC38FE69CE30E944F148F87F11004C04D
:100F90008150823008F400C32F85243031F48FE66D
:100FA0009CE30E94842A33E03F870F94F5080F9456
:100FB000DE088FE69CE30E94F12281110F943B1919
:100FC0008FE69CE30E943E2A82E00E9458C1E62EF2
:100FD0008FEF8E0D8A3008F0E1C2AE014A5F5F4F9D
:100FE000BE016B5F7F4F8E2D0E9466228E810E9414
:100FF00069DD8E8184700E94DDDD8D810F94500348
:101000000F2EFAEACF2EF2E4DF2EF02D8BE7D60179
:101010008C938DE611968C9311978CE212968C939B
:10102000129787E713968C9320E044E050E0B601D6
:10103000C8010F940C211F92EF9283EB99E29F93CA
:101040008F93DF92CF920F945A56F60101900020B1
:10105000E9F73197AF014A5A524420E0B601C8017E
:101060000F940C21ECE5F3E587858F9386858F93AC
:1010700085858F9384858F930F2EF7EBAF2EF9E242
:10108000BF2EF02DBF92AF92DF92CF920F945A569F
:10109000F60101900020E9F73197AF014A5A524416
:1010A00020E0B601C8010F940C218AE00E9458C1CB
:1010B0009F938F937F936F93BF92AF92DF92CF9264
:1010C0000F945A56F60101900020E9F73197AF01CD
:1010D0004A5A524420E0B601C8010F940C218BE01B
:1010E0000E9458C19F938F937F936F93BF92AF924B
:1010F000DF92CF920F945A56F60101900020E9F743
:101100003197AF014A5A524420E0B601C8010F940A
:101110000C210F2EF6E7CF2EF3E5DF2EF02DCDBFFD
:10112000DEBF412C512C320145010F2EFAEAAF2EC1
:10113000F2E4BF2EF02D2BC0D6018C9111969C911C
:10114000119712962C91129713963C91B4E0CB0E06
:10115000D11C3F932F939F938F939F928F92BF9217
:10116000AF920F945A56F50101900020E9F731979C
:10117000AF014A5A524420E0B501C8010F940C2136
:10118000EFEF4E1A5E0A6E0A7E0ACDBFDEBF0F94E5
:101190001A1C90E0A0E0B0E0481659066A067B06EB
:1011A00058F28DE78093AA4221E041E050E06AEADC
:1011B00072E4C8010F940C2165E08FE69CE30E9465
:1011C0003C140F9419198FE69CE30E9443250E945A
:1011D000575960E072E080E090E00E94495A109216
:1011E0004D4010924E408BEF92E40E9418A80E944E
:1011F000EA5B8111FCCFB82EF11004C00E941E20C2
:101200008823E1F389E00E9458C16F31710581059F
:10121000910508F59B01AC01012E1CE0220F331F44
:10122000441F551F1A95D1F7102D2B873C874D87EA
:101230005E87CA01B9010F9497080F94E31981E002
:101240000F94331C80E090E1A0E0B0E08F8398879A
:10125000A987BA873FC09B01AC01012E19E0220F7C
:10126000331F441F551F1A95D1F7102D2B873C872C
:101270004D875E87CA01B9010F9497080F94E3194F
:101280000F94631C80E092E0A0E0B0E08F83988729
:10129000A987BA871FC0412C512C32019F2CCB84C7
:1012A000DC84ED84FE840F94A01C8823E1F08D8102
:1012B0000F940D186BEF72E40E947BA8A82E0F9478
:1012C0008F1C9FEF491A590A690A790AA1100BC0AD
:1012D000F92C0FC02B853C854D855E85232B242B57
:1012E000252BC9F606C04C145D046E047F04D8F2A9
:1012F000F92C0F948A1C8BEF92E40E94DFA8E82E51
:101300000E94D65A0F94DE15EE2031F06F858FE6DD
:101310009CE30E943C14B2C184E295E40E94F5CEA5
:10132000882351F0F11008C06091234670E084E2F8
:1013300095E40E943FA909C0EAEAF2E41082118212
:1013400062E070E0CF010E943FA960E072E080E0BF
:1013500090E00E945F590E94EA5B8111FCCF8B856F
:101360009C85AD85BE85892B8A2B8B2B09F4F3C018
:10137000C12CD12C76010F2EFAEA2F2EF2E43F2E4B
:10138000F02D4F80588469847A8491E0491A51087D
:10139000610871080E942EA980934D4090934E40A1
:1013A000AE014F5F5F4FBC018D810E9450158823B5
:1013B00009F463C1C701B6012F81388549855A8573
:1013C0000F94EF534B015C01672B682B692BA1F540
:1013D000C701B6012F81388549855A850F94EF538F
:1013E000288B398B4A8B5B8B89E00E9458C1AB8973
:1013F000AF93BA89BF93E989EF93F889FF939F93DD
:101400008F937F936F932CEB39E23F932F933F920F
:101410002F920F945A56F10101900020E9F731976D
:10142000AF014A5A524420E0B101C8010F940C2187
:101430001092CE20CDBFDEBF2F81388549855A85D9
:10144000211582E038074105510509F4BAC021157C
:1014500030414105510509F4DDC0D701C60187704F
:101460009927AA27BB27892B8A2B8B2B09F043C0EE
:101470008C818F938B818F938A818F9389818F93B6
:10148000A7ECBAE2BF93AF933F922F920F945A56B4
:10149000F10101900020E9F73197AF014A5A524417
:1014A00020E0B101C8010F940C21C701B6012F81C2
:1014B000388549855A850F94EF532F5F3F4F4F4F23
:1014C0005F4F6F81788589859A850F94AD53CDBF25
:1014D000DEBFA7019601285F3F4F4F4F5F4F621756
:1014E00073078407950719F41092CE20C0C031E02D
:1014F0003093CE20BCC01092CE2084149504A60454
:10150000B70479F4EDE7D101EC9321E041E050E03C
:10151000B101C8010F940C210FC0ECE2D101EC9392
:1015200004C08091CE20882339F020E041E050E0D3
:10153000B101C8010F940C21FFEFCF1ADF0AEF0AA7
:10154000FF0A2B853C854D855E85C216D306E406D1
:10155000F50609F01FCF0E942A5A0F94DE150F944A
:10156000392A84E190E40F94FF4B6F858FE69CE36A
:101570000E943C140F946C098FE69CE30E94F122B8
:1015800081110F943B198FE69CE30E943E2ABB24F5
:10159000B39474C0B12C72C0B12C70C0B12C6EC0A9
:1015A0008FE69CE30E944F148F87F6CCFF24F394C0
:1015B0008FE69CE30E942B21B82E882309F45EC09D
:1015C000EFCF8C818F938B818F938A818F938981C9
:1015D0008F9347EC5AE25F934F933F922F920F9471
:1015E0005A56F10101900020E9F73197AF014A5AAC
:1015F000524420E0B101C8010F940C2191E0909376
:10160000CE20CDBFDEBF481459046A047B0409F024
:1016100084CF78CF8C818F938B818F938A818F93A6
:1016200089818F93E7ECFAE2FF93EF933F922F9239
:101630000F945A56F10101900020E9F73197AF015C
:101640004A5A524420E0B101C8010F940C2131E004
:101650003093CE20CDBFDEBF481459046A047B040A
:1016600009F05BCF4FCFECE2D101EC935ACF841459
:101670009504A604B704B9F745CFB82E8B2D639611
:10168000CDBFDEBFDF91CF911F910F91FF90EF9003
:10169000DF90CF90BF90AF909F908F907F906F9092
:1016A0005F904F903F902F900895CF92DF92EF92EE
:1016B000FF921F93CF93DF936115710509F474C0F6
:1016C0004630510508F472C0DB01EC91ED3409F0AD
:1016D0006FC01196EC91EC3209F06CC02115310508
:1016E00009F46AC0009709F469C069017A01EB0145
:1016F0002D81203341F440E060E00ADC11E08111EB
:1017000060C010E05EC0233541F5C6010E9438215B
:10171000182F882309F455C0C7010697029718F4BB
:101720000E9400AA0CC08E818C3219F00E9400AA7F
:1017300006C069EF6E0DCE0107960E94CBA9A601E7
:10174000485E5F4FB6016A5C7F4F80E00E94134A9B
:1017500011E0811136C010E034C00E94A62A182F73
:1017600081112EC08D811F928F9388EC99E29F93F7
:101770008F93CAEAD2E4DF93CF930F945A5609901D
:101780000020E9F72197AE014A5A524421E06AEA63
:1017900072E482E299E30F940C210F900F900F9066
:1017A0000F900F900F900DC010E00BC010E009C01B
:1017B00010E007C010E005C010E003C010E001C059
:1017C00010E0812FDF91CF911F91FF90EF90DF907C
:1017D000CF900895FC01892BA9F068307105A0F025
:1017E0008081813599F481818C3291F484818C32AD
:1017F00089F486818C3281F481E09581903369F09F
:1018000080E0089580E0089580E0089580E00895E4
:1018100080E0089580E0089580E00895EF92FF92BF
:101820000F931F93CF93DF9300D0CDB7DEB79CE229
:101830009B8321153105A9F161157105A1F1FA010B
:101840003197F39790F5823390F5803391F5C90184
:101850007A018B010E944F14843069F59E012F5F3D
:101860003F4F41E050E0BE016D5F7F4F84E190E467
:101870000F94514A9E012F5F3F4FA701B80184E1A9
:1018800090E40F94514A84E190E40F94FF4B0F943D
:10189000D21B8FE490E40E94FF9F0F94A81A81E06E
:1018A0000BC080E009C080E007C080E005C080E098
:1018B00003C081E001C080E02396CDBFDEBFDF9191
:1018C000CF911F910F91FF90EF900895FC01892B0C
:1018D00061F06330710558F080818C3451F481E0FF
:1018E00091819C3239F080E0089580E0089580E095
:1018F000089580E00895452BB1F00097B1F0672B73
:10190000B1F0FC0185818136A1F484E991E40E9463
:1019100032A0811110C060E070E084E991E40E947F
:101920003DA081E0089580E0089580E0089580E082
:10193000089580E0089580E00895CF93DF93452BCC
:10194000C9F10097C9F165317105C0F1FC0125812C
:101950002037B1F52781203319F41092A24109C034
:10196000213321F421E02093A24103C022E02093FF
:10197000A241EC0184E991E40E9432A0811122C0CD
:101980000E94F333811109C0BE01675F7F4F84E974
:1019900091E40E943DA081E018C08091A241811194
:1019A00013C0BE01675F7F4F8DEC9EE30E94A0A134
:1019B00081E00BC080E009C080E007C080E005C086
:1019C00080E003C080E001C081E0DF91CF91089505
:1019D000CF93DF93452B61F1009761F1653171057C
:1019E00058F1FC0125812E3649F52781203319F461
:1019F0001092A24109C0213321F421E02093A24199
:101A000003C022E02093A241EC0184E991E40E940A
:101A100032A0811115C08091A241882399F0BE01A6
:101A2000675F7F4F84E991E40E945EA081E00BC074
:101A300080E009C080E007C080E005C080E003C00E
:101A400080E001C081E0DF91CF910895009799F087
:101A50006630710590F0FC018581833681F484E95C
:101A600091E40E9432A0882361F00E94B39E1092FC
:101A7000944181E0089580E0089580E0089580E039
:101A8000089581E00895FC01892B49F066307105C5
:101A900040F081E09581933729F080E0089580E05F
:101AA000089580E00895FC01892B49F066307105A6
:101AB00040F081E09581953629F080E0089580E03E
:101AC000089580E00895BF92CF92DF92EF92FF9247
:101AD0000F931F93CF93DF9300D0CDB7DEB79CE277
:101AE0009B83882359F000918241002311F010E07C
:101AF00009C000914F401091504004C000918341B3
:101B0000109184410D3291E0190710F00CE211E0C0
:101B10000115110509F44CC0B82E9E012F5F3F4FEF
:101B200041E050E0BE016D5F7F4F84E190E40F948F
:101B3000514A109251401092524020E030E0C12CA6
:101B4000D12C0F2EFFE4EF2EF0E4FF2EF02DF90143
:101B5000E15BFF4B95819B839E012F5F3F4F41E0EF
:101B600050E0BE016D5F7F4F84E190E40F94514AD5
:101B700029813A81232B19F4EFEFCE1ADE0AF701FF
:101B8000228133812F5F3F4F228333832017310718
:101B9000F0F284E190E40F94FF4BB11004C0109276
:101BA00083411092844181E0CD2819F080E001C08A
:101BB00080E02396CDBFDEBFDF91CF911F910F91C3
:101BC000FF90EF90DF90CF90BF900895FC01892B9C
:101BD00049F06630710540F081E09581943629F036
:101BE00080E0089580E0089580E00895EAEAF2E454
:101BF0002BE720832CE621832CE22283662321F02D
:101C00002FE62093AD4203C025E62093AD42EAEAD9
